:020000040800F2
:104000000000022069010208D1E10108D9E101089C
:10401000E1E10108E9E10108F1E101080000000027
:10402000000000000000000000000000F9E10108AD
:1040300007E201080000000015E2010823E2010880
:10404000B9010208B9010208B9010208B901020860
:10405000B9010208B901020835E20108B9010208F4
:10406000B9010208B9010208B9010208B901020840
:10407000B9010208B9010208B9010208B901020830
:10408000B9010208B901020855E20108B9010208A4
:10409000B9010208B9010208B9010208B901020810
:1040A0008DE20108B9E20108DDE20108B901020868
:1040B00001E30108B901020825E3010849E3010809
:1040C0006DE30108B9010208B901020891E3010892
:1040D000B9010208B9010208B5E30108D9E30108F2
:1040E000FDE30108B9010208B901020825E401084D
:1040F00039E401085DE40108B9010208B9010208C8
:10410000B9010208B9010208B9010208B90102089F
:10411000B9010208B9010208B9010208B90102088F
:1041200081E40108B9010208B9010208B9010208D5
:10413000B90102080000000000000000B9010208F7
:10414000B9010208B9010208B9010208B90102085F
:10415000B9010208B9010208B9010208B90102084F
:10416000B9010208B9010208B9010208B90102083F
:10417000B9010208B9010208B901020800000000F3
:1041800000000000B901020800000000000000006B
:10419000A5E401080000000000000000B9010208C9
:1041A000000000000000000000000000B90102084B
:1041B000B9010208B9010208B9010208B9010208EF
:0441C000B901020837
:1080000001030100E90706300A01004000000000FA
:10801000000000000000000090BD2A3D0000803FED
:108020005839343C0000803F0000803F5839343CD0
:108030000000803FE02D103BACC52737D245E3431D
:10804000000000406F12033B0000B43C00606A4037
:108050000000B4420000804300000000FF0FFF0F4B
:10806000000000000000803F0000803F6740533A5E
:108070000821043D90C2F53C17B7D138009C0C464E
:1080800000A08C456666663F00007A4400401C46AE
:108090000000204100401C460000C84200007A4415
:1080A0000040744500003A4300000C420000FA45CD
:1080B00000008C420000F0410020034500C0F9445C
:1080C000000044420000E0410000C8450000E041DB
:1080D00000004040000070420000F04100A0254533
:1080E0000000003F0000A0410000803F6666E63EC1
:1080F0000000A0C10000B442FFFFFFFF7856341219
:10810000000000000000000000000000000000006F
:10811000000000000000000000000000000000005F
:10812000000000000000000000000000000000004F
:10813000000000000000000000000000000000003F
:10C0000001030100E90706300A01004000000000BA
:10C01000000000000000000090BD2A3D0000803FAD
:10C020005839343C0000803F0000803F5839343C90
:10C030000000803FE02D103BACC52737D245E343DD
:10C04000000000406F12033B0000B43C00606A40F7
:10C050000000B4420000804300000000FF0FFF0F0B
:10C06000000000000000803F0000803F6740533A1E
:10C070000821043D90C2F53C17B7D138009C0C460E
:10C0800000A08C456666663F00007A4400401C466E
:10C090000000204100401C460000C84200007A44D5
:10C0A0000040744500003A4300000C420000FA458D
:10C0B00000008C420000F0410020034500C0F9441C
:10C0C000000044420000E0410000C8450000E0419B
:10C0D00000004040000070420000F04100A02545F3
:10C0E0000000003F0000A0410000803F6666E63E81
:10C0F0000000A0C10000B442FFFFFFFF78563412D9
:10C10000000000000000000000000000000000002F
:10C11000000000000000000000000000000000001F
:10C12000000000000000000000000000000000000F
:10C1300000000000000000000000000000000000FF
:020000040801F1
:1000000010B5054C237833B9044B13B10448AFF352
:1000100000800123237010BD940000200000000028
:100020009C9E020808B5034B1BB103490348AFF37C
:10003000008008BD00000000980000209C9E02087F
:1000400001F0FF01102A2BDB10F0070F08D010F889
:10005000013B013A8B422DD010F0070F42B3F6D18D
:10006000F0B441EA012141EA014122F007047FF0A6
:1000700000070023F0E80256083C85EA010586EAFD
:10008000010685FA47F5A3FA87F586FA47F6A5FA39
:1000900087F68EB9EED1F0BC01F0FF0102F0070245
:1000A00032B110F8013B013A83EA010313B1F8D1F0
:1000B0000020704701387047002D06BF35460338D1
:1000C000073815F0010F07D1013015F4807F02BF0A
:1000D000013015F4C03F0130F0BC0138704700BF5B
:1000E00081F0004102E000BF83F0004330B54FEAE9
:1000F00041044FEA430594EA050F08BF90EA020F56
:100100001FBF54EA000C55EA020C7FEA645C7FEAE8
:10011000655C00F0E2804FEA5454D4EB5555B8BF0B
:100120006D420CDD2C4480EA020281EA030382EA7C
:10013000000083EA010180EA020281EA0303362D0E
:1001400088BF30BD11F0004F4FEA01314FF4801CE1
:100150004CEA113102D0404261EB410113F0004FF3
:100160004FEA03334CEA133302D0524263EB4303AA
:1001700094EA050F00F0A780A4F10104D5F1200E48
:100180000DDB02FA0EFC22FA05F2801841F10001A3
:1001900003FA0EF2801843FA05F359410EE0A5F177
:1001A00020050EF1200E012A03FA0EFC28BF4CF0A8
:1001B000020C43FA05F3C01851EBE37101F000455E
:1001C00007D54FF0000EDCF1000C7EEB00006EEB6B
:1001D0000101B1F5801F1BD3B1F5001F0CD34908F5
:1001E0005FEA30004FEA3C0C04F101044FEA44524C
:1001F00012F5800F80F09A80BCF1004F08BF5FEAD3
:10020000500C50F1000041EB045141EA050130BDB2
:100210005FEA4C0C404141EB0101013C28BFB1F5C4
:10022000801FE9D291F0000F04BF01460020B1FA0F
:1002300081F308BF2033A3F10B03B3F120020CDAE2
:100240000C3208DD02F1140CC2F10C0201FA0CF0C0
:1002500021FA02F10CE002F11402D8BFC2F1200C25
:1002600001FA02F120FA0CFCDCBF41EA0C019040DB
:10027000E41AA2BF01EB0451294330BD6FEA040424
:100280001F3C1CDA0C340EDC04F11404C4F120020F
:1002900020FA04F001FA02F340EA030021FA04F321
:1002A00045EA030130BDC4F10C04C4F1200220FA78
:1002B00002F001FA04F340EA0300294630BD21FAB6
:1002C00004F0294630BD94F0000F83F4801306BF7C
:1002D00081F480110134013D4EE77FEA645C18BF70
:1002E0007FEA655C29D094EA050F08BF90EA020F07
:1002F00005D054EA000C04BF1946104630BD91EAFF
:10030000030F1EBF0021002030BD5FEA545C05D101
:100310004000494128BF41F0004130BD14F5800440
:100320003CBF01F5801130BD01F0004545F0FE41B4
:1003300041F470014FF0000030BD7FEA645C1ABFE9
:10034000194610467FEA655C1CBF0B46024650EA20
:10035000013406BF52EA033591EA030F41F400214C
:1003600030BD00BF90F0000F04BF0021704730B5D2
:100370004FF4806404F132044FF000054FF00001A7
:1003800050E700BF90F0000F04BF0021704730B568
:100390004FF4806404F1320410F0004548BF40423D
:1003A0004FF000013EE700BF42004FEAE2014FEA92
:1003B00031014FEA02701FBF12F07F4393F07F4F6D
:1003C00081F06051704732F07F4208BF704793F070
:1003D0007F4F04BF41F40021704730B54FF4607483
:1003E00001F0004521F000411CE700BF50EA010286
:1003F00008BF704730B54FF000050AE050EA01022F
:1004000008BF704730B511F0004502D5404261EB9E
:1004100041014FF4806404F132045FEA915C3FF4DF
:10042000D8AE4FF003025FEADC0C18BF03325FEA7C
:10043000DC0C18BF033202EBDC02C2F1200300FA2D
:1004400003FC20FA02F001FA03FE40EA0E0021FA52
:1004500002F11444BDE600BF70B54FF0FF0C4CF440
:10046000E06C1CEA11541DBF1CEA135594EA0C0FF2
:1004700095EA0C0F00F0DEF82C4481EA030621EA2D
:100480004C5123EA4C5350EA013518BF52EA033568
:1004900041F4801143F4801338D0A0FB02CE4FF01A
:1004A0000005E1FB02E506F00042E0FB03E54FF04A
:1004B0000006E1FB03569CF0000F18BF4EF0010E42
:1004C000A4F1FF04B6F5007F64F5407404D25FEA3E
:1004D0004E0E6D4146EB060642EAC62141EA5551F1
:1004E0004FEAC52040EA5E504FEACE2EB4F1FD0C33
:1004F00088BFBCF5E06F1ED8BEF1004F08BF5FEAB1
:10050000500E50F1000041EB045170BD06F0004662
:1005100046EA010140EA020081EA0301B4EB5C040F
:10052000C2BFD4EB0C0541EA045170BD41F4801107
:100530004FF0000E013C00F3AB8014F1360FDEBF2C
:10054000002001F0004170BDC4F10004203C35DA08
:100550000C341BDC04F11404C4F1200500FA05F38B
:1005600020FA04F001FA05F240EA020001F000422C
:1005700021F0004110EBD37021FA04F642EB0601A2
:100580005EEA430E08BF20EAD37070BDC4F10C04CC
:10059000C4F1200500FA04F320FA05F001FA04F290
:1005A00040EA020001F0004110EBD37041F100017C
:1005B0005EEA430E08BF20EAD37070BDC4F1200587
:1005C00000FA05F24EEA020E20FA04F301FA05F2EF
:1005D00043EA020321FA04F001F0004121FA04F297
:1005E00020EA020000EBD3705EEA430E08BF20EA67
:1005F000D37070BD94F0000F0FD101F000464000A1
:1006000041EB010111F4801F08BF013CF7D041EA22
:10061000060195F0000F18BF704703F00046520026
:1006200043EB030313F4801F08BF013DF7D043EAF7
:100630000603704794EA0C0F0CEA135518BF95EAAD
:100640000C0F0CD050EA410618BF52EA4306D1D134
:1006500081EA030101F000414FF0000070BD50EA53
:10066000410606BF1046194652EA430619D094EADD
:100670000C0F02D150EA013613D195EA0C0F05D1C7
:1006800052EA03361CBF104619460AD181EA03011B
:1006900001F0004141F0FE4141F470014FF00000D3
:1006A00070BD41F0FE4141F4780170BD70B54FF06E
:1006B000FF0C4CF4E06C1CEA11541DBF1CEA1355EE
:1006C00094EA0C0F95EA0C0F00F0A7F8A4EB0504D0
:1006D00081EA030E52EA03354FEA013100F08880C7
:1006E0004FEA03334FF0805545EA131343EA126390
:1006F0004FEA022245EA111545EA10654FEA002645
:100700000EF000419D4208BF964244F1FD0404F5FD
:10071000407402D25B084FEA3202B61A65EB030559
:100720005B084FEA32024FF480104FF4002CB6EB16
:10073000020E75EB030E22BFB61A754640EA0C0096
:100740005B084FEA3202B6EB020E75EB030E22BFD6
:10075000B61A754640EA5C005B084FEA3202B6EB17
:10076000020E75EB030E22BFB61A754640EA9C00D6
:100770005B084FEA3202B6EB020E75EB030E22BFA6
:10078000B61A754640EADC0055EA060E18D04FEA64
:10079000051545EA16754FEA06164FEAC30343EA04
:1007A00052734FEAC2025FEA1C1CC0D111F4801FD1
:1007B0000BD141EA00014FF000004FF0004CB6E7CA
:1007C00011F4801F04BF01430020B4F1FD0C88BF69
:1007D000BCF5E06F3FF6AFAEB5EB030C04BFB6EB74
:1007E000020C5FEA500C50F1000041EB045170BD67
:1007F0000EF0004E4EEA113114EB5C04C2BFD4EB94
:100800000C0541EA045170BD41F480114FF0000E17
:10081000013C90E645EA060E8DE60CEA135594EA93
:100820000C0F08BF95EA0C0F3FF43BAF94EA0C0F96
:100830000AD150EA01347FF434AF95EA0C0F7FF40B
:1008400025AF104619462CE795EA0C0F06D152EA5F
:1008500003353FF4FDAE1046194622E750EA410643
:1008600018BF52EA43067FF4C5AE50EA41047FF454
:100870000DAF52EA43057FF4EBAE12E74FF0FF3CB9
:1008800006E000BF4FF0010C02E000BF4FF0010C8A
:100890004DF804CD4FEA410C7FEA6C5C4FEA430C03
:1008A00018BF7FEA6C5C1BD001B050EA410C0CBF52
:1008B00052EA430C91EA030F02BF90EA020F0020B4
:1008C000704710F1000F91EA030F58BF994208BF1B
:1008D00090422CBFD8176FEAE37040F001007047D8
:1008E0004FEA410C7FEA6C5C02D150EA013C07D12F
:1008F0004FEA430C7FEA6C5CD6D152EA033CD3D07A
:100900005DF8040B704700BF8446104662468C4673
:100910001946634600E000BF01B5FFF7B7FF0028A6
:1009200048BF10F1000F01BD4DF808EDFFF7F4FFCF
:100930000CBF012000205DF808FB00BF4DF808ED5A
:10094000FFF7EAFF34BF012000205DF808FB00BF7D
:100950004DF808EDFFF7E0FF94BF012000205DF89F
:1009600008FB00BF4DF808EDFFF7CEFF94BF012054
:1009700000205DF808FB00BF4DF808EDFFF7C4FF4D
:1009800034BF012000205DF808FB00BF4FEA4102A0
:10099000B2F1E04324BFB3F5001CDCF1FE5C0DD9DD
:1009A00001F0004C4FEAC0024CEA5070B2F1004F27
:1009B00040EB830008BF20F00100704711F0804F2A
:1009C00021D113F13872BCBF01F00040704741F4EF
:1009D00080114FEA5252C2F11802C2F1200C10FAF3
:1009E0000CF320FA02F018BF40F001004FEAC123D7
:1009F0004FEAD32303FA0CFC40EA0C0023FA02F37B
:100A00004FEA4303CCE77FEA625307D150EA013350
:100A10001EBF4FF0FE4040F44000704701F0004020
:100A200040F0FE4040F40000704700BF53B94AB99F
:100A3000002908BF00281CBF4FF0FF314FF0FF30E6
:100A400000F06AB9ADF1080C6DE904CE00F006F8CB
:100A5000DDF804E0DDE9022304B070472DE9F0473A
:100A6000089D0C46002B4ED194468C458646B2FA22
:100A700082F262D94AB1C2F12003914020FA03F315
:100A80000CFA02FC194300FA02FE4FEA1C471FFA57
:100A90008CF6B1FBF7F44FEA1E4307FB141143EA4F
:100AA000014304FB06F199420AD91CEB030304F14C
:100AB000FF3080F01281994240F20F81023C634482
:100AC000591A1FFA8EF3B1FBF7F007FB101143EA36
:100AD000014300FB06F69E420AD91CEB030300F11A
:100AE000FF3180F0FC809E4240F2F980634402387E
:100AF0009B1B40EA044000211DB1D3400022C5E900
:100B00000032BDE8F0878B4205D90DB1C5E900017F
:100B100000210846F5E7B3FA83F1002946D1A34244
:100B200002D39042C0F0F080861A64EB03030120E8
:100B3000002DE6D0C5E90063E3E7002A40F090808D
:100B4000A1EB0C044FEA1C481FFA8CF70121B4FBFF
:100B5000F8F64FEA1E4308FB164443EA044307FB3A
:100B600006F0984208D91CEB030306F1FF3402D2C9
:100B7000984200F2CD8026461C1A1FFA8EF3B4FB71
:100B8000F8F008FB104443EA044300FB07F79F42D8
:100B900008D91CEB030300F1FF3402D29F4200F29C
:100BA000B0802046DB1B40EA0640A5E7C1F12006E5
:100BB0008B4022FA06F71F4320FA06FC04FA01F3E1
:100BC00043EA0C03F44000FA01F8380C4FEA1349E9
:100BD000B4FBF0FE1FFA87FC00FB1E4449EA044404
:100BE0000EFB0CF9A14502FA01F20AD93C190EF1EB
:100BF000FF3A80F08480A14540F28180AEF1020E80
:100C00003C44A4EB09041FFA83F9B4FBF0F300FBA6
:100C1000134449EA044403FB0CFCA44507D93C19DE
:100C200003F1FF3067D2A44565D9023B3C4443EA57
:100C30000E40A0FB0293A4EB0C049C42CE469C46C3
:100C400051D34ED055B1B8EB0E0364EB0C0404FA4B
:100C500006F6CB401E43CC40C5E90064002150E7B6
:100C6000C2F1200320FA03F10CFA02FC24FA03F388
:100C700094400C434FEA1C4800FA02FE1FFA8CF71E
:100C8000B3FBF8F008FB1031230C43EA014300FBEF
:100C900007F1994208D91CEB030300F1FF362CD26F
:100CA00099422AD9023863445B1AA4B2B3FBF8F123
:100CB00008FB113344EA034401FB07F3A34208D9BC
:100CC0001CEB040401F1FF3613D2A34211D90239FF
:100CD0006444E41A41EA004139E70446F0E6084674
:100CE00006E7C845AED2B9EB020E63EB070C01383C
:100CF000A8E73146EDE7034699E73046D4E7D64604
:100D00007FE7634402384DE70646234608460FE76F
:100D1000023E634430E700BF704700BF80B500AFBC
:100D2000154B02221A70144B00225A70124B0022EB
:100D30009A70114B0222DA700F4B40F2EA729A80DD
:100D40000D4B07229A710C4B0522DA7105F000FA5F
:100D500000F016F800F03CF800F096F800F050F9BA
:100D600000F0F4F900F00EFA00F06CFA034B0022E8
:100D70001A6000BF80BD00BFB0000020240C00201E
:100D800080B500AF0121382007F048FE012139204D
:100D900007F044FE0121572007F040FE01215820B2
:100DA00007F03CFE0121592007F038FE01215A20AE
:100DB00007F034FE0121382007F0BCFE0121392064
:100DC00007F0B8FE0121572007F0B4FE00BF80BD38
:100DD00080B400AF294BD3F8D030294A1360284B98
:100DE00093ED007AF7EE006AC6EE877A244BC3EDE6
:100DF000017A224BD3F8D430214A93601F4BD3F8A9
:100E0000D8301F4A13611D4BD3ED377AFCEEE77AD9
:100E100017EE903A9AB21A4B9A81184BD3F8E430F5
:100E2000174A9361154BD3F8E030154A1363144BFE
:100E300093ED0C7AF7EE006AC6EE877A104BC3ED9D
:100E40000D7A0E4BD3F8E8300D4AD3610B4BD3F833
:100E5000EC300B4A1362094BD3F8F030084A936226
:100E6000064BD3F8F430064AD362054B054A5A6163
:100E700000BFBD465DF8047B704700BF980A0020A4
:100E8000100100200000F04180B500AF214B4FF071
:100E90007E52C3F888201F4B4FF07E52C3F88C203F
:100EA00000F03EF81B4B4FF00002DA65194B1A4A6E
:100EB0001A66184B4FF07F525A66164B4FF080421D
:100EC0009A66144B4FF00002DA66144B93ED057AE4
:100ED000124BD3ED0D7A67EE277AB6EE007A67EE05
:100EE000877A0C4BC3ED1E7A0A4B4FF08042C3F851
:100EF0008020084B4FF04042C3F88420054B4FF050
:100F00007E52C3F88820034B4FF07E52C3F88C20EA
:100F100000BF80BD48010020CDCC8C3F10010020D7
:100F200080B400AF354B4FF274529A87334B002296
:100F3000DA87324B1E22A3F84020304B1E22A3F842
:100F400042202E4BB3F9423007EE903AB8EEE77AE2
:100F5000F7EE006AC6EE877A284BC3ED117A274B6D
:100F6000B3F94020254B9A85244BB3F94020234BFD
:100F7000DA85224B3222A3F84820204BB3F92C30DB
:100F80009AB21E4BB3F942309BB213449BB21AB2D1
:100F90001A4B1A86194BB3F92C309AB2174BB3F986
:100FA00042309BB213449BB21AB2144B5A86134B75
:100FB0004FF4E1629A86114B4FF4E162DA860F4BEF
:100FC000B3F934309AB20D4BB3F942309BB21344AB
:100FD0009BB21AB2094B1A87084BB3F936309AB252
:100FE000064BB3F942309BB213449BB21AB2034B87
:100FF0005A8700BFBD465DF8047B7047480100205A
:1010000080B400AF414B424A9A63404B414ADA6395
:10101000414B4FF00002DA603F4B4FF000021A6183
:101020003D4B00221A703C4B00225A70374B3B4A12
:101030009A64364B3A4A9A66344B3A4ADA66334BEC
:101040004FF07E521A67314B374A5A672F4B374A57
:101050009A672E4B344ADA672C4B4FF07E52C3F816
:1010600080202A4B324AC3F88420284B4FF00002DC
:10107000C3F88820254B4FF00002C3F88C20234B87
:101080002B4AC3F89020214B2A4AC3F894201F4BC7
:10109000294AC3F898201D4B284AC3F8A0201B4BAF
:1010A0004FF00002C3F89C20184B002283F8282040
:1010B000164B002283F82920144B002283F82A20A3
:1010C000124B002283F82B20104B4FF00002DA6203
:1010D0000E4B4FF000021A630C4B194A5A630B4B2C
:1010E0004FF000021A66094B4FF000025A66074B98
:1010F0000D4A5A65054B134A9A65044B124ADA6544
:1011000000BFBD465DF8047B704700BFD8010020DA
:101110000000204100002040480100206F12833A67
:101120000000964300001644CDCCCC3D000048435F
:101130000000A041000040409A99993E00004842BA
:1011400017B751383333B33FACC5273980B400AF3C
:101150000A4BC8221A80094B40F6B8325A80084B15
:1011600008221A70064B04225A70054B50229A70BE
:1011700000BFBD465DF8047B704700BF7C020020C5
:101180002803002080B400AF274B284A5A60264B22
:10119000274A9A60244B93ED017A234BD3ED027AD0
:1011A00037EE677AF7EE006AC6EE877A1E4BC3ED1C
:1011B000037A1D4B1F4A1A611B4B1F4A5A611A4B77
:1011C00093ED047A184BD3ED057A37EE677AF7EE94
:1011D000006AC6EE877A144BC3ED067A124B174AA3
:1011E0005A64114B164A9A640F4B4FF07E52DA64E0
:1011F0000D4B4FF07E521A650B4B0022A3F8542082
:10120000094B0022A3F85620074B0022A3F85820D0
:10121000054B00221A70044B00225A7000BFBD46D5
:101220005DF8047B704700BF800200200000604230
:1012300000005C42000020C10000C0C0CDCCCC3D0D
:101240000AD7A33B80B400AF254B01221A70244B70
:1012500000221A72224B0022DA81214B00221A82CC
:101260001F4B00225A821E4B00229A821C4B4B229B
:101270005A811B4BB3F90A20194B9A81184BB3F9C9
:101280000A301A46164BB3F90A3002FB03F3144A2C
:101290005362134B9B6A124A5362114B322283F8FA
:1012A00048200F4B0022DA620D4B00221A630C4BD0
:1012B0000C4A9A630A4B002283F83C20084B002218
:1012C00083F83D20084B5B69054A1364064B5B6954
:1012D000034A536400BFBD465DF8047B704700BFFE
:1012E000DC02002080F0FA021001002080B400AF80
:1012F000094BDB68084A43F08073D360074B002238
:101300005A60064B1B68054A43F00103136000BF97
:10131000BD465DF8047B7047F0ED00E0001000E092
:1013200080B58EB000AF7A4B1B78002B00F0EC80BC
:10133000784B9B68784AA2FB03239B08BB86754BBE
:101340005B68754AA2FB03239B087B86714B5B6835
:1013500007EE903AB8EE677ADFED706AC7EE267A4C
:101360009FED6F7A67EE877AFCEEE77AC7ED017A38
:101370003B7987F831306B4B9B69FB85694BDB69A7
:10138000BB85684BD3ED157AFDEEE77A17EE903A00
:101390007B85644BD3ED167AFDEEE77A17EE903A33
:1013A0003B85614BD3ED007A9FED607A67EE877ADB
:1013B000FDEEE77A17EE903AFB845B4BD3ED017AB2
:1013C0009FED5A7A67EE877AFDEEE77A17EE903A4C
:1013D000BB84FF233B72FF237B721923BB72F5236F
:1013E000FB72BB8E1B0A9BB2DBB23B73BB8EDBB2C4
:1013F0007B737B8E1B0A9BB2DBB2BB737B8EDBB233
:10140000FB7397F831303B74494B1B787B74494B25
:101410001B78BB74B7F92E301B121BB2DBB2FB7406
:10142000FB8DDBB23B75B7F92C301B121BB2DBB264
:101430007B75BB8DDBB2BB75B7F92A301B121BB2B3
:10144000DBB2FB757B8DDBB23B76B7F928301B1224
:101450001BB2DBB27B763B8DDBB2BB76B7F92630B5
:101460001B121BB2DBB2FB76FB8CDBB23B77B7F90E
:1014700024301B121BB2DBB27B77BB8CDBB2BB7799
:10148000284B1B78FB77274B5B7887F82030254B60
:1014900093F92830DBB287F82130224B93F92930B9
:1014A000DBB287F82230002387F82330002387F847
:1014B000373012E097F8232097F83730303307F1B0
:1014C00008010B4413F8303C1344DBB287F8233097
:1014D00097F83730013387F8373097F837301A2BC1
:1014E000E8D997F823305B42DBB287F8233007F165
:1014F00008031C22194610480EF016FA08F000FCEA
:10150000044B00225A6000E000BF3837BD4680BD62
:101510004003002030030020398EE33800A00C4740
:101520000000C842480100205003002000007A4417
:1015300018000020050C0020EC53002080B582B07C
:1015400002AF1C4B1B78DBB2002B08D0194B5B7829
:101550001946652008F01AFC164B00221A70154B2C
:101560009B78DBB2002B0BD0124BDB781946114B6A
:101570001B791A46822008F0C7FC0E4B00229A7095
:101580000C4B5B79DBB2002B11D00A4B9B791946CF
:10159000084BDB791A46074B1B7A18460023009349
:1015A0000346692008F0EEFC024B00225A7100BF8E
:1015B000BD4680BD4403002080B500AF2E4B1B7894
:1015C000032B46D801A252F823F000BF7116010880
:1015D0000B1601082F160108DD150108274B0522FF
:1015E0001A70264B03225A7002F064F8002000F0B3
:1015F00051F8012000F04EF8214B1B68214A53603E
:101600001F4B5B68204A536033E01C4B05221A7065
:101610001A4B01225A701D4B4FF000021A61002034
:1016200000F038F8164B1B68164A536021E0134B44
:1016300005221A70114B02225A70144B4FF000020F
:10164000DA60012000F026F80D4B5B680E4A53600B
:101650000FE00A4B00221A70084B00225A700C4B04
:101660004FF000029A600A4B4FF00002DA6000E08F
:1016700000BF00BF80BD00BF040C0020AC030020F1
:1016800050030020740500200407002048010020BA
:10169000D801002080B5AEB000AF7860786801F066
:1016A00053FA7B68DBB2184602F080F94FF0000372
:1016B000C7F8AC30D24A7B6802339B001344043332
:1016C0001B68C7F88C30CE4A7B6822339B001344DA
:1016D000D3ED007A97ED237A67EE277AC7ED227A69
:1016E000C84A7B6808339B0013441B68C7F8AC30BA
:1016F000C34A7B6813441B7887F88730C04A7B68ED
:10170000083352F82330A7F88430BD4A7B6814337D
:101710009B00134404331B68C7F88030B84A7B68C9
:1017200014335B0013449B88A7F87E30B44A7B686F
:1017300014335B0013441B89A7F87C30B04A7B68E4
:1017400018335B0013449B88A7F87A30AC4A7B6857
:1017500018335B0013441B89A7F87830B7F984204D
:10176000A74BB3F93C3019460B469B000B445B007A
:101770009A420EDAA24B93ED177AA34BD3ED0C7A73
:1017800067EE277AC7ED2C7AFF2387F8AB3001F09C
:1017900075B89B4BB3F93C301A4613469B00134473
:1017A0005B001A46B7F984309A421ADCB7F98420F4
:1017B000934BB3F93E3019460B469B000B445B003C
:1017C0009A420EDA8E4B93ED187A8F4BD3ED0C7A4A
:1017D00067EE277AC7ED2C7A002387F8AB3001F04B
:1017E0004DB8874BB3F93E301A4613469B0013445D
:1017F0005B001A46B7F984309A4247DCB7F9842077
:101800007F4BB3F9403019460B469B000B445B00FD
:101810009A423BDA7A4B93ED187A794BD3ED1A6AF8
:10182000774BD3ED187A36EEE76A754BB3F9403053
:101830001A46734BB3F93E30D21A13469B00134439
:101840005B0007EE903AF8EEE77AC6EE276AB7F942
:1018500084206B4BB3F93E3019466FF0090301FB4E
:1018600003F3134407EE903AF8EEE77A66EEA77AB0
:1018700037EE277A644BD3ED0C7A67EE277AC7ED03
:101880002C7A012387F8AB3000F0F8BF5C4BB3F93A
:1018900040301A4613469B0013445B001A46B7F9C2
:1018A00084309A4218DCB7F98410B7F97E201346C9
:1018B0009B0013445B0099420EDA514B93ED1A7A68
:1018C000514BD3ED0C7A67EE277AC7ED2C7A0223C1
:1018D00087F8AB3000F0D2BFB7F97E2013469B00EB
:1018E00013445B001A46B7F984309A4200F3C68766
:1018F000B7F9843047F6FF72934200F0BF8797F83C
:101900008730052B00F2AA8701A252F823F000BF0E
:1019100029190108411A0108EF1B0108E31D0108FC
:10192000C7230108272601084FF00003C7F8AC3091
:10193000344A7B680A339B0013440433D3ED007AA6
:1019400097ED227A67EE277AC7ED2D7A2C4BD3EDEF
:101950001A7A97ED2D7AB4EEE77AF1EE10FA03D801
:10196000274B9B6EC7F8B430B7F97E2013469B0017
:1019700013445B001A46B7F984309A4246DCB7F943
:101980008410B7F97C2013469B0013445B009942F6
:101990003CDA1B4B93ED1A7A194BD3ED1A7AD7ED3B
:1019A0002D6A76EEE76AB7F98420B7F97E306FF0DA
:1019B000090101FB03F3134407EE903AF8EEE77ACE
:1019C00026EEA76AB7F97C20B7F97E30D21A134603
:1019D0009B0013445B0007EE903AF8EEE76AC6EE10
:1019E000267A37EE277A084BD3ED0C7A67EE277A02
:1019F000C7ED2C7A032387F8AB3000F034BF00BF6B
:101A000048010020D801002010010020B7F97C20F7
:101A100013469B0013445B001A46B7F984309A4280
:101A200000F32187DA4BD3ED0C7A97ED2D7A67EE30
:101A3000277AC7ED2C7A042387F8AB3000F013BF68
:101A4000D44BD3ED207A97ED207AB4EEE77AF1EE1D
:101A500010FA1DDDD04BD3ED127A97ED2B7A77EE8D
:101A6000677AC7ED2B7ACD4B14221A70CB4B042228
:101A70005A70CA4B50229A70D7ED2B7AF5EEC07A85
:101A8000F1EE10FA2ED84FF00003C7F8AC3029E081
:101A9000C04BD3ED217A97ED207AB4EEE77AF1EEE0
:101AA00010FA1FD8BC4BD3ED127A97ED2B7A77EE54
:101AB000277AC7ED2B7AB94B28221A70B74B04222C
:101AC0005A70B64B3C229A70B24BD3ED1B7A97ED0D
:101AD0002B7AB4EEE77AF1EE10FA03DBAD4BDB6E56
:101AE000C7F8AC3097ED227AD7ED2B7A37EE277A0C
:101AF000A94A7B680A339B0013440433D3ED007A70
:101B000067EE277AC7ED2D7AA24BD3ED1A7A97EDBF
:101B10002D7AB4EEE77AF1EE10FA03D89D4B9B6E66
:101B2000C7F8B430B7F97E2013469B0013445B001E
:101B30001A46B7F984309A423FDCB7F98410B7F9F6
:101B40007C2013469B0013445B00994235DA914B8D
:101B500093ED1A7A8F4BD3ED1A7AD7ED2D6A76EE84
:101B6000E76AB7F98420B7F97E306FF0090101FB0D
:101B700003F3134407EE903AF8EEE77A26EEA76AED
:101B8000B7F97C20B7F97E30D21A13469B00134474
:101B90005B0007EE903AF8EEE76AC6EE267A37EE7B
:101BA000277A7B4BD3ED0C7A67EE277AC7ED2C7A38
:101BB000032387F8AB3000F058BEB7F97C201346FA
:101BC0009B0013445B001A46B7F984309A4200F335
:101BD0004C866F4BD3ED0C7A97ED2D7A67EE277A12
:101BE000C7ED2C7A042387F8AB3000F03EBE4FF0EF
:101BF0000003C7F8AC30684A7B680A339B00134483
:101C00000433D3ED007A97ED227A67EE277AC7ED99
:101C10002D7A604BD3ED1A7A97ED2D7AB4EEE77AF0
:101C2000F1EE10FA03D85B4B9B6EC7F8B430B7F9EE
:101C30007E2013469B0013445B001A46B7F984309C
:101C40009A4200F3AD80B7F98410B7F97A201346B1
:101C50009B0013445B00994280F2A2804D4B93EDB0
:101C60001A7A4C4BD3ED1A7AD7ED2D6A76EEE76AE5
:101C7000B7F98420B7F97E306FF0090101FB03F357
:101C8000134407EE903AF8EEE77A26EEA76AB7F922
:101C90007A20B7F97E30D21A13469B0013445B00BA
:101CA00007EE903AF8EEE76AC6EE267A37EE277A24
:101CB000374BD3ED0C7A67EE277AC7ED2C7AB7F95C
:101CC0008420B7F97E306FF0090101FB03F31A4459
:101CD00013461B019B1A1B011946B7F97A20B7F965
:101CE0007E30D21A13469B0013445B0091FBF3F342
:101CF000DBB20A33DAB2294B1A70284B1B78FF2B60
:101D000002D1264BFF221A70B7F98420B7F97E3032
:101D10006FF0090101FB03F31A4413469B001344BF
:101D2000DA00D11AB7F97A20B7F97E30D21A134601
:101D30009B0013445B0091FBF3F3DBB2C3F1280378
:101D4000DAB2164B5A70B7F98420B7F97E306FF0CB
:101D5000090101FB03F31A4413469B001344DB0003
:101D60001946B7F97A20B7F97E30D21A13469B008C
:101D700013445B0091FBF3F3DBB2C3F12803DAB247
:101D8000064B9A70042387F8AB3000F070BD00BF9B
:101D90001001002048010020D80100202803002065
:101DA000B7F97A2013469B0013445B001A46B7F933
:101DB00084309A4200F35B85B7F9843047F6FF72AE
:101DC000934200F05485C24BD3ED0C7A97ED2D7AF7
:101DD00067EE277AC7ED2C7A062387F8AB3000F040
:101DE00046BD4FF00003C7F8AC30BA4B9B6F3B6465
:101DF000B84BDB6FFB63B74BD3F88030BB63B64B9C
:101E00007B63B64B3B63B34B93ED227AB44BD3ED7C
:101E10001A7AB4EEE77AF1EE10FA03DDAD4BD3F89F
:101E2000883001E0AE4B9B6EFB62FB6ABB6297EDB4
:101E3000207AD7ED0C7AB4EEE77AF1EE10FA40F39F
:101E4000BE8097ED207AD7ED107A77EE677AC7EDEE
:101E5000077AD7ED107A9FEDA37A67EE877AC7ED00
:101E6000067A97ED077AD7ED067AB4EEE77AF1EEC7
:101E700010FA0ADCD7ED067AF1EE677A97ED077A69
:101E8000B4EEE77AF1EE10FA3BD5D7ED077AF5EE2E
:101E9000C07AF1EE10FA1CDD934A7B689B00134474
:101EA00093ED007AD7ED0E7AF0EE086A67EEA66A37
:101EB000D7ED077A66EEA76AD7ED0D7A66EEA77AB8
:101EC00077EE277A884A7B689B001344C3ED007A3B
:101ED00017E0854A7B689B00134493ED007AD7EDA9
:101EE0000E6AD7ED077A66EEA76AD7ED0D7A66EE31
:101EF000A77A77EE277A7C4A7B689B001344C3ED70
:101F0000007AD7ED077AF5EEC07AF1EE10FA0CDD23
:101F1000D7ED0F7AB0EE087A67EE877A97ED077AF9
:101F200067EE277AC7ED297A07E097ED0F7AD7EDAC
:101F3000077A67EE277AC7ED297A664BD3ED237AC5
:101F4000F5EEC07AF1EE10FA03DD624BD3F88C3077
:101F500001E0D7F888307B61634A7B689B001344BB
:101F6000D3ED007A97ED297A77EE277AC7ED287AB4
:101F700097ED287AD7ED057AB4EEE77AF1EE10FA0C
:101F800002DD7B69C7F8A03097ED287AD7ED0B7A90
:101F9000B4EEE77AF1EE10FA02D5FB6AC7F8A0308A
:101FA0004C4A7B680A339B0013440433D3ED007A18
:101FB00097ED287A67EE277AC7ED2D7A16E1D7EDEF
:101FC0000C7AF1EE677A97ED207AB4EEE77AF1EECB
:101FD00010FA40F18B803F4BD3ED217A97ED0D7ACB
:101FE00067EE277AC7ED087A3F4A7B689B00134467
:101FF000D3ED007A97ED0A7AB4EEE77AF1EE10FAB3
:1020000023D5394A7B689B00134493ED007AD7EDC2
:10201000087A77EE677A344A7B689B001344C3EDF5
:10202000007A314A7B689B001344D3ED007A97ED28
:102030000A7AB4EEE77AF1EE10FA36DD2A4A7B68C6
:102040009B001344BA6A1A602FE0274A7B689B0002
:102050001344D3ED007A97ED0A7AB4EEE77AF1EE05
:1020600010FA22DD204A7B689B00134493ED007A2E
:10207000D7ED087A77EE277A1B4A7B689B001344DA
:10208000C3ED007A184A7B689B001344D3ED007AB5
:1020900097ED0A7AB4EEE77AF1EE10FA05D5124A16
:1020A0007B689B001344BA6A1A600F4A7B689B00E6
:1020B000134493ED007A074A7B680A339B0013446C
:1020C0000433D3ED007A67EE277AC7ED2D7A8DE0E1
:1020D00010010020D801002017B7D13800000C42B1
:1020E00048010020CDCC4C3D9C030020BD4BD3EDDE
:1020F000217AB6EE007A67EE877A97ED0D7A67EE71
:10210000277AC7ED097AB84A7B689B001344D3ED60
:10211000007A97ED0A7AB4EEE77AF1EE10FA23D559
:10212000B14A7B689B00134493ED007AD7ED097A9E
:1021300077EE677AAC4A7B689B001344C3ED007A64
:10214000A94A7B689B001344D3ED007A97ED0A7A85
:10215000B4EEE77AF1EE10FA36DDA34A7B689B0015
:102160001344BA6A1A602FE09F4A7B689B001344AD
:10217000D3ED007A97ED0A7AB4EEE77AF1EE10FA31
:1021800022DD994A7B689B00134493ED007AD7EDDA
:10219000097A77EE277A944A7B689B001344C3ED53
:1021A000007A914A7B689B001344D3ED007A97ED47
:1021B0000A7AB4EEE77AF1EE10FA05D58A4A7B681E
:1021C0009B001344BA6A1A60874A7B689B001344D9
:1021D00093ED007A834A7B680A339B0013440433EF
:1021E000D3ED007A67EE277AC7ED2D7A7D4BD3EDDC
:1021F000237AF5EEC07AF1EE10FA03DD794BD3F8CD
:102200008C3001E0D7F888303B61774A7B689B00CF
:102210001344D3ED007A97ED047AB4EEE77AF1EE49
:1022200010FA05D5704A7B689B0013443A691A601E
:102230006D4A7B689B001344D3ED007A97ED0B7ACF
:10224000B4EEE77AF1EE10FA05DD674A7B689B0091
:102250001344FA6A1A6097ED2D7AD7ED0B7AB4EE33
:10226000E77AF1EE10FA02D5FB6AC7F8B4305D4B9D
:10227000D3ED287A97ED0D7A67EE277AC7ED037ACA
:102280005A4A7B689B001344D3ED007A97ED2D7A70
:1022900077EE677AC7ED027A97ED027AD7ED037A87
:1022A000B4EEE77AF1EE10FA0CDD504A7B689B0041
:1022B0001344D3ED007A97ED037A77EE277AC7EDD2
:1022C0002D7A16E0D7ED037AF1EE677A97ED027A70
:1022D000B4EEE77AF1EE10FA0BD5444A7B689B0026
:1022E000134493ED007AD7ED037A77EE677AC7ED62
:1022F0002D7A3E4A7B689B001344D7F8B4201A60BD
:10230000B7F97E2013469B0013445B001A46B7F9C9
:1023100084309A423EDCB7F98410B7F97C2013462A
:102320009B0013445B00994234DA314B93ED1A7AE7
:102330002F4BD3ED1A7AD7ED2D6A76EEE76AB7F90F
:102340008420B7F97E306FF0090101FB03F31344D9
:1023500007EE903AF8EEE77A26EEA76AB7F97C2006
:10236000B7F97E30D21A13469B0013445B0007EE88
:10237000903AF8EEE76AC6EE267A37EE277A1D4BDA
:10238000D3ED0C7A67EE277AC7ED2C7A032387F812
:10239000AB306EE2B7F97C2013469B0013445B0020
:1023A0001A46B7F984309A4200F36382114BD3ED99
:1023B0000C7A97ED2D7A67EE277AC7ED2C7A0423F5
:1023C00087F8AB3055E24FF00003C7F8AC30D7EDDB
:1023D000207AF5EEC07AF1EE10FA0DDDD7F88030F4
:1023E0000CE000BFD80100209C030020A4030020C3
:1023F00048010020100100204FF00003FB65FB6D39
:10240000C7F89C30CE4BD3ED1B7A97ED277AB4EE0C
:10241000E77AF1EE10FA03DDC94BDB6EC7F89C30AA
:10242000C74BDB6EBB65C64B1B6F7B65C44B5B6FDD
:102430003B65D7ED157AB7EE007AF4EE477AF1EE08
:1024400010FA08D1D7ED276A97ED167AC6EE877A8B
:10245000C7ED267A0DE097ED277AD7ED167AC7EE0D
:10246000276AD7ED150AB0EE660A16F063FC87ED11
:10247000260AB7EE007AD7ED147A37EE677AD7EDF1
:10248000267A27EE277AD7ED147A37EE277AD7ED1A
:10249000227A27EE277AAA4A7B680A339B001344E4
:1024A0000433D3ED007A67EE277AC7ED2D7AA54B7A
:1024B000D3ED1A7A97ED2D7AB4EEE77AF1EE10FAB1
:1024C00003D8A04B9B6EC7F8B4309F4BFB649C4B6A
:1024D000D3ED287A97ED137A67EE277AC7ED127A53
:1024E0009A4A7B689B001344D3ED007A97ED2D7ACE
:1024F00077EE677AC7ED117A97ED117AD7ED127AF8
:10250000B4EEE77AF1EE10FA0CDD904A7B689B009E
:102510001344D3ED007A97ED127A77EE277AC7ED60
:102520002D7A16E0D7ED127AF1EE677A97ED117AEF
:10253000B4EEE77AF1EE10FA0BD5844A7B689B0083
:10254000134493ED007AD7ED127A77EE677AC7EDF0
:102550002D7A7E4A7B689B001344D7F8B4201A601A
:10256000B7F97E2013469B0013445B001A46B7F967
:1025700084309A423EDCB7F98410B7F97C201346C8
:102580009B0013445B00994234DA6E4B93ED1A7A48
:102590006C4BD3ED1A7AD7ED2D6A76EEE76AB7F970
:1025A0008420B7F97E306FF0090101FB03F3134477
:1025B00007EE903AF8EEE77A26EEA76AB7F97C20A4
:1025C000B7F97E30D21A13469B0013445B0007EE26
:1025D000903AF8EEE76AC6EE267A37EE277A5C4B39
:1025E000D3ED0C7A67EE277AC7ED2C7A032387F8B0
:1025F000AB3040E1B7F97C2013469B0013445B00ED
:102600001A46B7F984309A4200F33581504BD3ED26
:102610000C7A97ED2D7A67EE277AC7ED2C7A042392
:1026200087F8AB3027E14FF00003C7F8AC300DF06E
:10263000FBFD07EE900AB8EE677ADFED466AC7EE5B
:10264000267AC7ED1D7A3E4BD3ED247A9FED427A70
:1026500027EE877AD7ED1D7A67EE277AB0EE670A04
:1026600016F0DEFB87ED1C0A354BD3F89430C7F823
:102670009430334BD3ED267A97ED227A67EE277AA2
:10268000C7ED1B7A97ED257AD7ED1B7AB4EEE77A82
:10269000F1EE10FA02DDFB6EC7F8943097ED257A63
:1026A000D7ED1C7A27EE277AD7ED227A37EE277AF4
:1026B000234A7B680A339B0013440433D3ED007A2A
:1026C00067EE277AC7ED2D7A1E4BD3ED1A7A97ED78
:1026D0002D7AB4EEE77AF1EE10FA03D8194B9B6E1F
:1026E000C7F8B430184BBB66154BD3ED287A97ED7D
:1026F0001A7A67EE277AC7ED197A144A7B689B002D
:102700001344D3ED007A97ED2D7A77EE677AC7ED13
:10271000187A97ED187AD7ED197AB4EEE77AF1EED8
:1027200010FA1BDD094A7B689B001344D3ED007A45
:1027300097ED197A77EE277AC7ED2D7A25E000BF5D
:10274000D80100204801002017B75139A403002008
:102750001001002000007A44DB0FC940D7ED197A40
:10276000F1EE677A97ED187AB4EEE77AF1EE10FAA7
:102770000BD5AF4A7B689B00134493ED007AD7EDED
:10278000197A77EE677AC7ED2D7AA94A7B689B00A4
:102790001344D7F8B4201A60B7F97E2013469B0083
:1027A00013445B001A46B7F984309A423EDCB7F90D
:1027B0008410B7F97C2013469B0013445B009942B8
:1027C00034DA9C4B93ED1A7A9A4BD3ED1A7AD7ED03
:1027D0002D6A76EEE76AB7F98420B7F97E306FF09C
:1027E000090101FB03F3134407EE903AF8EEE77A90
:1027F00026EEA76AB7F97C20B7F97E30D21A1346C5
:102800009B0013445B0007EE903AF8EEE76AC6EED1
:10281000267A37EE277A884BD3ED0C7A67EE277A43
:10282000C7ED2C7A032387F8AB3026E0B7F97C207C
:1028300013469B0013445B001A46B7F984309A4252
:102840001BDC7D4BD3ED0C7A97ED2D7A67EE277A62
:10285000C7ED2C7A042387F8AB300EE0754B9B6EE6
:10286000C7F8B4300AE000BF08E000BF06E000BFD0
:1028700004E000BF02E000BF00E000BF4FF0000333
:10288000C7F89030B7F98410B7F97C2013469B0045
:1028900013445B0099423CDBD7ED2D7AB7EE087A02
:1028A000F4EEC77AF1EE10FA04D8644B9B6DC7F8CA
:1028B000903065E0D7ED2D7AB7EE087AF4EEC77A5E
:1028C000F1EE10FA17DDD7ED2D7AB0EE047AF4EEC2
:1028D000C77AF1EE10FA0ED8584B93ED167A574B93
:1028E000D3ED157A77EE277AB6EE007A67EE877A1F
:1028F000C7ED247A44E0D7ED2D7AB0EE047AF4EEF9
:10290000C77AF1EE10FA3BDD4C4B5B6DC7F89030A7
:1029100036E0B7F97C2013469B0013445B001A464F
:10292000B7F984309A421ADDB7F98420414BB3F9E4
:10293000403019460B469B000B445B009A420EDD6B
:102940003E4B93ED167A3D4BD3ED157A77EE277A11
:10295000B6EE007A67EE877AC7ED247A10E0354B41
:10296000B3F940301A4613469B0013445B001A46E5
:10297000B7F984309A4203DD4FF00003C7F8903076
:1029800097ED240A786800F061F82C4BD3ED277A94
:10299000F5EEC07AF1EE10FA0EDD284BD3ED277A72
:1029A00097ED2C7AB4EEE77AF1EE10FA04DD234BC2
:1029B000D3F89C30C7F8B0301F4BD3ED057A97EDB4
:1029C0002C7AB4EEE77AF1EE10FA03DB1A4B5B696E
:1029D000C7F8B0301A4A7B689B001344D7F8B02080
:1029E0001A6097F9AB10134A7B68134428330A46E0
:1029F0001A70124A7B6808339B001344D7F8AC2046
:102A00001A600D4B93ED0C7AD7ED2C6AC6EE877ADF
:102A10000C4A7B689B001344C3ED007A0A4A7B682A
:102A2000134497F8AB201A7000BFB837BD4680BD7D
:102A3000A40300204801002010010020D80100203C
:102A400050030020580300207003002080B487B09A
:102A500000AF786087ED000A3A4A7B6816339B0026
:102A6000134408331B683B6197ED047AD7ED007A75
:102A7000B4EEE77AF1EE10FA16DD324BD3ED177AA9
:102A800097ED047A77EE677AC7ED057A2D4BD3ED93
:102A9000167A97ED057AB4EEE77AF1EE10FA22DBBA
:102AA000284B9B6D7B611EE097ED047AD7ED007A91
:102AB000B4EEE77AF1EE10FA13D5224BD3ED177A84
:102AC00097ED047A77EE277AC7ED057AD7ED057A88
:102AD000F5EEC07AF1EE10FA05D84FF000037B61F5
:102AE00001E03B697B6197ED057AD7ED007A77EEDF
:102AF000677AC7ED037A134BD3ED177AF1EE677A55
:102B000097ED037AB4EEE77AF1EE10FA0BDD0D4B98
:102B1000D3ED177A97ED037AB4EEE77AF1EE10FA77
:102B200001D53B687B61074A7B6816339B001344E1
:102B300008337A691A6000BF1C37BD465DF8047B14
:102B4000704700BFD801002080B483B000AF786028
:102B5000734B1B78002B40F0DC80724A7B68134477
:102B60002A331B78002B70D0012B40F0D3806D4AA4
:102B70007B680A339B0013440433D3ED007AB7EE2D
:102B8000007AF4EEC77AF1EE10FA00D4C2E0664B98
:102B900093ED157A634BD3ED0F7AF1EE677AB4EECD
:102BA000E77AF1EE10FA00DCB4E05F4B93ED167AB1
:102BB0005C4BD3ED0F7AF1EE677AB4EEE77AF1EE83
:102BC00010FA00DCA6E0574B93ED0B7A554BD3ED92
:102BD0000D7A77EE277A534BC3ED0B7A514BD3ED39
:102BE0000B7AB7EE007AF4EEC77AF1EE10FA03DB57
:102BF0004C4B4FF07E52DA624A4B93ED0C7A494BC4
:102C0000D3ED0D7A77EE277A464BC3ED0C7A454B20
:102C1000D3ED0C7AB7EE007AF4EEC77AF1EE10FA43
:102C200000DA77E03F4B4FF07E521A633D4B0022B3
:102C300083F829203B4A7B6813442A331A783B4B9C
:102C40005A703A4B01221A7064E0364A7B680A33A4
:102C50009B0013440433D3ED007AF5EEC07AF1EE15
:102C600010FA00DC56E0304B93ED157A2D4BD3ED86
:102C70000F7AB4EEE77AF1EE10FA00D44AE02A4B6C
:102C800093ED167A274BD3ED0F7AB4EEE77AF1EE97
:102C900010FA00D43EE0234B93ED0B7A214BD3ED99
:102CA0000D7A77EE677A1F4BC3ED0B7A1D4BD3ED90
:102CB0000B7AF5EEC07AF1EE10FA03D8194B4FF00B
:102CC0000002DA62174B93ED0C7A164BD3ED0D7AB6
:102CD00077EE677A134BC3ED0C7A124BD3ED0C7A77
:102CE000F5EEC07AF1EE10FA00D913E00D4B4FF07B
:102CF00000021A630B4B002283F82920094A7B68E3
:102D000013442A331A78094B5A70084B01221A705F
:102D100000E000BF0C37BD465DF8047B704700BF84
:102D200072030020D8010020480100204403002045
:102D300080B584B002AF87ED010AD7ED017AB6EE17
:102D4000007AF4EEC77AF1EE10FA02DB4FF07C5312
:102D50007B60A34B93ED037AA14BD3ED017AB4EEE4
:102D6000E77AF1EE10FA52D59D4B93ED157A9D4B13
:102D7000D3ED0F7AF1EE677AB4EEE77AF1EE10FA5E
:102D80003FDD974B93ED167A964BD3ED0F7AF1EE2C
:102D9000677AB4EEE77AF1EE10FA32DD904B93EDFC
:102DA000037AD7ED017A77EE277A8D4BC3ED037A5C
:102DB0008B4B93ED047AD7ED017A77EE277A884B27
:102DC000C3ED047A864BD3ED037A77EEA77AFCEE57
:102DD000E77A17EE903A99B2814B1B781846804BF0
:102DE000D3ED047A77EEA77AFCEEE77A17EE903A05
:102DF0009BB27B4A527800920246662007F0C2F8E6
:102E000066E00022784979480CF08EFD60E0744B52
:102E100093ED037A724BD3ED017AB4EEE77AF1EEDB
:102E200010FA55DD6E4B93ED157A6E4BD3ED0F7A9C
:102E3000B4EEE77AF1EE10FA45D5694B93ED167AC8
:102E4000684BD3ED0F7AB4EEE77AF1EE10FA3AD58B
:102E5000634B93ED037AD7ED017AF0EE086A67EEE3
:102E6000A67A77EE677A5E4BC3ED037A5C4B93EDFF
:102E7000047AD7ED017AF0EE086A67EEA67A77EE6B
:102E8000677A574BC3ED047A554BD3ED037A77EE4F
:102E9000A77AFCEEE77A17EE903A99B2504B1B787E
:102EA00018464F4BD3ED047A77EEA77AFCEEE77A1B
:102EB00017EE903A9BB24A4A527800920246662038
:102EC00007F060F804E00022474948480CF02CFD68
:102ED000D7ED017AB1EE677A414BD3ED036A404BEF
:102EE000D3ED017A76EEE77AB4EEE77AF1EE10FAF6
:102EF00000D971E03A4B93ED037A394BD3ED017A67
:102F000077EE677A97ED017AB4EEE77AF1EE10FA90
:102F100000DA61E0324B5B68314AD360D7ED017A69
:102F2000B1EE677A2E4BD3ED046A2D4BD3ED027AC6
:102F300076EEE77AB4EEE77AF1EE10FA00D94BE0DC
:102F4000274B93ED047A264BD3ED027A77EE677A1E
:102F500097ED017AB4EEE77AF1EE10FA00DA3BE091
:102F60001F4B9B681E4A13610AF08EFF0022204906
:102F70001E480CF0D9FC1A4BD3ED037A0220B0EEB8
:102F8000670A0DF011F803460022194617480CF0A5
:102F9000CBFC0022174915480CF0C6FC104BD3EDB2
:102FA000037A77EEA77AFCEEE77A17EE903A99B2B9
:102FB0000B4B1B7818460A4BD3ED047A77EEA77AB1
:102FC000FCEEE77A17EE903A9BB2054A52780092EF
:102FD0000246662006F0D6FF00BF0837BD4680BD1A
:102FE00048010020D8010020B49E0208EC530020C4
:102FF000CC9E0208D89E020880B485B000AFB54BC5
:10300000D3ED027AF1EE677AB6EE007A27EE877A90
:10301000B14BD3ED0C6AB14BD3ED137A76EEE77A70
:1030200067EE277A9FEDAE7A27EE877AA94BD3ED2C
:10303000017A67EE277AFDEEE77A17EE903A1AB238
:10304000A64B9A82A34BD3ED027ABBEE047A67EECD
:10305000877AB6EE007A27EE877A9F4BD3ED0C6A1B
:103060009E4BD3ED137A76EEE77A67EE277A9FEDE3
:103070009C7A27EE877A974BD3ED017A67EE277A11
:10308000FDEEE77A17EE902A944B9A61934B9B6979
:10309000002B02DC914B00229A618E4BD3ED027A19
:1030A000BAEE047A67EE877AB6EE007A27EE877A70
:1030B000894BD3ED0C6A894BD3ED137A76EEE77A20
:1030C00067EE277A9FED867A27EE877A814BD3EDDC
:1030D000017A67EE277AFDEEE77A17EE902A7F4BAA
:1030E0001A627C4BD3ED027AF1EE677AB6EE007A83
:1030F00027EE877A7B4BD3ED0C6A784BD3ED147AAD
:1031000076EEE77A67EE277A9FED757A27EE877A73
:10311000704BD3ED017A67EE277AFDEEE77A17EE72
:10312000903A1AB26D4BDA826A4BD3ED027ABBEE5B
:10313000047A67EE877AB6EE007A27EE877A694BD3
:10314000D3ED0C6A654BD3ED147A76EEE77A67EE31
:10315000277A9FED637A27EE877A5E4BD3ED017A6B
:1031600067EE277AFDEEE77A17EE902A5B4BDA617D
:103170005A4BDB69002B02DC584B0022DA61554BBD
:10318000D3ED027ABAEE047A67EE877AB6EE007A69
:1031900027EE877A534BD3ED0C6A504BD3ED147A5C
:1031A00076EEE77A67EE277A9FED4D7A27EE877AFB
:1031B000484BD3ED017A67EE277AFDEEE77A17EEFA
:1031C000902A464B5A62434BD3ED027AF1EE677A6E
:1031D000B6EE007A27EE877A3F4BD3ED117ADFED1A
:1031E000426A67EEA67A27EE277A3A4BD3ED017A48
:1031F00067EE277A394BC3ED157A364BD3ED027A59
:10320000F1EE677AB6EE007A27EE877A354BD3ED8A
:10321000117ADFED356A67EEA67A27EE277A2D4B15
:10322000D3ED017A67EE277A2C4BC3ED167A2F4B3C
:10323000BB602F4B7B600023FB6040E0274AFB68AC
:1032400014339B001344043393ED007A294AFB683E
:103250009B001344D3ED007A77EE677A97ED027AFC
:1032600067EE277AC7ED007A234AFB689B00134478
:1032700093ED007A204AFB689B001344D3ED007A5B
:10328000D7ED006A76EEE76AD7ED017A66EEA77AA7
:1032900077EE277A184AFB689B001344C3ED007A47
:1032A0000E4AFB6814339B00134404331A68114917
:1032B000FB689B000B441A60FB680133FB60FB68F2
:1032C000012BBBDD00BF00BF1437BD465DF8047B9A
:1032D000704700BF100100207C040020480100203E
:1032E00035FA8E3CF80400203B77D63D00401C4662
:1032F0000AD7A33C680300206003002080B400AF1D
:10330000154B9B69154A82FB0312D210DB17D31AA7
:103310001AB2114B9A82104B9B69DA0F13445B105F
:103320001A460D4B1A620C4BDB690C4A82FB0312E6
:10333000D210DB17D31A1AB2074BDA82064BDB69BD
:10334000DA0F13445B101A46034B5A6200BFBD46A6
:103350005DF8047B704700BF480100206766666621
:1033600080B582B000AF0346FB71FB79022B24D0FD
:10337000022B35DC002B02D0012B0FD030E01A4B92
:103380001B881A4643F2BC4302FB03F318460AF0BB
:10339000C3FB164B1B6B164AD36421E0124B1B88F0
:1033A0001A4643F2BC4302FB03F318460AF0B4FB8F
:1033B000104B1B6B0E4A136512E00B4B1B881A4611
:1033C00043F2BC4302FB03F318460AF0A5FB074B8C
:1033D0001B6B074AD364074B1B6B054A136500BF81
:1033E00000BF0837BD4680BD7C0200207C04002061
:1033F00048010020F804002080B582B000AF0346E9
:103400000A46FB711346BB71BB79002B02D0012B1E
:1034100061D0A2E0FB79534A08335B001344B3F94F
:1034200004301A464F4BB3F9403019464D4BB3F9AF
:1034300042300B449A422CDDFB794A4A08335B0048
:103440001344B3F904309AB2464BB3F942309BB2FD
:1034500013449AB2FB7911B2424A14335B0013440D
:103460000A461A81FB793F4A14335B001344B3F9CF
:1034700008309AB23B4BB3F942309BB2D31A9AB29E
:10348000FB7911B2374A14335B0013440A469A8021
:1034900063E00022344935480CF046FA314BB3F969
:1034A00040309AB22F4BB3F942309BB213449AB2D8
:1034B000FB7911B22B4A14335B0013440A461A817C
:1034C000FB79284AB2F94010264A14335B001344B2
:1034D0000A469A8041E0FB79224A08335B00134494
:1034E000B3F904301946FB791E4A14335B001344C8
:1034F000B3F908301A461B4BB3F9483013449942CC
:1035000025DDFB79FA79174908335B000B44B3F9E1
:103510000400144902F118035B000B4402469A8030
:10352000FB79104A18335B001344B3F904309AB2A4
:103530000C4BB3F942309BB213449AB2FB7911B2EF
:10354000084A18335B0013440A461A8104E000223B
:10355000074906480CF0E8F900BF00BF0837BD4630
:1035600080BD00BF48010020E09E0208EC5300200F
:10357000009F020880B582B000AF0346FB710B4686
:10358000BB711346BB80BB79002B02D0012B48D006
:1035900084E0444BB3F940301A46424BB3F9423011
:1035A0001A44BB889A4232DABA88FB793D4918330B
:1035B0005B000B44B3F9043019463A4BB3F9483079
:1035C000CB1A9A4223DAFB79B7F90410354A14333F
:1035D0005B0013440A461A81FB79324A14335B00BC
:1035E0001344B3F908309AB22E4BB3F942309BB270
:1035F000D31A9AB2FB7911B22A4A14335B001344EE
:103600000A469A80274B002283F84A2046E000228F
:10361000254926480CF088F9224B022283F84A20DB
:103620003CE0BA88FB791F4914335B000B44B3F9C3
:10363000083019461B4BB3F948300B449A4223DD3E
:10364000FB79B7F90410174A18335B0013440A4694
:103650009A80FB79134A18335B001344B3F90430A2
:103660009AB2104BB3F942309BB213449AB2FB7931
:1036700011B20C4A18335B0013440A461A81094BF5
:10368000002283F84A2008E00022094907480CF08C
:103690004BF9044B022283F84A2000BF00BF0837D1
:1036A000BD4680BD48010020249F0208EC53002045
:1036B000009F020880B400AFAA4B1B78002B40F09B
:1036C0004A81A94B1B680133A74A1360A74B93F8A3
:1036D0002A30012B04D0A54B93F82B30012B03D1BA
:1036E000A34B01221A600CE0A04B93F82A30002B68
:1036F00004D09E4B93F82B30002B02D19C4B002220
:103700001A609A4B93F82830012B4FD1994B93EDC7
:10371000157A994BD3ED007AB4EEE77AF1EE10FA10
:1037200044DD944B93ED167A934BD3ED007AB4EECF
:10373000E77AF1EE10FA39DD904B01221A60904BD6
:103740001B6801338E4A13608D4B1A688D4B1B68C2
:103750009A4240F30281854B93F82A30002B05D022
:10376000824B93F82B30002B40F0F780804B0122E6
:103770001A607E4B012283F82A207C4B012283F8B9
:103780002B207A4B012283F82920784B93F82920AB
:103790007D4BDA70754B93F829207B4B1A717A4B6D
:1037A00001229A70794B0322DA70D6E0714B93EDC7
:1037B000157A774BD3ED007AB4EEE77AF1EE10FA92
:1037C0000AD46C4B93ED167A714BD3ED007AB4EEBC
:1037D000E77AF1EE10FA3BD5684B4FF0FF321A60F2
:1037E000674B1B68013B664A13606A4B1B685A4271
:1037F000634B1B689A4240F3B2805C4B93F82A30CB
:10380000012B05D0594B93F82B30012B40F0A780AA
:10381000574B00221A60554B002283F82A20534B45
:10382000002283F82B20514B022283F829204F4B92
:1038300093F82920544BDA704C4B93F82920524BC3
:103840001A71514B01229A70504BFD22DA7086E0BA
:10385000484B93ED157A504BD3ED007AB4EEE77AEE
:10386000F1EE10FA70D5434B93ED157A4A4BD3ED38
:10387000007AF1EE677AB4EEE77AF1EE10FA63DDE2
:103880003C4B93ED167A444BD3ED007AB4EEE77AD5
:10389000F1EE10FA58D5374B93ED167A3E4BD3ED37
:1038A000007AF1EE677AB4EEE77AF1EE10FA4BDDCA
:1038B0002E4B93F82A30012B04D02C4B93F82B304D
:1038C000012B32D12D4B4FF0FF321A602C4B1B686D
:1038D000013B2B4A1360314B1B685A42284B1B6833
:1038E0009A4230DD224B00221A60204B002283F8DE
:1038F0002A201E4B002283F82B201C4B022283F827
:1039000029201A4B93F829201F4BDA70174B93F894
:1039100029201D4B1A711C4B01229A701B4BFD2252
:10392000DA70174B00221A600DE0104B93F82A3022
:10393000002B04D00D4B93F82B30002B30D1104BC3
:1039400000221A602CE02BE00C4B00221A600C4B7A
:1039500000221A6025E000BF23E000BF21E000BF85
:103960001FE000BF7203002080030020D801002068
:103970007C03002048010020000000207403002088
:10398000780300200C0000204403002028030020BE
:103990000400002010000020080000201400002077
:1039A00000BFBD465DF8047B704700BF80B483B0A4
:1039B00000AF0346FB712A4B93ED1B7AFB79284A33
:1039C00002339B0013440433D3ED007AF6EE006A11
:1039D00067EEA67AB4EEE77AF1EE10FA00DC38E092
:1039E000FB791F4A02339B0013440433D3ED007A62
:1039F000B6EE007A67EE877A194BC3ED1B7A184B47
:103A0000DB6E174A1367164BDB6E154A5367144B70
:103A1000D3ED1C7A77EEA77AFCEEE77AC7ED007A51
:103A20003B78DAB20F4B9A710D4BD3ED1D7A77EEDE
:103A3000A77AFCEEE77AC7ED007A3B78DAB2094B59
:103A4000DA71074B93F87C20064B1A72054B012262
:103A50005A7100BF0C37BD465DF8047B704700BF4C
:103A60004801002044030020B0B594B000AF4FF0EF
:103A700080437B644FF47A733B6441F28833FB6389
:103A8000A74B07F10C041D460FCD0FC40FCD0FC47B
:103A900095E8030084E80300A24A3B1D92E8030076
:103AA00083E803000A2387F83B30022387F83A3083
:103AB0000CF0BAFB78639C4B5B78092B03D09A4BD4
:103AC0009B78092B1DD1994B00221A70974B00222D
:103AD0005A70974B4FF000025A60954B5B68954ABD
:103AE0005360934B4FF000021A60914B1B68914A50
:103AF0001360914B00221A708B4B09221A7000F050
:103B00001DBC894B5B78012B3DD1874B9B78012BEA
:103B100039D1002289498A480BF006FF824B0122E5
:103B20001A70884B1B6D884A1360864B5B6D874A01
:103B300013607F4B4FF000025A607D4B5B687D4AFB
:103B400053607B4B4FF000021A60794B1B68794A37
:103B50001360764B00221A70774B00221A70734B59
:103B600000225A70704B00229A606F4B9B686E4A1D
:103B70005360774B01221A70764B03221A706E4BFA
:103B800003221A70DAE3684B5B68002B42D1664B64
:103B90009B68002B3ED1654B05221A70664B0322B1
:103BA0001A70624B03225A707B68624A53607B68CA
:103BB0005F4A53605C4A7B6B53615B4B5B695A4A5B
:103BC0001361604B93ED147AD7ED037A77EE277A81
:103BD0005D4BC3ED007A5B4B93ED157AD7ED037A1D
:103BE00077EE277A594BC3ED007A574B5B6B4E4A01
:103BF0001362564B5B6B4C4A53624B4B01229A60EB
:103C0000494B9B68484A5360002253494C480BF08B
:103C10008BFE93E3444B5B78002B40F0B981424B21
:103C20001B697A6BD31A404A9361474B93ED117A23
:103C3000D7ED117AF1EE677AB4EEE77AF1EE10FA89
:103C400040F1BF80404B93ED0D7A374BD3ED087AAE
:103C500077EE677AF5EEC07AF1EE10FA08DD3A4BAE
:103C600093ED0D7A304BD3ED087A77EE677A09E061
:103C7000354BD3ED0D7AB1EE677A2B4BD3ED087A45
:103C800077EE677AC7ED137AD7ED137A9FED337A23
:103C9000F4EEC77AF1EE10FA07DD9FED317AD7ED39
:103CA000137A77EE677AC7ED137AD7ED137A9FED23
:103CB0002C7AF4EEC77AF1EE10FA40F382802948AC
:103CC0000CF078F8184B9B7B0133DAB2164B9A73E1
:103CD000154A7B6B13611C4B5B6B134A1362124BCF
:103CE0009B7B97F83B209A4252D80F4B00229A7345
:103CF0000D4B1B7B0133DAB20B4B1A730A4B1B7B48
:103D000097F83A209A4231D817480CF053F8064BEE
:103D100009225A70074B4FF000025A600EE300BFB1
:103D2000E4A202080CA30208B8000020AC030020A3
:103D30000407002074050020040C0020489F02089E
:103D4000EC530020980A00207C040020F804002096
:103D5000E000002018000020609F020800003443AB
:103D60000000B443849F0208C89F0208A34B1B7B3A
:103D70009B0050333B444C3BD3ED007A0120B0EE26
:103D8000670A0CF011F9034619469D480CF012F829
:103D90009C4B93ED147A994B9B7B9B0050333B4497
:103DA000443BD3ED007A77EE277A974BC3ED007A48
:103DB000924B1B7B9B0050333B444C3B1B68934A0C
:103DC0005360914BD3ED117AF5EEC07AF1EE10FA13
:103DD00003DD8D4BD3ED117A04E08B4BD3ED117ADB
:103DE000F1EE677A97ED117AF4EEC77AF1EE10FAF8
:103DF00067DD824B9B69FA6B9A4280F0D1807F4BE2
:103E00009B7B19467D4B1B7B1A4681480BF0D2FFEA
:103E10007A4B9B7B0133DAB2784B9A73774A7B6B90
:103E20001361794B5B6B754A1362744B9B7B97F8FC
:103E30003B209A422BD8714B00229A736F4B1B7B0D
:103E40000133DAB26D4B1A736C4B1B7B97F83A2037
:103E50009A420AD86F480BF0ADFF684B09225A709E
:103E60006A4B4FF000025A6068E2644B1B7B9B0078
:103E700050333B444C3BD3ED007A0120B0EE670A4F
:103E80000CF092F8034619465D480BF093FF5D4B2A
:103E900093ED147A594B9B7B9B0050333B44443B3E
:103EA000D3ED007A77EE277A574BC3ED007A534B68
:103EB0001B7B9B0050333B444C3B1B68534A536075
:103EC0006EE04E4B9B693A6C9A4269D24B4B9B7B9E
:103ED00019464A4B1B7B1A464F480BF06BFF474B6A
:103EE0009B7B0133DAB2454B9A73444A7B6B136177
:103EF000454B5B6B414A1362404B9B7B97F83B20E1
:103F00009A422BD83D4B00229A733C4B1B7B0133CA
:103F1000DAB23A4B1A73394B1B7B97F83A209A4224
:103F20000AD83E480BF046FF344B09225A70374BF3
:103F30004FF000025A6001E2304B1B7B9B00503374
:103F40003B444C3BD3ED007A0120B0EE670A0CF005
:103F50002BF8034619462A480BF02CFF294B93ED0A
:103F6000147A264B9B7B9B0050333B44443BD3ED60
:103F7000007A77EE277A244BC3ED007A1F4B1B7B28
:103F80009B0050333B444C3B1B68204A536007E086
:103F90001E4B4FF000025A601C4B4FF000021A609B
:103FA000164B9B78002B40F0C181144B5B697A6BF8
:103FB000D31A124AD3611A4B93ED117AD7ED117AC5
:103FC000F1EE677AB4EEE77AF1EE10FA40F1AB80E9
:103FD000134B93ED0D7A094BD3ED097A77EE677A9F
:103FE000F5EEC07AF1EE10FA1CDD0D4B93ED0D7A73
:103FF000024BD3ED097A77EE677A1DE0B800002016
:104000000CA00208980A00207C04002074050020FF
:104010002CA0020868A00208A8A00208F0A00208CC
:10402000F80400209E4BD3ED0D7AB1EE677A9D4BDC
:10403000D3ED097A77EE677AC7ED127AD7ED127A67
:104040009FED997AF4EEC77AF1EE10FA07DD9FED55
:10405000977AD7ED127A77EE677AC7ED127AD7EDB5
:10406000127A9FED927AF4EEC77AF1EE10FA5ADDE9
:104070008F480BF09FFE8B4BDB7B0133DAB2894B11
:10408000DA73884A7B6B5361854B5B6B854A53625D
:10409000844BDB7B97F83B209A422BD8814B002244
:1040A000DA73804B5B7B0133DAB27E4B5A737D4B04
:1040B0005B7B97F83A209A420AD87E480BF07AFE4A
:1040C000784B09229A707C4B4FF000025A6035E120
:1040D000744B5B7B9B0050333B444C3BD3ED007AED
:1040E0000120B0EE670A0BF05FFF034619467348E4
:1040F0000BF060FE724B93ED157A6A4BDB7B9B00F5
:1041000050333B44443BD3ED007A77EE277A644B3F
:10411000C3ED007A634B5B7B9B0050333B444C3BCD
:104120001B68654A53605E4BD3ED117AF5EEC07A99
:10413000F1EE10FA03DD5A4BD3ED117A04E0584B3F
:10414000D3ED117AF1EE677A97ED117AF4EEC77A32
:10415000F1EE10FA67DD534BDB69FA6B9A4280F09F
:10416000ED80504BDB7B19464E4B5B7B1A46554826
:104170000BF020FE4B4BDB7B0133DAB2494BDA7399
:10418000484A7B6B5361464B5B6B464A5362454BD7
:10419000DB7B97F83B209A422BD8424B0022DA7304
:1041A000404B5B7B0133DAB23E4B5A733D4B5B7B3A
:1041B00097F83A209A420AD843480BF0FBFD394B56
:1041C00009229A703C4B4FF000025A60B6E0354B22
:1041D0005B7B9B0050333B444C3BD3ED007A01208A
:1041E000B0EE670A0BF0E0FE0346194633480BF0C9
:1041F000E1FD334B93ED157A2A4BDB7B9B0050336B
:104200003B44443BD3ED007A77EE277A244BC3ED51
:10421000007A244B5B7B9B0050333B444C3B1B6838
:10422000254A53608AE01F4BDB693A6C9A4280F062
:1042300085801C4BDB7B19461A4B5B7B1A46234857
:104240000BF0B8FD174BDB7B0133DAB2154BDA7399
:10425000144A7B6B5361124B5B6B124A5362114BD6
:10426000DB7B97F83B209A4246D80E4B0022DA734C
:104270000C4B5B7B0133DAB20A4B5A73094B5B7B05
:1042800097F83A209A4225D811480BF093FD054B38
:1042900009229A70084B4FF000025A604EE000BFAE
:1042A000F8040020B8000020000034430000B443AC
:1042B00034A1020878A1020804070020BCA102086A
:1042C000980A0020DCA1020818A2020858A20208DD
:1042D000A0A202081B4B5B7B9B0050333B444C3B32
:1042E000D3ED007A0120B0EE670A0BF05DFE0346C5
:1042F000194615480BF05EFD144B93ED157A114BE2
:10430000DB7B9B0050333B44443BD3ED007A77EE9C
:10431000277A0F4BC3ED007A0A4B5B7B9B0050332F
:104320003B444C3B1B680B4A536007E0094B4FF082
:1043300000025A60074B4FF000021A605037BD462A
:10434000B0BD00BFB8000020BCA10208980A002040
:10435000F80400200407002090B593B000AF4FF0A0
:1043600080433B64974B3C1D0FCB84E80F00964B7A
:10437000FB63964BBB63964B7B630BF055FF386337
:10438000944B5B78092B03D0924B9B78092B1CD163
:10439000914B00221A70904B00225A708F4B4FF0B5
:1043A00000025A608D4B5B688D4A53608B4B4FF017
:1043B00000021A60894B1B68894A1360894B0022EE
:1043C0001A70844B09221A70CCE2824B5B78012B65
:1043D00032D1804B9B78012B2ED17E4B1B78012B49
:1043E00005D081480BF0E6FC7A4B01221A707B4B1A
:1043F0004FF000025A60794B5B68794A5360774B03
:104400004FF000021A60754B1B68754A1360724BBF
:1044100000221A70734B00221A706F4B00225A70E0
:10442000724B1B78002B00F09C82714B03221A7098
:104430006C4B03221A7094E2664BDB78002B50D150
:10444000644B1B79002B4CD1634B05221A70654BD2
:1044500003221A70604B03225A705E4A3B6BD36092
:104460005C4BDB685B4A93605A4B01221A71594BD3
:104470001A79584BDA70574B02225A76554B5A7EAE
:10448000544B1A765B4B1B6B524AD3615A4B1B6BD6
:10449000504A1362594BB3F9143007EE903AF8EED4
:1044A000E77A4C4BC3ED097A544BB3F9163007EE5B
:1044B000903AF8EEE77A474BC3ED0A7AFB68474A31
:1044C0005360464B5B68464A5360444B4FF00002D2
:1044D0001A60424B1B68424A136049480BF06AFC61
:1044E00040E200237B6437E23A4A7B6C1344013399
:1044F0001B78002B40F02C827B6C002B02D13D4BB3
:104500005B6C01E03C4B5B6CFB627B6C002B02D173
:10451000384B1B6B01E0384B1B6BBB627B6C002B79
:1045200007D1364BB3F9143007EE903AF8EEE77A3C
:1045300006E0324BB3F9163007EE903AF8EEE77A20
:10454000C7ED097A97ED0B7AD7ED0D7AB4EEE77ADD
:10455000F1EE10FA5FDD1F4A7B6C134418331B78B1
:10456000002B58D01B4A7B6C134418331B78013B3B
:10457000D9B2184A7B6C134418330A461A70154A8C
:104580007B6C134418331B789B0048333B44443BFB
:104590001B683B627B6C002B01D11A4C00E01A4C6B
:1045A000012097ED080A0BF0FFFC03461A4621464E
:1045B00016480BF0FFFB7B6C002B29D1084A3B6AA5
:1045C000536028E020A5020800C05A45000034438B
:1045D00000007A43E0000020AC0300200407002024
:1045E00074050020040C002014A30208F50B002021
:1045F000180000207C040020F8040020480100205E
:1046000034A3020860A3020868A3020870A302088A
:10461000A84A3B6A5360D7ED107AF1EE677A97EDBE
:104620000B7AB4EEE77AF1EE10FA33D5A24A7B6C3E
:1046300006339B001344043393ED007AD7ED0A7AD6
:1046400077EE677AC7ED077A97ED077AD7ED0E7A9E
:10465000B4EEE77AF1EE10FA1CDD7B6C002B01D191
:10466000964B00E0964B194696480BF0A3FB924AF6
:104670007B6C1344013309221A707B6C002B04D12C
:10468000914B4FF000025A606CE18A4B4FF00002F0
:104690005A6067E1884A7B6C023352F823303A6BE8
:1046A000D31A44F6206293421CD97B6C002B01D1B3
:1046B000824B00E0824B194684480BF07BFB7E4A1C
:1046C0007B6C1344013309221A707B6C002B04D1DC
:1046D0007D4B4FF000025A6044E1764B4FF00002F0
:1046E0005A603FE1744A7B6C08339B0013440433E7
:1046F000D3ED007A97ED097A77EE677A97ED0F7A26
:10470000B4EEE77AF1EE10FA1CD57B6C002B01D1E8
:104710006A4B00E06A4B19466D480BF04BFB664A4A
:104720007B6C1344013309221A707B6C002B04D17B
:10473000654B4FF000025A6014E15E4B4FF00002EF
:104740005A600FE1D7ED0B7AF5EEC07AF1EE10FA70
:1047500002DDD7ED0B7A03E0D7ED0B7AF1EE677A45
:1047600097ED107AF4EEC77AF1EE10FACCBF012380
:104770000023DBB2FB76504A7B6C13442C331B784E
:10478000002B08D0FB7E002B05D14B497B6C0433FA
:104790003A6B41F82320FB7E002B40F0D280464A42
:1047A0007B6C043352F823303A6BD31A40F2EE227A
:1047B000934240F2C680404A7B6C13442C331B78F2
:1047C000002B35D07B6C002B01D13C4B00E03C4BE7
:1047D000194640480BF0EEFA7B6C002B04D13A4BA3
:1047E0004FF000025A6003E0324B4FF000025A6073
:1047F000796C39480BF0DEFA7B6CDBB21846FEF7B9
:10480000AFFD796C35480BF0D5FA2B4A7B6C13441D
:10481000013301221A707B6C002B04D12A4B4FF01C
:1048200000025A6087E0234B4FF000025A6082E09A
:10483000214A7B6C134418331B78022B52D81E4A32
:104840007B6C134418331B780133D9B21A4A7B6C42
:10485000134418330A461A70174A7B6C13441833F2
:104860001B789B0048333B44443B1B687B617B6C5B
:10487000002B01D1114C00E0114C012097ED050AED
:104880000BF092FB03461A46214615480BF092FAAC
:104890007B6C002B03D10C4A7B69536002E0054A14
:1048A0007B695360044A7B6C13442C3300221A70DA
:1048B00041E000BF04070020E000002060A30208E0
:1048C00068A302089CA3020874050020D0A3020874
:1048D0000CA4020840A4020868A402088CA40208E0
:1048E000B0A402087B6C002B01D1204B00E0204BD0
:1048F000194620480BF05EFA7B6C002B04D11E4B4E
:104900004FF000025A6003E01C4B4FF000025A6067
:10491000796C1B480BF04EFA7B6CDBB21846FEF745
:104920001FFD796C17480BF045FA174A7B6C13444E
:10493000013301221A7014497B6C04333A6B41F83D
:104940002320114A7B6C13442C33FA7E1A7000E04A
:1049500000BF7B6C01337B647B6C012B7FF7C4ADA4
:1049600000E000BF4C37BD4690BD00BF60A3020809
:1049700068A30208DCA402087405002004070020D4
:1049800068A402088CA40208E000002080B483B070
:1049900000AF78607B689B6843F080427B689A60D8
:1049A00000BF0C37BD465DF8047B704780B582B010
:1049B00002AF00F0F5FE00F02FFF134B1B68012B38
:1049C0001DD1124B9B78012B19D1114B1B68013360
:1049D0000F4A13600F4B00930F4B104A10491148B8
:1049E00000F09CF8104B0093104B114A0C491148F1
:1049F00000F094F8104A0A490A4800F055FA00F00D
:104A00001DF800BFBD4680BD04090020AC03002096
:104A100014090020280400207C040020A0050020A8
:104A2000E0030020B803002040040020F804002028
:104A300030070020CA0300200004002080B500AF2A
:104A4000354B1B78082B59D801A252F823F000BF30
:104A5000754A01089B4A0108C14A0108D14A010868
:104A6000D14A0108D14A0108D14A0108D74A0108B0
:104A7000DD4A0108284B9B78012B02D1264B0122ED
:104A80001A700121012004F055F80121022004F0E0
:104A900051F8214B00225A703CE00121012004F022
:104AA00049F80121022004F045F81B4B00225A70FE
:104AB00001F0FEFD01F0CEFE174B02221A7029E034
:104AC00001F0F6FD01F0C6FE134B00225A7021E002
:104AD00000F03AFA1EE000F0A7FD1BE00E4B0022AA
:104AE0005A700121012004F025F80121022004F070
:104AF00021F801F0DDFD01F0ADFE0BE00121012008
:104B000004F018F80121022004F014F8024B0022EE
:104B10001A7000BF00BF80BDAC03002080B586B016
:104B200000AFF860B9607A603B6000237B613B6A4C
:104B300093ED007ABB68D3ED057AB4EEE77AF1EE37
:104B400010FA06DDFB6801221A727B6943F001034B
:104B50007B613B6A93ED017ABB68D3ED057AB4EED5
:104B6000E77AF1EE10FA06DDFB6801225A727B69E2
:104B700043F480737B613B6A93ED027ABB68D3EDAB
:104B8000057AB4EEE77AF1EE10FA06DDFB68012251
:104B90009A727B6943F480337B613B6A93ED007AC0
:104BA000BB68D3ED047AB4EEE77AF1EE10FA06D5DD
:104BB000FB6801225A717B6943F002037B613B6A07
:104BC00093ED017ABB68D3ED047AB4EEE77AF1EEA7
:104BD00010FA06D5FB6801229A717B6943F40073D1
:104BE0007B613B6A93ED027ABB68D3ED047AB4EE45
:104BF000E77AF1EE10FA06D5FB680122DA717B69DB
:104C000043F400337B613B6A93ED037ABB68D3EDD9
:104C1000077AB4EEE77AF1EE10FA07D5FB680122C5
:104C2000DA727B6943F004037B6111E03B6A93ED28
:104C3000037ABB68D3ED067AB4EEE77AF1EE10FAA8
:104C400006DDFB680122DA727B6943F008037B61B1
:104C50003B6A93ED047ABB68D3ED077AB4EEE77A4A
:104C6000F1EE10FA07D5FB6801221A737B6943F451
:104C700080637B6111E03B6A93ED047ABB68D3EDFE
:104C8000067AB4EEE77AF1EE10FA06DDFB6801224F
:104C90001A737B6943F400637B613B6A93ED057A89
:104CA000BB68D3ED077AB4EEE77AF1EE10FA07D5D8
:104CB000FB6801225A737B6943F480237B6111E016
:104CC0003B6A93ED057ABB68D3ED067AB4EEE77ADA
:104CD000F1EE10FA06DDFB6801225A737B6943F49A
:104CE00000237B617B68D3ED007AF5EEC07AF1EEAC
:104CF00010FA03DD7B68D3ED007A04E07B68D3ED26
:104D0000007AF1EE677ABB6893ED027AF4EEC77A27
:104D1000F1EE10FA06DDFB6801221A707B6943F0A0
:104D200010037B617B68D3ED017AF5EEC07AF1EE7A
:104D300010FA03DD7B68D3ED017A04E07B68D3EDE4
:104D4000017AF1EE677ABB6893ED027AF4EEC77AE6
:104D5000F1EE10FA06DDFB6801225A707B6943F41C
:104D600080537B617B68D3ED027AF5EEC07AF1EE79
:104D700010FA03DD7B68D3ED027A04E07B68D3EDA3
:104D8000027AF1EE677ABB6893ED027AF4EEC77AA5
:104D9000F1EE10FA06DDFB6801229A707B6943F49C
:104DA00080137B617B68D3ED057AF5EEC07AF1EE76
:104DB00010FA03DD7B68D3ED057A04E07B68D3ED60
:104DC000057AF1EE677ABB6893ED027AF4EEC77A62
:104DD000F1EE10FA06DDFB680122DA707B6943F020
:104DE00080737B617B68D3ED067AF5EEC07AF1EED5
:104DF00010FA03DD7B68D3ED067A04E07B68D3ED1F
:104E0000067AF1EE677ABB6893ED027AF4EEC77A20
:104E1000F1EE10FA06DDFB6801221A717B6943F09E
:104E200080737B613B68D3ED117AF5EEC07AF1EEC9
:104E300010FA03DD3B68D3ED117A04E03B68D3ED53
:104E4000117AF1EE677ABB6893ED037AF4EEC77AD4
:104E5000F1EE10FA06DDFB6801229A737B6943F0DC
:104E600080637B610E4B1B6803F07F437A691343B9
:104E70007B610B4B1B687A699A420CD0084A7B69AC
:104E80001360084B1B78002B05D0054B1B68194697
:104E9000F32004F0F5FF00BF1837BD4680BD00BF0A
:104EA000140C0020180C002080B586B000AFF8600C
:104EB000B9607A6000237B617B6893ED017ABB68FF
:104EC000D3ED007AB4EEE77AF1EE10FA07DDFB6875
:104ED000012283F825207B6943F080437B617B6856
:104EE00093ED017ABB68D3ED017AB4EEE77AF1EE87
:104EF00010FA07D5FB68012283F824207B6943F070
:104F000000437B610E4B1B6823F07F437A69134398
:104F10007B610B4B1B687A699A420CD0084A7B690B
:104F20001360084B1B78002B05D0054B1B681946F6
:104F3000F32004F0A5FF00BF1837BD4680BD00BFB9
:104F4000140C0020180C002080B500AF384B5B78A3
:104F500003F00103002B20D0012B25D1354B1B681A
:104F6000002B0ED0344B1B68013303F00103002BE0
:104F70000ED000F067F8314B1B6801332F4A1360E5
:104F800006E000F05FF82D4B1B6801332B4A1360DD
:104F90000021012003F0CEFD0DE001F089FB01218D
:104FA000012003F0C7FD06E001F082FB0121012092
:104FB00003F0C0FD00BF1E4B5B785B08DBB203F063
:104FC0000103002B1FD0012B24D11A4B1B68002B8F
:104FD0000DD0194B1B6803F00103002B0ED000F01D
:104FE000A9F9174B1B680133154A136006E000F05E
:104FF000A1F9134B1B680133114A136000210220F1
:1050000003F098FD0DE001F025FC0121022003F0E2
:1050100091FD06E001F01EFC0121022003F08AFD53
:1050200000BF054B1B680133034A136000BF80BDFE
:10503000AC0300201C000020080900200C090020FF
:105040001009002080B500AFF7EE000AB7EE000AA5
:105050009F49A04802F0A6F99F4B1B78062B18D158
:105060009E4BD3ED077A9D4B93ED017A9B4BD3ED8D
:10507000096AB0EE661A9A499A48F0EE470AB0EE0D
:10508000670A01F053FFF0EE407A974BC3ED027AC6
:1050900007E0F7EE000AB7EE000A9449924802F0E2
:1050A00081F9914B93ED637A914BD3ED117A27EE11
:1050B000277A904BD3ED187A67EE277A8A4BC3EDA7
:1050C0004C7A894BD3ED037A874B93ED117A834B5E
:1050D000D3ED026AB0EE661A87498848F0EE470AB7
:1050E000B0EE670A01F072FEF0EE407A7E4BC3ED3F
:1050F000147A7D4BD3ED027A7B4B93ED107A774B8C
:10510000D3ED026AB0EE661A7D497E48F0EE470A9A
:10511000B0EE670A01F05AFEF0EE407A724BC3ED32
:10512000137A714B93ED137A6F4BD3ED137A27EE0D
:10513000277A6D4BD3ED146A6B4BD3ED147A66EE80
:10514000A77A77EE277AB0EE670A13F04BFEF0EEFF
:10515000407A654BC3ED267A634B93ED277A624B19
:10516000D3ED267A77EE677AF5EEC07AF1EE10FA93
:1051700012DD654B93ED027A5B4BD3ED276A5A4BF8
:10518000D3ED267A76EEE77A27EE277A564BD3EDE3
:10519000267A77EE277A13E05B4BD3ED027AB1EEF5
:1051A000677A514BD3ED266A4F4BD3ED277A76EED3
:1051B000E77A27EE277A4C4BD3ED267A77EE277ADB
:1051C000494BC3ED277A484B93ED277AF7EE006AF7
:1051D000C6EE877A444BC3ED287A3F4B1B78032BEE
:1051E00006D1434B494A4A494A4801F0B5FC3AE0E6
:1051F0003D4B93ED277A394BD3ED027AB4EEE77A43
:10520000F1EE10FA20DD384B93ED137A334BD3EDEA
:10521000027A27EE277A344BD3ED287A67EE277A85
:10522000314BC3ED157A304B93ED147A2B4BD3ED04
:10523000027A27EE277A2C4BD3ED287A67EE277A6D
:10524000294BC3ED167A07E0274BDB6C264A5365E2
:10525000254B1B6D244A9365254B2F4A2C492D481D
:1052600001F07AFC00BF1D4BD3ED037AB0EE670A64
:105270002A49284801F0D6FC1D4B294A29492748CC
:1052800001F01EFC184B93ED147A174BD3ED257AE1
:1052900077EE677A144BC3ED4D7A134B93ED137A87
:1052A000114BD3ED247A77EE677A0F4BC3ED457A35
:1052B0000A4B1D4A19491D4801F0CEFE1B49012029
:1052C00002F036F803461A46194B5A7400BF80BDE7
:1052D0008005002078050020AC0300200004002099
:1052E00060060020D0060020740500207C05002008
:1052F0007C040020D80100204006002090060020F9
:105300003006002070060020EC08002098050020E0
:10531000D0050020D8050020C8050020F005002099
:1053200004060020FC0500201806002024060020AA
:10533000B803002080B500AFF7EE000AB7EE000A10
:10534000A049A14802F02EF8A04B1B78062B18D1DB
:105350009F4BD3ED077A9E4B93ED017A9C4BD3ED97
:10536000096AB0EE661A9B499B48F0EE470AB0EE18
:10537000670A01F0DBFDF0EE407A984BC3ED027A4C
:1053800007E0F7EE000AB7EE000A9549934802F0ED
:1053900009F8924B93ED637A924BD3ED117A27EE95
:1053A000277A914BD3ED197A67EE277A8B4BC3EDB1
:1053B0004C7A8A4BD3ED037A884B93ED117A844B68
:1053C000D3ED026AB0EE661A88498948F0EE470AC2
:1053D000B0EE670A01F0FAFCF0EE407A7F4BC3EDC5
:1053E000147A7E4BD3ED027A7C4B93ED107A784B96
:1053F000D3ED026AB0EE661A7E497F48F0EE470AA6
:10540000B0EE670A01F0E2FCF0EE407A734BC3EDB8
:10541000137A724B93ED137A704BD3ED137A27EE18
:10542000277A6E4BD3ED146A6C4BD3ED147A66EE8B
:10543000A77A77EE277AB0EE670A13F0D3FCF0EE86
:10544000407A664BC3ED267A644B93ED277A634B23
:10545000D3ED267A77EE677AF5EEC07AF1EE10FAA0
:1054600012DD664B93ED027A5C4BD3ED276A5B4B02
:10547000D3ED267A76EEE77A27EE277A574BD3EDEF
:10548000267A77EE277A13E05C4BD3ED027AB1EE01
:10549000677A524BD3ED266A504BD3ED277A76EEDE
:1054A000E77A27EE277A4D4BD3ED267A77EE277AE7
:1054B0004A4BC3ED277A494B93ED277AF7EE006A02
:1054C000C6EE877A454BC3ED287A404B1B78032BF9
:1054D00006D1444B4A4A4B494B4801F03DFB3AE068
:1054E0003E4B93ED277A3A4BD3ED027AB4EEE77A4E
:1054F000F1EE10FA20DD394B93ED137A344BD3EDF6
:10550000027A27EE277A354BD3ED287A67EE277A91
:10551000324BC3ED157A314B93ED147A2C4BD3ED0E
:10552000027A27EE277A2D4BD3ED287A67EE277A79
:105530002A4BC3ED167A07E0284BDB6C274A5365EC
:10554000264B1B6D254A9365264B304A2D492E4824
:1055500001F002FB00BF1E4BD3ED037AB0EE670AE9
:105560002B49294801F05EFB1E4B2A4A2A4928484C
:1055700001F0A6FA194B93ED147A184BD3ED257A66
:1055800077EE677A154BC3ED4D7A144B93ED137A92
:10559000124BD3ED247A77EE677A104BC3ED457A40
:1055A0000B4B1E4A1A491E4801F056FD1C490220A9
:1055B00001F0BEFE03461A461A4B83F8232000BFB3
:1055C00080BD00BF1007002008070020AC030020AA
:1055D00000040020F00700206008002004070020DD
:1055E0000C070020F8040020D8010020D00700207C
:1055F00020080020C007002000080020EC08002040
:1056000028070020600700206807002058070020B6
:1056100080070020940700208C070020A8070020A6
:10562000B4070020B803002080B500AF294B5B7899
:1056300003F00103002B13D0012B18D1264B93F854
:105640002130012B05D100F04BF8234B002283F8C9
:105650002120FFF7F7FC0021012003F06BFA0DE099
:1056600001F026F80121012003F064FA06E001F0C0
:105670001FF80121012003F05DFA00BF154B5B7894
:105680005B08DBB203F00103002B13D0012B18D110
:10569000124B93F82130012B05D100F051F80F4B3C
:1056A000002283F82120FFF745FE0021022003F0AD
:1056B00041FA0DE001F0CEF80121022003F03AFAA0
:1056C00006E001F0C7F80121022003F033FA00BF21
:1056D00000BF80BDAC0300207C040020F804002043
:1056E00080B500AFF2EE040AB2EE040A0E490F488C
:1056F00001F058FE0E4BD3ED077A0E4B93ED117A65
:105700000C4BD3ED136AB0EE661A0B490B48F0EE62
:10571000470AB0EE670A01F059FBF0EE407A044BFD
:10572000C3ED017A00BF80BD900500208C050020EC
:10573000740500207C04002050060020B0060020E4
:1057400080B500AFF2EE040AB2EE040A0E490F482B
:1057500001F028FE0E4BD3ED077A0E4B93ED117A34
:105760000C4BD3ED136AB0EE661A0B490B48F0EE02
:10577000470AB0EE670A01F029FBF0EE407A044BCD
:10578000C3ED017A00BF80BD200700201C07002068
:1057900004070020F8040020E00700204008002053
:1057A00080B400AF1A4B1A881A4B1A80184B5A88CB
:1057B000184B5A80164B9A88164B9A80144BDA88ED
:1057C000144BDA80124B1A89124B1A81104B5A89EA
:1057D000104B5A810E4B9A890E4B9A810C4BDA89E9
:1057E0000C4BDA810A4B1A8A0A4B1A82084B5A8AE6
:1057F000084B5A82064B9A8A064B9A82044BDA8AE5
:10580000044BDA8200BFBD465DF8047B704700BFE1
:10581000640A00209408002080B500AFB24B9B8A38
:1058200007EE903AB8EEE77AB04BD3ED197A67EE0F
:10583000277AAE4BC3ED007AAB4B1B8807EE903A4C
:10584000F8EE677AA94BC3ED0A7AA74B5B8807EE9F
:10585000903AF8EE677AA54BC3ED107AA24B1B89FC
:1058600007EE903AF8EE677AA04BC3ED0B7A9E4BA9
:105870005B8907EE903AF8EE677A9C4BC3ED117A9C
:10588000994B1B8A07EE903AF8EE677A974BC3ED77
:105890000C7A954B5B8A07EE903AF8EE677A934B59
:1058A000C3ED127A924B9B78002B03D0012B00F0B2
:1058B000778170E18E4B9B8801339AB28C4B9A8032
:1058C0008B4B9B8841F28832934207D9884B012247
:1058D0009A70874B41F289329A8062E1844B0022B0
:1058E0001A70834B00225A70814B00229A707F4BB2
:1058F00093ED0D7A7D4BD3ED0A7A77EE677AF5EE6C
:10590000C07AF1EE10FA12DD7A4B93ED027A774B02
:10591000D3ED0D6A754BD3ED0A7A76EEE77A27EE72
:10592000277A724BD3ED0A7A77EE277A13E0714B20
:10593000D3ED027AB1EE677A6C4BD3ED0A6A6B4B0A
:10594000D3ED0D7A76EEE77A27EE277A674BD3ED23
:105950000A7A77EE277A654BC3ED0D7A634B93EDA8
:105960000E7A624BD3ED0B7A77EE677AF5EEC07A5A
:10597000F1EE10FA12DD5F4B93ED027A5B4BD3ED43
:105980000E6A5A4BD3ED0B7A76EEE77A27EE277A3A
:10599000564BD3ED0B7A77EE277A13E0554BD3EDC8
:1059A000027AB1EE677A514BD3ED0B6A4F4BD3EDD0
:1059B0000E7A76EEE77A27EE277A4C4BD3ED0B7A08
:1059C00077EE277A494BC3ED0E7A484B93ED0F7A69
:1059D000464BD3ED0C7A77EE677AF5EEC07AF1EEAE
:1059E00010FA12DD434B93ED027A404BD3ED0F6A70
:1059F0003E4BD3ED0C7A76EEE77A27EE277A3B4BD7
:105A0000D3ED0C7A77EE277A13E03A4BD3ED027A96
:105A1000B1EE677A354BD3ED0C6A344BD3ED0F7A88
:105A200076EEE77A27EE277A304BD3ED0C7A77EED5
:105A3000277A2E4BC3ED0F7A2C4B93ED137A2B4B19
:105A4000D3ED107A77EE677AF5EEC07AF1EE10FAC0
:105A500012DD284B93ED027A244BD3ED136A234BCE
:105A6000D3ED107A76EEE77A27EE277A1F4BD3ED47
:105A7000107A77EE277A13E01E4BD3ED027AB1EE5F
:105A8000677A1A4BD3ED106A184BD3ED137A76EE82
:105A9000E77A27EE277A154BD3ED107A77EE277A3F
:105AA000124BC3ED137A114B93ED147A0F4BD3EDD8
:105AB000117A77EE677AF5EEC07AF1EE10FA1BDD17
:105AC0000C4B93ED027A094BD3ED146A074BD3EDDF
:105AD000117A76EEE77A27EE277A044BD3ED117A26
:105AE00077EE277A1CE000BF940800200004002015
:105AF000AC030020E0080020BE4BD3ED027AB1EEEB
:105B0000677ABD4BD3ED116ABB4BD3ED147A76EEB9
:105B1000E77A27EE277AB84BD3ED117A77EE277A1A
:105B2000B54BC3ED147AB44B93ED157AB24BD3ED6C
:105B3000127A77EE677AF5EEC07AF1EE10FA12DD9E
:105B4000AC4B93ED027AAC4BD3ED156AAA4BD3ED77
:105B5000127A76EEE77A27EE277AA74BD3ED127A00
:105B600077EE277A13E0A34BD3ED027AB1EE677A92
:105B7000A14BD3ED126AA04BD3ED157A76EEE77AFE
:105B800027EE277A9C4BD3ED127A77EE277A9A4B41
:105B9000C3ED157A05E0994B012283F8262000E039
:105BA00000BF954B93ED0A7A934BD3ED0D7A37EE08
:105BB000677A914BD3ED1A7A67EE277A904BC3ED53
:105BC0000B7A8D4B93ED0B7A8B4BD3ED0E7A37EE30
:105BD000677A894BD3ED1A7A67EE277A884BC3ED43
:105BE0000C7A854B93ED0C7A834BD3ED0F7A37EE1D
:105BF000677A814BD3ED1A7A67EE277A804BC3ED33
:105C00000D7A7D4B93ED107A7B4BD3ED137A37EE03
:105C1000677A794BD3ED1A7A67EE277A794BC3ED21
:105C20000B7A754B93ED117A734BD3ED147A37EEF3
:105C3000677A714BD3ED1A7A67EE277A714BC3ED11
:105C40000C7A6D4B93ED127A6B4BD3ED157A37EEE0
:105C5000677A694BD3ED1A7A67EE277A694BC3ED01
:105C60000D7A694B9A88694BA3F85C20664BDA88F9
:105C7000674BA3F85C20644B9A89644BA3F85E20C1
:105C8000614BDA89624BA3F85E206049012001F084
:105C900073FD03461A46594B1A745D49022001F000
:105CA0006BFD03461A46554B83F82220524B93ED69
:105CB000017A514BD3ED007A77EE677AF5EEC07A30
:105CC000F1EE10FA12DD534B93ED027A4A4BD3ED0D
:105CD000016A494BD3ED007A76EEE77A27EE277A10
:105CE000454BD3ED007A77EE277A13E0494BD3ED9D
:105CF000027AB1EE677A404BD3ED006A3E4BD3EDAA
:105D0000017A76EEE77A27EE277A3B4BD3ED007ADD
:105D100077EE277A384BC3ED017A374BD3ED017A12
:105D20009FED3D7A27EE877A334BD3ED1B7A67EEF2
:105D3000277A314BC3ED027A2F4BD3ED027A9FEDD8
:105D4000377A67EE877A2C4BC3ED087A2A4BD3ED6E
:105D5000017AB6EE007A67EE877A274BC3ED047AB4
:105D6000254B93ED047A244BD3ED1B7A67EE277A0B
:105D7000214BC3ED037A204B93ED047AF7EE006AD2
:105D8000C6EE877A1C4BC3ED057A1B4B93ED1D7A4B
:105D9000194BD3ED057A67EE277A174BC3ED067AD8
:105DA000174BD3ED087A144B93ED1C7AF0EE470AAB
:105DB000B0EE670A154800F03FF8144B184A19492D
:105DC000194800F07DFE0F4BD3ED087A0A4B93ED96
:105DD0001C7AF0EE470AB0EE670A0D4800F02CF886
:105DE0000B4B124A1249134800F06AFE00F0DEF82D
:105DF00000BF80BDE008002000040020B8030020A0
:105E00007405002004070020940800207C04002072
:105E1000F8040020EC080020D7B35D3FCDCC4C3F08
:105E2000B4050020AC050020A00500204407002098
:105E30003C0700203007002080B586B000AFF86036
:105E400087ED020AC7ED010A00237B61234B1B7813
:105E5000033B012B19D8FB683C33D7ED010A1846E8
:105E600097ED020A00F042F8FB68D3ED0F7A9FED40
:105E70001C7A67EE877A9FED1B7A67EE877AFCEED5
:105E8000E77A17EE903A7B6110E0FB68D3ED0D7A6C
:105E90009FED137A67EE877A9FED127A67EE877A25
:105EA000FCEEE77A17EE903A7B6100BF7B69C3F3A3
:105EB0000A030D4A9B0013441A68FB685A657B6904
:105EC00003F2FF13C3F30A03074A9B0013441A6843
:105ED000FB689A6500BF1837BD4680BDAC03002043
:105EE00000000045610B363B50B1020880B485B01C
:105EF00000AF87ED030AB860C7ED010ABB6893EDF8
:105F0000007AD7ED036AD7ED017A66EEA77ADFED66
:105F10001B6A67EEA67A77EE277ABB68C3ED007A34
:105F2000BB68D3ED007A9FED157AF4EEC77AF1EEF7
:105F300010FA0ADBBB68D3ED007A9FED107A77EE9A
:105F4000C77ABB68C3ED007A12E0BB68D3ED007A74
:105F5000F5EEC07AF1EE10FA00D409E0BB68D3ED9B
:105F6000007A9FED067A77EE877ABB68C3ED007AF8
:105F700000BF1437BD465DF8047B70470000B44392
:105F800080B500AF074B1B78012B09D100F036F824
:105F900000F060F8034B00221A700348FEF7F6FC8D
:105FA00000BF80BDAC0800200022014080B582B057
:105FB00000AF0A23FB710A4B1B8801339AB2084BCE
:105FC0001A80FB799AB2064B1B889A4204D200F0E1
:105FD00009F8034B00221A8000BF0837BD4680BD78
:105FE0001809002080B400AF034B01221A7000BFD3
:105FF000BD465DF8047B7047AC08002080B400AF5C
:10600000124B1A88124B5A80104B5A88104B9A80A8
:106010000E4B9A880E4BDA800C4BDA880C4B1A81A7
:106020000A4B1A890A4B5A81084B5A89084B9A81A4
:10603000064B9A89064BDA81044BDA89044B1A82A3
:1060400000BFBD465DF8047B704700BF540A0020C6
:10605000AC08002080B400AF3A4B5B8807EE903A62
:10606000B8EEE77A384BD3ED167A67EE277A354BE0
:10607000C3ED057A334B9B8807EE903AB8EEE77A8A
:10608000314BD3ED167A67EE277A2E4BC3ED067AA5
:106090002C4BDB8807EE903AB8EEE77A2A4BD3ED2B
:1060A000167A67EE277A274BC3ED077A254B1B89B3
:1060B00007EE903AB8EEE77A234BD3ED167A67EE07
:1060C000277A204BC3ED087A1E4B5B8907EE903A86
:1060D000B8EEE77A1C4BD3ED167A67EE277A194BA8
:1060E000C3ED097A174B9B8907EE903AB8EEE77A31
:1060F000154BD3ED167A67EE277A124BC3ED0A7A69
:10610000104BDB8907EE903AB8EEE77A0E4BD3EDF1
:10611000167A67EE277A0B4BC3ED0B7A094B1B8A75
:1061200007EE903AB8EEE77A074BD3ED167A67EEB2
:10613000277A044BC3ED0C7A00BFBD465DF8047BA3
:10614000704700BFAC0800200004002000000000E1
:106150002DE9B04300AF0121012002F05FFC0121D5
:10616000022002F05BFC0121012002F0E3FC01218E
:10617000022002F0DFFCAA4B1A7AAA4B83F87C219A
:10618000A84B93F87C315B08DAB2A64B83F87D21EB
:10619000A34BDB68A34AC2F88431A14B1B69A14A17
:1061A000C2F888319E4B5B699E4AC2F880319C4B95
:1061B0009B699C4AC2F88C31994BDB69994AC2F8B9
:1061C000BC30974B1B6A974AC2F8C030944B5B6A4D
:1061D000944AC2F8C430924B9B6A924AC2F8CC30BF
:1061E0008F4BDB6A8F4AC2F8D0308D4B1B6B8D4AC8
:1061F000C2F8D4308B4B8C4AC3F8D820884B5B6BE9
:10620000884AC2F8DC30864B9B6B864AC2F8E03085
:10621000834BDB6B834AC2F8E430814B1B6C814AB1
:10622000C2F8EC307E4B5B6C7E4AC2F8F0307D4B9E
:1062300093F87D217D4B1A73794B5A897B4B9A8059
:10624000774B9B6C794A9360754BDB6C774A136193
:10625000734B1B6D754A1360714BB3F85820734B29
:10626000A3F864206E4BB3F85A20704BA3F8662055
:106270006B4BB3F85C206D4BA3F86020684BB3F810
:106280005E206A4BA3F86220654BB3F86020674B31
:10629000A3F86820624BB3F86220644BA3F86A202D
:1062A0005F4B5B6E614AD3665D4B9B6E5F4A1367C3
:1062B0005C4B93F87C215E4B83F87C215C4B93F81C
:1062C0007C315B08DAB25A4B83F87D21554BD3F809
:1062D0008431574AC2F88431524BD3F88831544A3A
:1062E000C2F888314F4BD3F88031514AC2F880311F
:1062F0004C4BD3F88C314E4AC2F88C31494BD3F811
:10630000BC304B4AC2F8BC30464BD3F8C030484A88
:10631000C2F8C030464B93ED2F7AF7EE006AC6EE16
:10632000877A434BC3ED317A3E4BD3F8CC30404AA9
:10633000C2F8CC303B4BD3F8D0303D4AC2F8D03015
:106340003B4B93ED337AF7EE006AC6EE877A384B13
:10635000C3ED357A334BD3F8DC30354AC2F8DC3044
:10636000304BD3F8E030324AC2F8E030304B93ED96
:10637000377AF7EE006AC6EE877A2D4BC3ED397A8D
:10638000284BD3F8EC302A4AC2F8EC30254BD3F82E
:10639000F030274AC2F8F030254B93F87D21254B89
:1063A0001A73224B9A88234B9A80204B9B68214A70
:1063B00093601E4B1B691F4A1361194B5B6D1D4A8D
:1063C00013601A4BB3F864201A4BA3F86420174BE0
:1063D000B3F86620174BA3F86620144BB3F860207F
:1063E000144BA3F86020114BB3F86220114BA3F8B3
:1063F00062200E4BB3F868200E4BA3F868200B4BBD
:10640000B3F86A200B4BA3F86A20084BDB6E094AED
:10641000D366064B1B6F074A1367014BDB6E0BE01D
:10642000980A0020740500206F12033C7C040020B1
:1064300004070020F8040020954A9365954B1B6FD4
:10644000934AD365934B5B6F914A1366904BD3EDA0
:10645000166A8F4B93ED177AC6EE877A8C4BC3ED95
:10646000197A8B4BD3ED167AF1EE676A884B93ED70
:10647000187AC6EE877A864BC3ED1A7A854B9B6FE6
:10648000834A1367834BDB6F814A9367814BD3F851
:1064900080307F4A53677F4BD3F884307C4AD36681
:1064A0007C4BD3F888307C4A13607A4BD3F88C301D
:1064B000794A5360784B5B681846F9F775FF0446D4
:1064C0000D46754B1B681846F9F76EFF6EA3D3E9AE
:1064D0000023F9F7C1FF02460B46904699466E4BE2
:1064E0005B681846F9F760FF02460B46404649468E
:1064F000F9F7FCFD02460B4620462946FAF7D6F886
:1065000002460B4610461946FAF740FA0346624A1D
:106510009360604BD3F89030604A13605D4BD3F8C2
:1065200094305E4A53605D4B5B681846F9F73CFF58
:1065300004460D46594B1B681846F9F735FF52A320
:10654000D3E90023F9F788FF02460B4690469946A7
:10655000524B5B681846F9F727FF02460B46404648
:106560004946F9F7C3FD02460B4620462946FAF78D
:106570009DF802460B4610461946FAF707FA0346FD
:10658000464A9360434BD3F89830454A1360414BD9
:10659000D3F89C30424A5360414B5B681846F9F788
:1065A00003FF04460D463E4B1B681846F9F7FCFEF8
:1065B00035A3D3E90023F9F74FFF02460B46904677
:1065C0009946374B5B681846F9F7EEFE02460B46D4
:1065D00040464946F9F78AFD02460B4620462946C1
:1065E000FAF764F802460B4610461946FAF7CEF958
:1065F00003462B4A9360274BD3F8A030294A5361B6
:10660000244BD3F8A430274A1361224BD3F8A83087
:10661000244A93601F4BD3F8AC30224AD3601D4B01
:10662000D3F8B0301F4A13601A4BD3F8B4301D4A68
:106630005360184BD3F8B8301A4A9361154BD3F80E
:10664000BC30184AD361134BD3F8C030104AD36121
:10665000104BD3F8C4300E4A53620E4BD3F8C830F7
:10666000114A93640B4BD3F8CC300F4AD364094BD7
:10667000D3F8C8300D4A9364064BD3F8CC300B4A9C
:10668000D36400BFBDE8B083112D4454FB211940F1
:1066900000040020980A0020EC080020E0080020F8
:1066A000F8080020E00300207C040020F80400200B
:1066B00080B400AF654B4FF000021A60634B4FF09F
:1066C00000025A60614B4FF000029A605F4B4FF03E
:1066D0000002DA605D4B4FF000025A615B4B4FF0F5
:1066E00000021A61594B4FF000021A62574B4FF0EB
:1066F00000025A62554B4FF000029A62534B4FF022
:106700000002C3F8FC20514B4FF00002C3F80021F7
:106710004E4B4FF00002C3F804214C4B4FF00002E7
:10672000C3F80C21494B4FF00002C3F81021474B2E
:106730004FF00002C3F81421444B4FF00002C3F89D
:106740001821424B4FF00002C3F81C213F4B4FF081
:106750000002C3F820213D4B4FF00002C3F8242172
:106760003A4B4FF00002C3F82C21384B4FF0000297
:10677000C3F83021354B4FF00002C3F83421334BBE
:106780004FF00002C3F83821304B4FF00002DA64BA
:106790002E4B4FF000021A652C4B4FF000025A6549
:1067A0002A4B4FF000029A65284B4FF000025A66C0
:1067B000264B4FF000029A66244B4FF00002DA6637
:1067C000234BD3ED1D7AFCEEE77A17EE902A1F4B90
:1067D000C3F8B0201E4BD3ED1D7AFCEEE77A17EE1E
:1067E000902A1A4BC3F8B420194BD3ED1D7AFCEE56
:1067F000E77A17EE902A154BC3F8B820134B4FF0E9
:106800000002C3F83C21114B4FF00002C3F84021B5
:106810000E4B4FF00002C3F844210C4B4FF0000226
:10682000C3F84C21094B4FF00002C3F85021074B2D
:106830004FF00002C3F85421044B4FF00002C3F89C
:10684000582100BFBD465DF8047B704774050020E9
:106850000004002080B400AF654B4FF000021A60C6
:10686000634B4FF000025A60614B4FF000029A6098
:106870005F4B4FF00002DA605D4B4FF000025A614F
:106880005B4B4FF000021A61594B4FF000021A6245
:10689000574B4FF000025A62554B4FF000029A627C
:1068A000534B4FF00002C3F8FC20514B4FF0000255
:1068B000C3F800214E4B4FF00002C3F804214C4BAB
:1068C0004FF00002C3F80C21494B4FF00002C3F80F
:1068D0001021474B4FF00002C3F81421444B4FF0F6
:1068E0000002C3F81821424B4FF00002C3F81C21EC
:1068F0003F4B4FF00002C3F820213D4B4FF0000208
:10690000C3F824213A4B4FF00002C3F82C21384B36
:106910004FF00002C3F83021354B4FF00002C3F8AE
:106920003421334B4FF00002C3F83821304B4FF085
:106930000002DA642E4B4FF000021A652C4B4FF028
:1069400000025A652A4B4FF000029A65284B4FF01F
:1069500000025A66264B4FF000029A66244B4FF015
:106960000002DA66234BD3ED1D7AFCEEE77A17EED0
:10697000902A1F4BC3F8B0201E4BD3ED1D7AFCEEBE
:10698000E77A17EE902A1A4BC3F8B420194BD3EDCF
:106990001D7AFCEEE77A17EE902A154BC3F8B82063
:1069A000134B4FF00002C3F83C21114B4FF0000293
:1069B000C3F840210E4B4FF00002C3F844210C4BAA
:1069C0004FF00002C3F84C21094B4FF00002C3F80E
:1069D0005021074B4FF00002C3F85421044B4FF0F5
:1069E0000002C3F8582100BFBD465DF8047B704724
:1069F000040700200004002080B500AF154BDB79B0
:106A000003F00103002B1FD1002113480FF076FB88
:106A1000042111480FF072FB08210F480FF06EFBA4
:106A200000210D4810F0A4FB04210B4810F0A0FB3E
:106A30000821094810F09CFB064BDB7943F0010369
:106A4000DAB2044BDA7103E0024B0122DA7100BFC3
:106A500000BF80BDAC030020680D002080B500AFF2
:106A6000154B1B7A03F00103002B1FD100211348A3
:106A70000FF044FB042111480FF040FB08210F48A0
:106A80000FF03CFB00210D4810F072FB04210B4875
:106A900010F06EFB0821094810F06AFB064B1B7AC8
:106AA00043F00103DAB2044B1A7203E0024B0122F5
:106AB0001A7200BF00BF80BDAC030020880E00200A
:106AC00080B485B000AFF860B9607A603B60FB6865
:106AD0001A68BB681A60FB6893ED017AFB68D3ED16
:106AE000027A77EE677A9FED1B7A67EE877ABB684A
:106AF000C3ED017ABB6893ED017A3B68D3ED157A5B
:106B000027EE277ABB68D3ED006A3B68D3ED167A8F
:106B100066EEA77A77EE277A7B68C3ED007ABB68CA
:106B200093ED017A3B68D3ED167A27EE277ABB689E
:106B3000D3ED006A3B68D3ED157A66EEA77A77EE5F
:106B4000677A7B68C3ED017A00BF1437BD465DF8F4
:106B5000047B70473ACD133F80B485B000AFF86036
:106B6000B9607A603B607B68D3ED017AB1EE677AF9
:106B70003B68D3ED157A27EE277A7B68D3ED006A60
:106B80003B68D3ED167A66EEA77A77EE277ABB6874
:106B9000C3ED007A7B6893ED017A3B68D3ED167AFA
:106BA00027EE277A7B68D3ED006A3B68D3ED157A30
:106BB00066EEA77A77EE277ABB68C3ED017ABB68E9
:106BC0001A68FB681A60BB68D3ED007ABEEE007AE3
:106BD00027EE877ABB68D3ED017ADFED116A67EEA5
:106BE000A67A77EE277AFB68C3ED017ABB68D3ED0E
:106BF000007ABEEE007A27EE877ABB68D3ED017A81
:106C0000DFED076A67EEA67A77EE677AFB68C3ED79
:106C1000027A00BF1437BD465DF8047B704700BFA1
:106C2000D7B35D3F80B487B000AFF860B96087ED3F
:106C3000010AFB6893ED027AFB68D3ED007A77EEE8
:106C4000677AC7ED057AFB6893ED007AFB68D3EDB0
:106C5000017A37EE677AD7ED057A67EE277AF5EE97
:106C6000C07AF1EE10FA02DDFB681B6815E0FB68E4
:106C700093ED017AFB68D3ED027A37EE677AD7EDB0
:106C8000057A67EE277AF5EEC07AF1EE10FA02DBAC
:106C9000FB689B6801E0FB685B683B61D7ED047AA9
:106CA000B6EE007A67EE877AC7ED047AFB6893ED5B
:106CB000007AD7ED047A77EE277ABB68C3ED007AC5
:106CC000FB6893ED017AD7ED047A77EE277ABB68FB
:106CD000C3ED017AFB6893ED027AD7ED047A77EE83
:106CE000277ABB68C3ED027ABB68D3ED007A97EDD3
:106CF000017AB4EEE77AF1EE10FA02D5D7ED017A17
:106D000013E0BB6893ED007AD7ED017AF1EE677A74
:106D1000B4EEE77AF1EE10FA04D5D7ED017AF1EE90
:106D2000677A02E0BB68D3ED007ABB68C3ED007AF6
:106D3000BB68D3ED017A97ED017AB4EEE77AF1EE14
:106D400010FA02D5D7ED017A13E0BB6893ED017A12
:106D5000D7ED017AF1EE677AB4EEE77AF1EE10FA48
:106D600004D5D7ED017AF1EE677A02E0BB68D3ED86
:106D7000017ABB68C3ED017ABB68D3ED027A97ED67
:106D8000017AB4EEE77AF1EE10FA02D5D7ED017A86
:106D900013E0BB6893ED027AD7ED017AF1EE677AE2
:106DA000B4EEE77AF1EE10FA04D5D7ED017AF1EE00
:106DB000677A02E0BB68D3ED027ABB68C3ED027A62
:106DC00000BF1C37BD465DF8047B704780B487B0B8
:106DD00000AF87ED050AC7ED040AF860B96087EDDA
:106DE000011A97ED057AD7ED047A77EE677AFB689A
:106DF000C3ED007ABB6893ED007AFB68D3ED007AAF
:106E000067EE277AFB68C3ED017AFB6893ED017AA0
:106E1000BB68D3ED016AFB6893ED006AFB68D3EDB4
:106E2000065ABB68D3ED027A65EEA77A76EE677AEA
:106E300066EEA77A37EE277AFB68D3ED027A37EE53
:106E4000277AFB68D3ED057A77EE277AFB68C3EDE6
:106E5000047AFB68D3ED047A97ED017AB4EEE77A11
:106E6000F1EE10FA02D5D7ED017A13E0FB6893ED4D
:106E7000047AD7ED017AF1EE677AB4EEE77AF1EEB3
:106E800010FA04D5D7ED017AF1EE677A02E0FB68DB
:106E9000D3ED047AFB68C3ED077AFB6893ED027AC1
:106EA000BB68D3ED016AFB6893ED006AFB68D3ED24
:106EB000065ABB68D3ED027A65EEA77A76EE677A5A
:106EC00066EEA77A77EE277AFB68C3ED027AFB6855
:106ED000D3ED027A97ED017AB4EEE77AF1EE10FA8B
:106EE00002D5D7ED017A13E0FB6893ED027AD7ED76
:106EF000017AF1EE677AB4EEE77AF1EE10FA04D592
:106F0000D7ED017AF1EE677A02E0FB68D3ED027A01
:106F1000FB68C3ED027AFB68DB6907EE903AB0EEDE
:106F2000670A1C37BD465DF8047B704780B487B0A4
:106F300000AF87ED050AC7ED040AF860B96087ED78
:106F4000011A97ED057AD7ED047A77EE677AFB6838
:106F5000C3ED007ABB6893ED007AFB68D3ED007A4D
:106F600067EE277AFB68C3ED017AFB6893ED017A3F
:106F7000BB68D3ED016AFB68D3ED007A66EEA77AB1
:106F800037EE277AFB68D3ED027A77EE277AFB6833
:106F9000C3ED047AFB68D3ED047AF5EEC07AF1EE26
:106FA00010FA02DBDFED2B7A13E0FB6893ED047A35
:106FB000D7ED017AF1EE677AB4EEE77AF1EE10FAE6
:106FC00004D5D7ED017AF1EE677A02E0FB68D3EDE4
:106FD000047AFB68C3ED077AFB6893ED027ABB681D
:106FE000D3ED016AFB68D3ED007A66EEA77A77EEFF
:106FF000277AFB68C3ED027AFB68D3ED027AF5EEDF
:10700000C07AF1EE10FA02DBDFED127A13E0FB68D2
:1070100093ED027AD7ED017AF1EE677AB4EEE77A72
:10702000F1EE10FA04D5D7ED017AF1EE677A02E0BD
:10703000FB68D3ED027AFB68C3ED027AFB68DB697B
:1070400007EE903AB0EE670A1C37BD465DF8047B48
:10705000704700BF0000000080B489B000AFF86046
:10706000B9607A603B60BB6893ED007A3B68D3ED12
:10707000057A67EE277A7B68C3ED007ABB6893EDEB
:10708000017A3B68D3ED057A7B68043367EE277A93
:10709000C3ED007ABB6893ED027A3B68D3ED057AC5
:1070A0007B68083367EE277AC3ED007ABB6893EDFF
:1070B000007A3B68D3ED067A27EE277A3B68D3ED5A
:1070C0001D7AB4EEE77AF1EE10FA03DD3B68D3EDFA
:1070D0001D7A1FE0BB6893ED007A3B68D3ED067A1A
:1070E00027EE277A3B68D3ED1D7AF1EE677AB4EE8E
:1070F000E77AF1EE10FA05D53B68D3ED1D7AF1EE93
:10710000677A07E0BB6893ED007A3B68D3ED067AB7
:1071100067EE277AC7ED057ABB6893ED017A3B6885
:10712000D3ED067A27EE277A3B68D3ED1D7AB4EECD
:10713000E77AF1EE10FA03DD3B68D3ED1D7A1FE02C
:10714000BB6893ED017A3B68D3ED067A27EE277A88
:107150003B68D3ED1D7AF1EE677AB4EEE77AF1EE93
:1071600010FA05D53B68D3ED1D7AF1EE677A07E09A
:10717000BB6893ED017A3B68D3ED067A67EE277A18
:10718000C7ED067ABB6893ED027A3B68D3ED067AC9
:1071900027EE277A3B68D3ED1D7AB4EEE77AF1EE5D
:1071A00010FA03DD3B68D3ED1D7A1FE0BB6893ED59
:1071B000027A3B68D3ED067A27EE277A3B68D3ED57
:1071C0001D7AF1EE677AB4EEE77AF1EE10FA05D5A2
:1071D0003B68D3ED1D7AF1EE677A07E0BB6893ED6B
:1071E000027A3B68D3ED067A67EE277AC7ED077A15
:1071F00097ED057A3B68D3ED1D7A37EE277A3B6829
:10720000D3ED1E7AB4EEE77AF1EE10FA05DD3B68B5
:10721000D3ED1E7AFCEEE77A19E097ED057A3B682C
:10722000D3ED1D7A77EE277AB7EE007AF4EEC77ABF
:10723000F1EE10FA02D8DFED3D7A08E097ED057A1D
:107240003B68D3ED1D7A77EE277AFCEEE77AFB6890
:10725000C3ED007A97ED067A3B68D3ED1D7A37EEE1
:10726000277A3B68D3ED1E7AB4EEE77AF1EE10FA96
:1072700005DD3B68D3ED1E7AFCEEE77A19E097ED69
:10728000067A3B68D3ED1D7A77EE277AB7EE007A5F
:10729000F4EEC77AF1EE10FA02D8DFED247A08E0B6
:1072A00097ED067A3B68D3ED1D7A77EE277AFCEEF0
:1072B000E77AFB680433C3ED007A97ED077A3B6801
:1072C000D3ED1D7A37EE277A3B68D3ED1E7AB4EE04
:1072D000E77AF1EE10FA05DD3B68D3ED1E7AFCEE9D
:1072E000E77A19E097ED077A3B68D3ED1D7A77EEE0
:1072F000277AB7EE007AF4EEC77AF1EE10FA02D8E8
:10730000DFED0A7A08E097ED077A3B68D3ED1D7A46
:1073100077EE277AFCEEE77AFB680833C3ED007A54
:1073200000BF2437BD465DF8047B704701000000B4
:1073300080B483B000AF03463960FB71FB79012B49
:1073400002D0022B11D021E0144B1B683A6812685E
:107350005A63124B1B683A6852689A630F4B1B685A
:107360003A689268DA63002311E00D4B1B683A68B3
:1073700012685A630A4B1B683A6852689A63084B52
:107380001B683A689268DA63002300E0012318461C
:107390000C37BD465DF8047B704700BF680D0020C8
:1073A000880E002080B485B000AFF860B96087ED2A
:1073B000010AC7ED000ABB6893ED007AFB68D3EDC4
:1073C000007AB4EEE77AF1EE10FA1CD5BB6893EDC3
:1073D000007AD7ED017A77EE277ABB68C3ED007AA1
:1073E000BB6893ED007AFB68D3ED007AB4EEE77AE0
:1073F000F1EE10FA02DDFB681B6801E0BB681B6858
:10740000BA68136027E0BB6893ED007AFB68D3EDA0
:10741000007AB4EEE77AF1EE10FA00DC1BE0BB680C
:1074200093ED007AD7ED007A77EE677ABB68C3ED0B
:10743000007ABB6893ED007AFB68D3ED007AB4EE76
:10744000E77AF1EE10FA02D5FB681B6801E0BB6831
:107450001B68BA68136000BF1437BD465DF8047B33
:107460007047000080B483B000AF03463960FB7101
:10747000FB79012B40F0B780AD4B1B685B6A9BB278
:107480005B429AB23B689A823B689A693B68DB8AA6
:1074900019463B689B8ACB1A1B041B141A443B6891
:1074A0009A613B6893ED077A3B68DB8A1A463B6832
:1074B0009B8AD31A1B041B1407EE903AF8EEE77A66
:1074C00077EE277A3B68C3ED077A3B689B693A6899
:1074D0009288934207DD3B689B693A6892889A1AC2
:1074E0003B689A610AE03B689B69002B06DA3B68BF
:1074F0009B693A6892881A443B689A613B689B6929
:1075000007EE903AB8EEE77A3B68D3ED027A67EE81
:10751000277A3B68C3ED0B7A3B6893ED077A3B68AB
:10752000D3ED027A67EE277A3B68C3ED0C7A3B68AD
:107530009A8A3B68DA823B6893ED0B7A3B681B7B47
:1075400007EE903AF8EE677A67EE277A3B68C3ED6C
:107550000D7A3B6893ED0D7A3B68D3ED0D7ADFED44
:10756000756A67EEA67AFCEEE77A17EE903A9BB260
:1075700007EE903AF8EE677ADFED706A67EEA67A6A
:1075800037EE677A3B68D3ED007A77EE277A3B686F
:10759000C3ED0D7A3B68D3ED0D7A9FED687AF4EE7A
:1075A000C77AF1EE10FA0ADB3B68D3ED0D7A9FED56
:1075B000637A77EEC77A3B68C3ED0D7A11E03B68DA
:1075C000D3ED0D7AF5EEC07AF1EE10FA09D53B68ED
:1075D000D3ED0D7A9FED597A77EE877A3B68C3ED4C
:1075E0000D7A0023C1E0FB79022B40F0BD80524BA5
:1075F0001B685B6A9AB23B689A823B689A693B68EF
:10760000DB8A19463B689B8ACB1A1B041B141A445D
:107610003B689A613B6893ED077A3B68DB8A1A46C0
:107620003B689B8AD31A1B041B1407EE903AF8EEB2
:10763000E77A77EE277A3B68C3ED077A3B689B6968
:107640003A689288934207DD3B689B693A68928862
:107650009A1A3B689A610AE03B689B69002B06DA3C
:107660003B689B693A6892881A443B689A613B6818
:107670009B6907EE903AB8EEE77A3B68D3ED027A61
:1076800067EE277A3B68C3ED0B7A3B6893ED077A88
:107690003B68D3ED027A67EE277A3B68C3ED0C7A3C
:1076A0003B689A8A3B68DA823B6893ED0B7A3B68C9
:1076B0001B7B07EE903AF8EE677A67EE277A3B6815
:1076C000C3ED0D7A3B6893ED0D7A3B68D3ED0D7AEF
:1076D000DFED186A67EEA67AFCEEE77A17EE903ACD
:1076E0009BB207EE903AF8EE677ADFED146A67EE28
:1076F000A67A37EE677A3B68D3ED007A77EE277A81
:107700003B68C3ED0D7A3B68D3ED0D7A9FED0B7AA4
:10771000F4EEC77AF1EE10FA12DB3B68D3ED0D7A86
:107720009FED067A77EEC77A3B68C3ED0D7A19E0D4
:10773000B00D0020610B363BF80D00200000B44373
:107740003B68D3ED0D7AF5EEC07AF1EE10FA09D56B
:107750003B68D3ED0D7A1FED077A77EE877A3B68A9
:10776000C3ED0D7A002300E0012318460C37BD4617
:107770005DF8047B704700BF80B584B000AF03465E
:107780003960FB710A23FB73FB79012B40F08C807D
:107790003B6893F820300133DAB23B6883F820204D
:1077A0003B6893F82030FA7B9A427BD28A4B1B6865
:1077B0005B6A9BB25B429AB23B685A843B689B8C83
:1077C0001A463B685B8CD31A1B041A143B689A62F6
:1077D0003B689B6A07EE903AB8EEE77A3B68D3EDD8
:1077E000047A67EE277A17EE900AF8F7DDFD78A3A2
:1077F000D3E90023F8F730FE02460B46104619463F
:10780000F9F7C4F802463B681A643B685A8C3B6837
:107810009A843B6893ED117A3B68D3ED107A77EE4A
:10782000677AF5EEC07AF1EE10FA12DD6B4B93ED4C
:10783000027A3B68D3ED116A3B68D3ED107A76EE9D
:10784000E77A27EE277A3B68D3ED107A77EE277A2E
:1078500013E0624BD3ED027AB1EE677A3B68D3ED69
:10786000106A3B68D3ED117A76EEE77A27EE277A35
:107870003B68D3ED107A77EE277A3B68C3ED117A37
:107880003B68D3ED117A9FED567A67EE877A3B68B5
:10789000C3ED147A3B68002283F820203B68012264
:1078A00083F8212000238EE0FB79022B40F08A80B0
:1078B0003B6893F820300133DAB23B6883F820202C
:1078C0003B6893F82030FA7B9A4279D2454B1B688B
:1078D0005B6A9AB23B685A843B689B8C1A463B6849
:1078E0005B8CD31A1B041A143B689A623B689B6A30
:1078F00007EE903AB8EEE77A3B68D3ED047A67EE8C
:10790000277A17EE900AF8F74FFD31A3D3E9002349
:10791000F8F7A2FD02460B4610461946F9F736F86D
:1079200002463B681A643B685A8C3B689A843B6801
:1079300093ED117A3B68D3ED107A77EE677AF5EE26
:10794000C07AF1EE10FA12DD244B93ED027A3B6817
:10795000D3ED116A3B68D3ED107A76EEE77A27EE25
:10796000277A3B68D3ED107A77EE277A13E01B4B2A
:10797000D3ED027AB1EE677A3B68D3ED106A3B68CB
:10798000D3ED117A76EEE77A27EE277A3B68D3EDCE
:10799000107A77EE277A3B68C3ED117A3B68D3ED16
:1079A000117A9FED0F7A67EE877A3B68C3ED147A00
:1079B0003B68002283F820203B68012283F82120C5
:1079C000002300E0012318461037BD4680BD00BFEC
:1079D000696FF085C954D53FB00D0020F80800202C
:1079E0003B77D63DF80D002080B590B000AF07F191
:1079F000340300221A605A609A6007F124030022BF
:107A00001A605A609A60DA603B1D202200211846F5
:107A100010F010FD4D4B4E4A1A604C4B4FF4803223
:107A20005A604A4B00229A60484B01221A61474B28
:107A300000221A76454B002283F82020434B002277
:107A4000DA62424B434A9A62404B0022DA603F4B73
:107A50000122DA613D4B002283F830203B4B0022AB
:107A60005A613A4808F030FC0346002B01D002F07E
:107A700040F911237B630023BB630023FB6307F101
:107A800034031946314809F027FC0346002B01D086
:107A900002F02FF900237B620123BB620023FB620B
:107AA00007F124031946294808F0C2FE0346002BBB
:107AB00001D002F01EF900237B600123BB60042388
:107AC0007B610023FB604FF480133B620023FB616A
:107AD00000237B7600233B7600233B613B1D194648
:107AE0001A4809F05FFA0346002B01D002F001F9B1
:107AF00008237B600223BB603B1D1946134809F035
:107B000051FA0346002B01D002F0F3F803237B6007
:107B10000323BB603B1D19460C4809F043FA03469A
:107B2000002B01D002F0E5F80B237B600423BB603F
:107B30003B1D1946054809F035FA0346002B01D0D4
:107B400002F0D7F800BF4037BD4680BD1C090020B9
:107B5000002001400100000F80B58CB000AF07F19C
:107B6000200300221A605A609A60DA603B462022A5
:107B70000021184610F05EFC3F4B404A1A603E4B15
:107B80004FF480325A603C4B00229A603A4B0122FB
:107B90001A61394B00221A76374B002283F82020D5
:107BA000354B0022DA60344B0122DA61324B00227D
:107BB00083F83020304B00225A612F4808F084FBB4
:107BC0000346002B01D002F094F801233B6201230D
:107BD0007B620023BB6207F120031946264808F0A8
:107BE00027FE0346002B01D002F083F801233B60FF
:107BF00001237B6004233B610023BB6001237B7571
:107C000000233B750023FB603B4619461A4809F0E8
:107C1000C9F90346002B01D002F06BF809233B6041
:107C200002237B603B461946134809F0BBF9034623
:107C3000002B01D002F05DF80F233B6003237B6033
:107C40003B4619460C4809F0ADF90346002B01D01C
:107C500002F04FF80E233B6004237B603B4619463D
:107C6000054809F09FF90346002B01D002F041F8C6
:107C700000BF3037BD4680BD6409002000210140AF
:107C800080B58CB000AF07F1200300221A605A6063
:107C90009A60DA603B4620220021184610F0CAFBA9
:107CA000744B754A1A60734B4FF480325A60714BB3
:107CB00000229A606F4B01221A616E4B01221A76E4
:107CC0006C4B002283F820206A4B0022DA60694B5B
:107CD0000822DA61674B012283F83020654B0022CD
:107CE0005A61644808F0F0FA0346002B01D002F014
:107CF00000F804233B6201237B620023BB6207F18F
:107D0000200319465B4808F093FD0346002B01D081
:107D100001F0EFFF05233B6202237B6207F12003A2
:107D20001946544808F084FD0346002B01D001F0A9
:107D3000E0FF06233B6203237B6207F12003194621
:107D40004C4808F075FD0346002B01D001F0D1FF2F
:107D500007233B6204237B6207F120031946454851
:107D600008F066FD0346002B01D001F0C2FF082396
:107D70003B6205237B6207F1200319463D4808F06A
:107D800057FD0346002B01D001F0B3FF09233B62EE
:107D900006237B6207F120031946364808F048FDA8
:107DA0000346002B01D001F0A4FF0E233B62072302
:107DB0007B6207F1200319462E4808F039FD03467F
:107DC000002B01D001F095FF0F233B6208237B625B
:107DD00007F120031946274808F02AFD0346002B27
:107DE00001D001F086FF02233B6001237B60042366
:107DF0003B610023BB6001237B7500233B7500239F
:107E0000FB603B4619461B4809F0CCF80346002BA3
:107E100001D001F06EFF0A233B6002237B603B46EA
:107E20001946144809F0BEF80346002B01D001F0B2
:107E300060FF0C233B6003237B603B4619460D48E3
:107E400009F0B0F80346002B01D001F052FF0D23DA
:107E50003B6004237B603B461946064809F0A2F8C4
:107E60000346002B01D001F044FF00BF3037BD4670
:107E700080BD00BFAC0900200022014080B594B055
:107E800000AF786007F13C0300221A605A609A60E4
:107E9000DA601A617B681B68684A934264D10023E8
:107EA000BB63674B5B6C664A43F480735364644BFB
:107EB0005B6C03F48073BB63BB6B00237B63604B21
:107EC0001B6B5F4A43F0040313635D4B1B6B03F0B2
:107ED00004037B637B6B00233B63594B1B6B584A4A
:107EE00043F001031363564B1B6B03F001033B6329
:107EF0003B6B0023FB62524B1B6B514A43F0020366
:107F000013634F4B1B6B03F00203FB62FB6A0223FC
:107F1000FB6303233B6400237B6407F13C031946A6
:107F200048480AF0B9FB0923FB6303233B640023A1
:107F30007B6407F13C03194643480AF0ADFB01237B
:107F4000FB6303233B6400237B6407F13C03194676
:107F50003E480AF0A1FB00220021122009F017FB85
:107F6000122009F030FB11E17B681B68384A93420C
:107F700070D10023BB62324B5B6C314A43F4007317
:107F800053642F4B5B6C03F40073BB62BB6A00232A
:107F90007B622B4B1B6B2A4A43F001031363284B74
:107FA0001B6B03F001037B627B6A00233B62244B63
:107FB0001B6B234A43F004031363214B1B6B03F039
:107FC00004033B623B6A0023FB611D4B1B6B1C4A95
:107FD00043F0020313631A4B1B6B03F00203FB61B4
:107FE000FB690223FB6303233B6400237B6407F1EB
:107FF0003C03194614480AF04FFB3023FB6303236C
:108000003B6400237B6407F13C0319460D480AF0EA
:1080100043FB0223FB6303233B6400237B6407F1E0
:108020003C03194609480AF037FB002200211220C0
:1080300009F0ADFA122009F0C6FAA7E000200140CD
:1080400000380240000802400000024000040240E4
:10805000002101407B681B684E4A934240F09680A5
:108060000023BB614C4B5B6C4B4A43F4806353640D
:10807000494B5B6C03F48063BB61BB6900237B618C
:10808000454B1B6B444A43F020031363424B1B6B6D
:1080900003F020037B617B6900233B613E4B1B6B3C
:1080A0003D4A43F0040313633B4B1B6B03F0040393
:1080B0003B613B690023FB60374B1B6B364A43F047
:1080C00001031363344B1B6B03F00103FB60FB687C
:1080D0004FF4FF63FB6303233B6400237B6407F1DE
:1080E0003C0319462D480AF0D7FA0D23FB630323FE
:1080F0003B6400237B6407F13C03194628480AF0DF
:10810000CBFA0423FB6303233B6400237B6407F166
:108110003C03194623480AF0BFFA234B234A1A604E
:10812000214B4FF080625A601F4B00229A601E4B19
:108130000022DA601C4B4FF480621A611A4B4FF434
:1081400000625A61184B4FF400529A61164B4FF47B
:108150008072DA61144B00221A62134B00225A62B9
:10816000114809F043FB0346002B01D001F0C1FD8B
:108170007B680D4A9A630C4A7B6893630022002156
:10818000122009F004FA122009F01DFA00BF50373E
:10819000BD4680BD0022014000380240001402406C
:1081A0000008024000000240F40900201064024070
:1081B00080B582B000AF78607B681B682B4A934221
:1081C00015D12B4B5B6C2A4A23F480735364022134
:1081D00028480AF0F5FB092127480AF0F1FB0121A4
:1081E00026480AF0EDFB122009F0FBF93AE07B6823
:1081F0001B68234A934215D11D4B5B6C1C4A23F428
:108200000073536402211C480AF0DAFB302119483C
:108210000AF0D6FB022119480AF0D2FB122009F01D
:10822000E0F91FE07B681B68164A93421AD1104B95
:108230005B6C0F4A23F4806353644FF4FF61124870
:108240000AF0BEFB0D210B480AF0BAFB04210A48D4
:108250000AF0B6FB7B689B6B184609F075FB122091
:1082600009F0BFF900BF0837BD4680BD00200140BE
:1082700000380240000802400000024000040240B2
:1082800000210140002201400014024080B584B06A
:1082900000AF78607B68974A934240F02781964B05
:1082A0005B68FB600121934808F044FE03469AB2E4
:1082B000924B1A8002218F4808F03CFE03469AB286
:1082C0008E4B5A8003218B4808F034FE03469AB245
:1082D0008A4B9A800421874808F02CFE03469AB204
:1082E000864BDA800121864808F024FE03469AB2C4
:1082F000824B1A810221824808F01CFE03469AB282
:108300007E4B5A8103217E4808F014FE03469AB240
:108310007A4B9A8104217A4808F00CFE03469AB2FF
:10832000764BDA810121774808F004FE03469AB2C1
:10833000724B1A820221734808F0FCFD03469AB280
:108340006E4B5A8203216F4808F0F4FD03469AB23F
:108350006A4B9A8204216B4808F0ECFD03469AB2FE
:10836000664BDA8268490120FFF77CF803461A461B
:10837000664BDA7366490220FFF774F803461A4623
:10838000624B83F82120634B1B78002B02D0FAF755
:10839000B5FF01E0FAF730FE5F4B1B78032B06D0E8
:1083A000032B73DC012B43D0022B03D06EE0F9F7D3
:1083B00003F970E0594B1B68002B02D0FBF7CCFF90
:1083C00028E0564B1B68002B24D1554B4FF0000280
:1083D0005A60534B5B68534A5360514B4FF0000255
:1083E0001A604F4B1B684F4A13604F4B00221A70A4
:1083F0004E4B00221A704C4B00225A704C4807F02A
:10840000D9FC4C4B01221A70434B03221A70474B84
:1084100003221A70484B1B68002B39D1454B1B783F
:10842000092B35D102220A21232000F0BFFF2FE0C3
:10843000424B1B78012B0DD13B4B9B78012B09D173
:10844000394B1B78012B05D93D4B1B78002B01D1F3
:10845000FBF70AFB3B4B1B68002B09D103220E21C3
:10846000092000F0A3FF374B1B680133354A136026
:10847000354B1B68002B0DD1344B1B78092B09D1D0
:1084800001220321282000F091FF03E000BF02E059
:1084900000BF00E000BFFCF789FA174B5A68FB6881
:1084A000D31ABB602A4ABB681360294B5B68BA6861
:1084B0009A4202D9264ABB685360254BDB68002BE1
:1084C00003D1234ABB6893600BE0214B9B6819469C
:1084D000BB681F4A92689B1A1B110B441A461C4B1F
:1084E0009A601B4BDB680133194AD36000BF103719
:1084F000BD4680BD1C090020001000E0640A002079
:1085000064090020AC0900207C040020B80300208E
:10851000F8040020720300201800002094030020BB
:108520000407002074050020AC030020040C002088
:1085300030A50208E000002090030020120C00206B
:10854000050C00208403002088030020B8000020D0
:108550003003002080B483B000AF786000BF0C37D8
:10856000BD465DF8047B704780B483B000AF0F4B0D
:108570001B8907EE903AB8EEE77A0D4BD3ED007AFF
:1085800077EE677A9FED0B7A37EEC77ADFED0A6AEE
:10859000C7EE267AC7ED017A7B6807EE903AB0EE17
:1085A000670A0C37BD465DF8047B7047540A00200B
:1085B0007C0A002000E0FF44A48BC64180B483B055
:1085C00000AF0F4B5B8907EE903AB8EEE77A0D4BA0
:1085D000D3ED007A77EE677A9FED0B7A37EEC77AA4
:1085E000DFED0A6AC7EE267AC7ED017A7B6807EEEF
:1085F000903AB0EE670A0C37BD465DF8047B7047D1
:10860000540A0020800A002000E0FF44A48BC641E9
:1086100080B582B000AF3B4600221A605A60144B0E
:10862000144A1A60124809F000F80346002B01D0E2
:1086300001F05FFB00233B6000237B603B46002290
:1086400019460B4809F082F80346002B01D001F0CF
:1086500050FB3B4610221946054809F077F80346BF
:10866000002B01D001F045FB00BF0837BD4680BD9F
:10867000840A00200074004080B58AB000AF7860A2
:1086800007F1140300221A605A609A60DA601A61D6
:108690007B681B68174A934227D100233B61164B26
:1086A0001B6C154A43F000531364134B1B6C03F00F
:1086B00000533B613B690023FB600F4B1B6B0E4A71
:1086C00043F0010313630C4B1B6B03F00103FB60CE
:1086D000FB6830237B610323BB610023FB6107F14F
:1086E00014031946054809F0D7FF00BF2837BD46D7
:1086F00080BD00BF0074004000380240000002400E
:1087000080B582B000AF78607B681B68084A9342EE
:1087100009D1084B1B6C074A23F000531364302126
:1087200005480AF04DF900BF0837BD4680BD00BFBF
:1087300000740040003802400000024080B582B062
:1087400000AF00237B600C4B1B6B0B4A43F4800390
:108750001363094B1B6B03F480037B607B6800226F
:108760000021382008F013FF382008F02CFF00BF4C
:108770000837BD4680BD00BF0038024080B584B0D8
:1087800000AF2D4BBB602D4A2C4B9A4219D12C4B7C
:108790007B600023FB730AE07A68131D7B60BB6873
:1087A000191DB96012681A60FB7B0133FB73FB7BF8
:1087B0003F2BF1D9032000F071F8032000F06EF890
:1087C00036E01E4A1D4B9A4219D11E4B7B60002396
:1087D000FB730AE07A68131D7B60BB68191DB960E2
:1087E00012681A60FB7B0133FB73FB7B3F2BF1D9D3
:1087F000022000F053F8022000F050F818E0124B6D
:108800007B600023FB730AE07A68131D7B60BB6802
:10881000191DB96012681A60FB7B0133FB73FB7B87
:108820003F2BF1D9022000F039F8022000F036F891
:1088300000BF1037BD4680BD980A0020785634121C
:108840000080000800C0000850D1020880B588B040
:1088500000AF78600023FB6109F08AFC0023BB6055
:108860007B683B6101237B610223BB6107F11C0232
:1088700007F108031146184609F0ECFD0346002BEA
:1088800001D0012305E009F095FC092007F0D8FC90
:10889000002318462037BD4680BD00002DE9B043B7
:1088A00086B000AF0346FB714023BB60584B3B6171
:1088B000FB79022B51D1574BFB600023FB750CE079
:1088C0003B691A1D3A611A68FB68191DF9601B683B
:1088D0009A4207D1FB7D0133FB75FB7DBA689A4252
:1088E000EED800E000BFFB7DBA689A4201D10023B8
:1088F00089E0474B3B61474BFB6009F039FC0220A4
:10890000FFF7A4FF09F056FC092007F099FC09F0D5
:108910002FFC0023FB7517E0FB681A1DFA6019464F
:108920003B691A1D3A611B680022984691464246EF
:108930004B46022009F0C8FB0346002B01D001235F
:1089400061E0FB7D0133FB75FB7DBA689A42E3D899
:10895000092007F075FC09F02DFCFB79032B51D1A0
:108960002D4BFB600023FB750CE03B691A1D3A613F
:108970001A68FB68191DF9601B689A4207D1FB7DD4
:108980000133FB75FB7DBA689A42EED800E000BF68
:10899000FB7DBA689A4201D1002334E01C4B3B6155
:1089A0001D4BFB6009F0E4FB0320FFF74FFF09F0CC
:1089B00001FC092007F044FC09F0DAFB0023FB75F9
:1089C00017E0FB681A1DFA6019463B691A1D3A61E7
:1089D0001B6800221C46154622462B46022009F041
:1089E00073FB0346002B01D001230CE0FB7D013318
:1089F000FB75FB7DBA689A42E3D8092007F020FC9A
:108A000009F0D8FB002318461837BD46BDE8B083EF
:108A1000980A00200080000800C00008B0B596B099
:108A200000AF03460A46FB711346BB712D4B07F19D
:108A300020041D460FCD0FC40FCD0FC40FCD0FC4A2
:108A400095E8030084E8030007F10C0300221A6094
:108A50005A609A60DA601A61FB79902B3ED8FB79F4
:108A6000214A52F83330002B38D097F90630B3F151
:108A7000FF3F26D097F90630062B22DCFB791A4AF5
:108A8000DB0013449B88FB6097F90630DB0058330A
:108A90003B4453F8383C3B6197F90630DB005833D0
:108AA0003B4453F8343C7B610023BB61FB790E4AA5
:108AB00052F8333007F10C021146184609F0ECFD6C
:108AC0000CE0FB79084A52F83320FB790649DB00B9
:108AD0000B449B881946104609F072FF00BF5837B7
:108AE000BD46B0BD58A5020850D2020880B582B07C
:108AF00000AF0346FB71FB79902B14D8FB790C4A2D
:108B000052F83330002B0ED0FB79094A52F833204B
:108B1000FB790749DB000B449B88194610460AF095
:108B200043F8034600E0002318460837BD4680BDE1
:108B300050D2020880B582B000AF03460A46FB71EE
:108B40001346BB71FB79902B2AD8FB79164A52F851
:108B50003330002B24D097F90630002B0DDAFB7947
:108B6000114A52F83320FB790F49DB000B449B88F4
:108B7000194610460AF049F812E0FB790A4A52F801
:108B80003300FB79084ADB001344998897F90630D3
:108B9000002B14BF01230023DBB21A460AF01CF895
:108BA00000BF0837BD4680BD50D2020880B58EB0E8
:108BB00000AF07F1240300221A605A609A60DA605D
:108BC0001A6100233B62964B1B6B954A43F01003DE
:108BD0001363934B1B6B03F010033B623B6A002350
:108BE000FB618F4B1B6B8E4A43F0040313638C4B6A
:108BF0001B6B03F00403FB61FB690023BB61884B23
:108C00001B6B874A43F020031363854B1B6B03F0F8
:108C10002003BB61BB6900237B61814B1B6B804AD6
:108C200043F0800313637E4B1B6B03F080037B6177
:108C30007B6900233B617A4B1B6B794A43F001034C
:108C40001363774B1B6B03F001033B613B6900230C
:108C5000FB60734B1B6B724A43F002031363704B50
:108C60001B6B03F00203FB60FB680023BB606C4BD3
:108C70001B6B6B4A43F008031363694B1B6B03F0D8
:108C80000803BB60BB6800237B60654B1B6B644AB9
:108C900043F040031363624B1B6B03F040037B60A4
:108CA0007B68012204215F4809F096FF002207211A
:108CB0005D4809F091FF01224FF480515A4809F0B4
:108CC0008BFF00224FF48051584809F085FF0022A5
:108CD0000221574809F080FF04237B620123BB6215
:108CE0000123FB6202233B6307F1240319464D482D
:108CF00009F0D2FC4FF400537B624FF48813BB623F
:108D00000023FB6207F1240319464A4809F0C4FC1A
:108D100007237B620123BB620023FB6200233B63CA
:108D200007F124031946404809F0B6FC4FF480537C
:108D30007B620123BB620123FB6202233B6307F1D9
:108D400024031946384809F0A7FC4FF480537B628E
:108D50000123BB620023FB6200233B6307F1240372
:108D60001946324809F098FC4FF400437B624FF4F7
:108D70008813BB620023FB6207F1240319462C48C9
:108D800009F08AFC4FF400737B620023BB6200236E
:108D9000FB6207F124031946274809F07DFC4FF4D4
:108DA000E0537B620223BB620023FB6203233B632D
:108DB0000A237B6307F1240319461F4809F06CFC62
:108DC00002237B620123BB620023FB6200233B631F
:108DD00007F124031946164809F05EFC01237B6263
:108DE0004FF48813BB620023FB6207F1240319468A
:108DF0000C4809F051FC00220021062008F0C7FBB6
:108E0000062008F0E0FB00220021282008F0BFFB2C
:108E1000282008F0D8FB00BF3837BD4680BD00BF12
:108E200000380240001002400014024000040240DA
:108E3000000C0240000802400000024080B483B0F1
:108E400000AF0346FB80FB88B3F5004F0AD10F4B00
:108E500000229A610E4B9B78012B10D00C4B012203
:108E60009A700CE0FB88012B09D10A4B00229A6111
:108E7000074B5B78012B02D0054B01225A7000BFD3
:108E80000C37BD465DF8047B704700BFF804002036
:108E9000B80000207C04002080B500AF124B134ABC
:108EA0001A60114B124A5A600F4B00229A600E4B07
:108EB0000022DA600C4B4FF480421A610A4B002208
:108EC0005A61094B00229A61074B0022DA61064B76
:108ED00000221A62044809F0CBFE0346002B01D0A1
:108EE00000F007FF00BF80BD980B00200054004039
:108EF000A086010080B58AB000AF786007F1140346
:108F000000221A605A609A60DA601A617B681B68F6
:108F1000214A93423BD100233B61204B1B6B1F4AEC
:108F200043F0020313631D4B1B6B03F002033B6111
:108F30003B69C0237B611223BB610023FB610323D8
:108F40003B6204237B6207F114031946144809F0BD
:108F5000A3FB0023FB60114B1B6C104A43F400136E
:108F600013640E4B1B6C03F40013FB60FB680022C0
:108F70000A211F2008F00BFB1F2008F024FB002211
:108F80000A21202008F003FB202008F01CFB00BF72
:108F90002837BD4680BD00BF005400400038024065
:108FA0000004024090B585B000AF04460846114663
:108FB0001A462346FB710346BB710B467B71134671
:108FC0003B71FB793B72BB797B727B79BB723B79DE
:108FD000FB7297F820303B7397F824307B7397F837
:108FE0002830BB7300F00EF807F10803072219467A
:108FF000034806F099FC00BF1437BD4690BD00BF82
:10900000A853002080B500AF054B1B78002B04D07F
:10901000034B00221A7004F01FFF00BF80BD00BF89
:10902000EC0B002090B589B004AF04460846114609
:109030001A462346FB710346BB800B467B801346D2
:10904000BB710023BB7397F90730002B71DC9E4B7B
:109050001B6801339C4A1360B7F90420B7F902304A
:109060001344DA0F13445B10BB81B7F90C30B3F52E
:10907000E16F02DB3C23FB7314E0B7F90C30002BEB
:1090800002DC0023FB730DE0B7F90C309A1E134687
:109090001B019B1A9B008D4A82FB03125212DB17A5
:1090A000D31AFB738A4B1B78FA7B9A4200F0078134
:1090B000874AFB7B1370874B00221A70854B1A7806
:1090C000854B1A7097F90730002B17D1FB7B03F003
:1090D0003F03DBB24033D8B297F8244097F8202002
:1090E000B97997F83030029397F82C30019397F8BC
:1090F000283000932346FFF755FFE0E0FB7BC3F1E8
:109100003C03DBB203F03F03DBB24033D8B297F845
:10911000304097F82C2097F8281097F824300293C5
:1091200097F820300193BB7900932346FFF73AFF6D
:10913000C5E0B7F90430B3F5E16F02DB1E23FB7322
:1091400014E0B7F90430002B02DC0023FB730DE0C0
:10915000B7F904309A1E13461B019B1A5B005B4A49
:1091600082FB03125212DB17D31AFB735A4B1B7884
:10917000FA7B9A423ED0584AFB7B1370544B002234
:109180001A7097F90730022B17D1FB7B03F03F03CE
:10919000DBB2803BD8B297F8244097F82020B97909
:1091A00097F83030029397F82C30019397F82830D5
:1091B00000932346FFF7F6FE19E0FB7BC3F11E0385
:1091C000DBB203F03F03DBB2803BD8B297F830400C
:1091D00097F82C2097F8281097F82430029397F8E6
:1091E00020300193BB7900932346FFF7DBFEBB7B66
:1091F0000133BB73B7F90230B3F5E16F02DB1E2315
:10920000FB7314E0B7F90230002B02DC0023FB7380
:109210000DE0B7F902309A1E13461B019B1A5B0042
:109220002A4A82FB03125212DB17D31AFB73294B13
:109230001B78FA7B9A4242D0264AFB7B1370244B60
:1092400000221A70BB7B002B03D04DF2F02004F0FB
:1092500063FC97F90730022B17D1FB7B03F03F0328
:10926000DBB2403BD8B297F8244097F82020B97978
:1092700097F83030029397F82C30019397F8283004
:1092800000932346FFF78EFE19E0FB7BC3F11E031C
:10929000DBB203F03F03DBB2403BD8B297F830407B
:1092A00097F82C2097F8281097F82430029397F815
:1092B00020300193BB7900932346FFF773FE00BF74
:1092C0001437BD4690BD00BFF00B002093B6DB48BD
:1092D000FC0B0020FD0B0020FE0B002090B58BB096
:1092E00004AFF860B9607A603B603B680A2B01DC30
:1092F0000F233B6001237B6115E07B69DBB203F048
:109300003F03D8B2FB68D9B2BB68DAB27B68DBB284
:10931000FF240294FF240194FF240094FFF742FEEF
:109320007B6901337B617B693B2BE6DDFB68D9B24E
:10933000BB68DAB27B68DBB20020029000200190AB
:10934000002000903C20FFF72DFE3B6843F2BC421A
:1093500002FB03F3184604F0DFFB01233B6112E03C
:109360003B69DBB203F03F03D8B2FF230293FF2334
:109370000193FF230093032303220321FFF712FE2F
:109380003B6901333B613B693B2BE9DD00230293E1
:1093900000230193002300930323032203213C2095
:1093A000FFF700FE00BF1C37BD4690BD90B58BB0E7
:1093B00004AFF860B9607A6001237B6115E07B69D6
:1093C000DBB203F03F03D8B2FB68D9B2BB68DAB2B4
:1093D0007B68DBB2FF240294FF240194FF240094F5
:1093E000FFF7E0FD7B6901337B617B693B2BE6DDA9
:1093F000FB68D9B2BB68DAB27B68DBB200200290AE
:1094000000200190002000903C20FFF7CBFD00BF22
:109410001C37BD4690BD000080B58AB004AF5D4BDF
:1094200001221A7001237B6115E07B69DBB203F036
:109430003F03D8B20023029300230193002300933B
:10944000332303220321FFF7ADFD052006F0F8FECC
:109450007B6901337B617B693C2BE6DD3C233B610F
:1094600015E03B69DBB203F03F03D8B2002302935F
:109470000023019300230093662310221021FFF79D
:1094800091FD032006F0DCFE3B69013B3B613B693B
:10949000002BE6DC0123FB6015E0FB68DBB203F088
:1094A0003F03D8B2002302930023019300230093CB
:1094B00099231D221D21FFF775FD042006F0C0FE33
:1094C000FB680133FB60FB683C2BE6DD3C23BB60A3
:1094D00015E0BB68DBB203F03F03D8B20023029370
:1094E0000023019300230093CC232A222A21FFF793
:1094F00059FD032006F0A4FEBB68013BBB60BB68BE
:10950000002BE6DC01237B6015E07B68DBB203F017
:109510003F03D8B20023029300230193002300935A
:10952000FF2337223721FFF73DFD032006F088FE99
:109530007B6801337B607B683C2BE6DD3C233B6032
:1095400015E03B68DBB203F03F03D8B2002302937F
:109550000023019300230093032303220321FFF739
:1095600021FD032006F06CFE3B68013B3B603B683D
:10957000002BE6DC074B00221A70074B1B780133E7
:10958000DAB2054B1A70054B01221A7000BF18376A
:10959000BD4680BDF40B0020F50B0020110C00200F
:1095A000B0B588B006AF604B1B78002B00F0B680DA
:1095B0005E4B93F90330002B0FDD1423322232214E
:1095C0000520FFF78BFE594B93F90330DBB2013BCB
:1095D000DBB25AB2554BDA7073E0544B93F9033057
:1095E000002B0FDA1423052214215020FFF776FEFA
:1095F0004E4B93F90330DBB20133DBB25AB24B4B23
:10960000DA705EE04A4BD3ED0B7AB7EE007AF4EEF7
:10961000C77AF1EE10FA1CDB464B00221A60464B6B
:10962000B3F91610444BB3F91400404B1C783F4B70
:109630005B783E4A9278032504950325039503251C
:10964000029501920093234602460320FFF7EAFCAD
:1096500037E0374BD3ED0B7A9FED387AF4EEC77ACB
:10966000F1EE10FA2DD8334B1B68002B29D10123C2
:109670007B6012E07B68DBB203F03F03D8B2FF23CC
:109680000293FF230193FF2300930323032203216B
:10969000FFF788FC7B6801337B607B683B2BE9DD4F
:1096A000002302930023019300230093032303224A
:1096B00003213C20FFF776FC1E4B1B6801331D4A3B
:1096C00013601A4B93F90430002B0EDD1E23052284
:1096D00014215020FFF702FE144B93F90430DBB243
:1096E000013BDBB25AB2114B1A71154B1B78002BA0
:1096F00016D10E4B93F90430002B12DA32231922C3
:1097000014210520FFF7EAFD084B93F90430DBB282
:109710000133DBB25AB2054B1A7102E000BF00E020
:1097200000BF0837BD46B0BDF50B00202803002060
:10973000D8010020F80B002048010020CDCCCC3D02
:10974000F40B002080B582B000AF7860124B1A682D
:10975000124B1B7819464FF47A73B3FBF1F3B2FB4B
:10976000F3F3184607F04FFF0346002B01D0012307
:109770000EE07B680F2B0AD8002279684FF0FF308B
:1097800007F005FF064A7B681360002300E0012311
:1097900018460837BD4680BD240000204000002048
:1097A0003C000020B0B586B004AF06F007FD00F025
:1097B00013FA00F083FAFFF7F9F9FEF7BFFFFEF79F
:1097C00027FFFFF769FB04F0D1FB04F005FC04F070
:1097D000BFFE04F0DBFF05F085F805F03DF905F06C
:1097E00079FF05F0ABFFFEF74BFAFEF7FDF8FEF749
:1097F000B3F904F077FF06F0AFFC05F01BF805F0B5
:1098000097FC0021A54807F04FFF1021A34807F05F
:109810004BFF0822A249A34806F0DCFEA24807F04D
:10982000B7FAA24807F0B4FA9E4807F0B1FA3C2113
:109830009F480CF063FE3C219E480CF05FFE0C211B
:109840009D480CF05BFC0C219B480DF091FC9A4B61
:109850001B681A68984B1B6822F001021A60974B2C
:109860001B681A68954B1B6822F001021A600021E0
:1098700093480CF07BFB002192480CF077FB3820DA
:1098800007F0AFFE8C4B1B681A688B4B1B6842F0CD
:1098900001021A60894B1B681A68884B1B6842F0EA
:1098A00001021A60FDF7A8F8FDF7D8F8FEF766FF89
:1098B000002302930023019300230093002300223E
:1098C00000217C20FFF76EFB6D2006F0B9FCF7F756
:1098D00025FA632006F0B4FC7B4B01221A707B4B07
:1098E0001B78002B22D1794B01221A70784806F0A0
:1098F00061FA784B1B781846764B5B781C46754BA3
:109900009B781D46734B9B881A46724B9B79194670
:10991000704BDB790293019100922B46224601465F
:109920006D4806F047FA694B00221A70F7F7DEFC23
:109930006A4804F031FA6A4804F04EFA694804F0C3
:109940006BFA694804F078FA684804F065FA4FF455
:10995000FA737B600523FB7005F002FC00F070FFDA
:1099600006F092FB06F060FC03461A46604B1A6054
:10997000604B1B68002B24D15F4B1B78012B20D13F
:109980005E4B1B78032B1CD15D4BD3ED117AB1EEEE
:10999000047AF4EEC77AF1EE10FA12D5594BD3EDF2
:1099A000117AB1EE047AF4EEC77AF1EE10FA08D526
:1099B0000220F9F7D5FC504B1B780133DAB24E4B3D
:1099C0001A70514B1B78012B16D1504B1B78002B72
:1099D00012D14F4B1B78002B0ED13C4B1B78002B28
:1099E00008D13A4B01221A704A4806F0E3F9374B86
:1099F00000221A70FFF710FD474B1B68002B22D086
:109A0000464B00221A60464B00221A603F4B002250
:109A10001A70384B01221A603B4B00221A703A4BE5
:109A200000229A70384B9A78374B5A70364B002286
:109A30001A71354B1A79344BDA70304B02221A7096
:109A4000354B00221A60374B1B680133354A1360CF
:109A5000FEF7B4FDF0EE407A334BC3ED007AFCF72D
:109A60008FFA324B1B68002B69D0304B1B68032BDD
:109A70005ED0032B63DC012B02D0022B07D05EE00B
:109A80000020F9F76DFC294B00221A6057E00120F5
:109A9000F9F766FC254B00221A6050E0840A00208A
:109AA000540A0020AC0900201C0900206409002091
:109AB000B00D0020F80D0020680D0020880E002059
:109AC000D00E0020400E0020120C0020100C0020B0
:109AD00090A50208B0000020C4A502083D150108A9
:109AE00011DF010831DF010811A50108A195010866
:109AF000080C002094030020110C00201800002006
:109B00007C040020F8040020E0000020F50B002079
:109B1000F40B0020E4A50208980300208C03002029
:109B200090030020000C00200C0C002020000020DE
:109B30000220F9F715FC264B00221A6000BF254BC6
:109B40001B687A6893FBF2F2796801FB02F29B1AB8
:109B5000002B0CD101213820FEF7ECFF0121392028
:109B6000FEF7E8FF01215720FEF7E4FFF4E6194B6A
:109B70001B687A6893FBF2F2796801FB02F29A1A89
:109B800097F90330796891FBF3F39A423FF4E4AE1E
:109B9000104B1B687A6893FBF2F2796801FB02F2C2
:109BA0009A1A97F90330796891FBF3F35B009A42B4
:109BB0007FF4D2AE00213920FEF7BCFF002138200F
:109BC000FEF7B8FF00215720FEF7B4FFC4E600BF40
:109BD00020000020080C002080B594B000AF07F1F1
:109BE0001C033422002118460EF024FC07F1080360
:109BF00000221A605A609A60DA601A6100237B6062
:109C00002C4B1B6C2B4A43F080531364294B1B6C69
:109C100003F080537B607B6800233B60264B1B680E
:109C2000254A43F440431360234B1B6803F440432D
:109C30003B603B680123FB614FF480333B620223AE
:109C40007B634FF48003BB630623FB63B4233B6455
:109C500002237B640223BB640223FB6407F11C0321
:109C600018460BF057FC0346002B01D000F041F8DA
:109C70000AF012FE0346002B01D000F03AF80F2341
:109C8000BB600223FB6000233B614FF4A0537B6168
:109C90004FF48053BB6107F10803052118460AF011
:109CA0004BFE0346002B01D000F023F800BF5037D5
:109CB000BD4680BD003802400070004080B598B0BD
:109CC00000AF3B1D5C22002118460EF0B3FB1023B1
:109CD0007B60012387F85C303B1D18460AF046FF85
:109CE0000346002B01D000F004F800BF6037BD46EA
:109CF00080BD80B400AF72B600BF00BFFDE70000BA
:109D000080B582B000AF40F60D23BB803B1D022220
:109D10001946034805F008FE00BF0837BD4680BD60
:109D2000EC53002080B584B000AF0346FB71FF23E5
:109D30003B72FF237B720223BB72FB79FB72002311
:109D40003B730023FB730BE03A7BFB7B10333B44FC
:109D500013F8083C1344DBB23B73FB7B0133FB730A
:109D6000FB7B032BF0D93B7B5B42DBB23B7307F100
:109D7000080305221946044805F0D6FDFFF7C0FF89
:109D800000BF1037BD4680BDEC53002080B584B0C5
:109D900000AF03460A46FB711346BB71FF233B72BB
:109DA000FF237B720323BB72FB79FB72BB793B738E
:109DB00000237B730023FB730BE07A7BFB7B103368
:109DC0003B4413F8083C1344DBB27B73FB7B013349
:109DD000FB73FB7B042BF0D97B7B5B42DBB27B7399
:109DE00007F1080306221946044805F09DFDFFF718
:109DF00087FF00BF1037BD4680BD00BFEC53002079
:109E000080B584B000AF03460A46FB711346BB80A1
:109E1000FF233B72FF237B720423BB72FB79FB722F
:109E2000BB881B0A9BB2DBB23B73BB88DBB27B7384
:109E30000023BB730023FB730BE0BA7BFB7B103367
:109E40003B4413F8083C1344DBB2BB73FB7B013388
:109E5000FB73FB7B052BF0D9BB7B5B42DBB2BB7397
:109E600007F1080307221946044805F05DFDFFF7D6
:109E700047FF00BF1037BD4680BD00BFEC53002038
:109E800080B586B000AF03463960FB71FF233B739A
:109E9000FF237B730623BB73FB79FB733B681B0EAD
:109EA000DBB23B743B681B0CDBB27B743B681B0A68
:109EB000DBB2BB743B68DBB2FB7400233B75002351
:109EC000FB750BE03A7DFB7D18333B4413F80C3CEB
:109ED0001344DBB23B75FB7D0133FB75FB7D072B28
:109EE000F0D93B7D5B42DBB23B7507F10C030922E5
:109EF0001946044805F018FDFFF702FF00BF1837A8
:109F0000BD4680BDEC53002080B586B000AF03464F
:109F1000FB710B46BB8013467B80FF233B73FF2303
:109F20007B730623BB73FB79FB73BB88DBB23B748B
:109F30007B88DBB27B7400233B750023FB750BE051
:109F40003A7DFB7D18333B4413F80C3C1344DBB2E1
:109F50003B75FB7D0133FB75FB7D072BF0D93B7D0A
:109F60005B42DBB23B7507F10C030922194604483A
:109F700005F0DAFCFFF7C4FE00BF1837BD4680BD10
:109F8000EC53002090B587B000AF04460846114658
:109F90001A462346FB710346BB800B467B80134663
:109FA0003B80FF233B73FF237B730823BB73FB7949
:109FB000FB73BB88DBB23B747B88DBB27B743B8872
:109FC000DBB2BB743B8DDBB2FB740023BB7500239B
:109FD000FB750BE0BA7DFB7D18333B4413F80C3C5A
:109FE0001344DBB2BB75FB7D0133FB75FB7D092B95
:109FF000F0D9BB7D5B42DBB2BB7507F10C030B22D2
:10A000001946044805F090FCFFF77AFE00BF1C37A4
:10A01000BD4690BDEC53002080B594B000AF06F073
:10A0200003F90346C04AA2FB03231B09A7F84C30DF
:10A03000BE4B9B69A7F84A30BC4BDB69A7F8483098
:10A04000BA4BD3ED157AFDEEE77A17EE903AA7F802
:10A050004630B64BD3ED167AFDEEE77A17EE903A1E
:10A06000A7F84430B24BD3ED007AFDEEE77A17EE55
:10A07000903AA7F84230AE4BD3ED017AFDEEE77A85
:10A0800017EE903AA7F84030AA4BD3ED017A9FED36
:10A09000AA7A67EE877AFDEEE77A17EE903AFB87A9
:10A0A000A64BD3ED017A9FEDA47A67EE877AFDEE99
:10A0B000E77A17EE903ABB879E4BD3ED117A9FED6E
:10A0C0009E7A67EE877AFDEEE77A17EE903A7B8705
:10A0D0009A4BD3ED117A9FED987A67EE877AFDEE71
:10A0E000E77A17EE903A3B87954BD3ED007A9FEDD8
:10A0F000957A67EE877AFDEEE77A17EE903AFB865F
:10A100008F4BD3ED017A9FED8F7A67EE877AFDEE64
:10A11000E77A17EE903ABB868B4BD3ED007A9FED32
:10A12000897A67EE877AFCEEE77A17EE903A7B86BB
:10A130007E4BD3ED037A9FED837A67EE877AFDEE4F
:10A14000E77A17EE903A3B86784BD3ED047A9FED91
:10A150007D7A67EE877AFDEEE77A17EE903AFB8517
:10A16000FF233B71FF237B712623BB714123FB71CE
:10A17000B7F84C301B0A9BB2DBB23B72B7F84C30DD
:10A18000DBB27B72B7F94A301B121BB2DBB2BB7277
:10A19000B7F84A30DBB2FB72B7F948301B121BB27A
:10A1A000DBB23B73B7F84830DBB27B73B7F94630AC
:10A1B0001B121BB2DBB2BB73B7F84630DBB2FB73CA
:10A1C000B7F944301B121BB2DBB23B74B7F8443012
:10A1D000DBB27B74B7F942301B121BB2DBB2BB742B
:10A1E000B7F84230DBB2FB74B7F940301B121BB238
:10A1F000DBB23B75B7F84030DBB27B75B7F93E3068
:10A200001B121BB2DBB2BB75FB8FDBB2FB75B7F960
:10A210003C301B121BB2DBB23B76BB8FDBB27B76D2
:10A22000B7F93A301B121BB2DBB2BB767B8FDBB2C5
:10A23000FB76B7F938301B121BB2DBB23B773B8F92
:10A24000DBB27B77B7F936301B121BB2DBB2BB77C0
:10A25000FB8EDBB2FB77B7F934301B121BB2DBB2DB
:10A2600087F82030BB8EDBB287F821307B8E1B0A4B
:10A270009BB2DBB287F822307B8EDBB287F82330CB
:10A280002A4B1B7887F82430284B5B7887F82530D9
:10A290002E4B1B7887F826302C4B5B7887F82730BD
:10A2A000B7F930301B121BB2DBB287F828303B8E77
:10A2B000DBB287F82930B7F92E301B121BB2DBB2A4
:10A2C00087F82A30FB8DDBB287F82B30002387F824
:10A2D0002C30002387F84F3010E097F82C2097F8A7
:10A2E0004F3050333B4413F84C3C1344DBB287F8F7
:10A2F0002C3097F84F30013387F84F3097F84F30B4
:10A30000272BEAD997F82C305B42DBB287F82C3048
:10A310003B1D292219460E4805F006FBFFF7F0FC0D
:10A3200000BF5037BD4680BD1F85EB51480100205E
:10A33000600300207405002000007A440407002018
:10A34000580300200000C8420004002070030020D1
:10A35000EC53002080B588B000AF644B1B6801331C
:10A36000624A136005F060FF0346614AA2FB0323C3
:10A370001B09BB83FF233B72FF237B720E23BB723F
:10A380004123FB72BB8B1B0A9BB2DBB23B73BB8BC3
:10A39000DBB27B73574B9B699BB21B0A9BB2DBB250
:10A3A000BB73544B9B69DBB2FB73524BDB699BB2B3
:10A3B0001B0A9BB2DBB23B744E4BDB69DBB27B7496
:10A3C0004D4B93ED017A4D4BD3ED0D7A67EE277A25
:10A3D0009FED4B7A67EE877AFCEEE77A17EE903ABC
:10A3E0009BB21B0A9BB2DBB2BB74434B93ED017A69
:10A3F000424BD3ED0D7A67EE277A9FED417A67EEF7
:10A40000877AFCEEE77AC7ED017A3B79DBB2FB7421
:10A410003C4B93ED017A394BD3ED0D7A67EE277AF9
:10A420009FED377A67EE877AFCEEE77A17EE903A7F
:10A430009BB21B0A9BB2DBB23B75324B93ED017AA8
:10A440002E4BD3ED0D7A67EE277A9FED2D7A67EECE
:10A45000877AFCEEE77AC7ED017A3B79DBB27B7550
:10A46000294BD3ED007A9FED267A67EE877AFCEED2
:10A47000E77A17EE903A9BB21B0A9BB2DBB2BB7530
:10A48000214BD3ED007A9FED1E7A67EE877AFCEEC2
:10A49000E77AC7ED017A3B79DBB2FB7500233B76A7
:10A4A0000023FB770DE03A7EFB7F183307F10801AC
:10A4B0000B4413F8183C1344DBB23B76FB7F0133AB
:10A4C000FB77FB7F0F2BEED93B7E5B42DBB23B760B
:10A4D00007F10803112219460C4805F025FAFFF789
:10A4E0000FFC00BF2037BD4680BD00BF1C0C002004
:10A4F0001F85EB5148010020740500201001002049
:10A500000000C8420407002000040020EC53002093
:10A5100080B500AF134805F04DFC134BD3ED007A26
:10A520000220B0EE670A05F03FFD0346184605F02D
:10A5300041FC0E4805F03EFC0B4BD3ED007A9FED3D
:10A540000C7A67EE877AFCEEE77A17EE903A9AB2C9
:10A55000084B1A80074B1B8819460520FFF750FC53
:10A5600000BF80BD0CA602080004002018A6020847
:10A570000000C842200C002080B500AF074B1B78BC
:10A58000002B03D0064803F027FC02E0054803F047
:10A5900023FC054803F030FC00BF80BD190C0020EF
:10A5A00019A0010855A301082113010880B500AFC7
:10A5B00003F05EFC03F074FC00BF80BD80B500AF0B
:10A5C0000C4B1B68002B0AD0012B11D100220A4929
:10A5D0000A4805F0A9F9074B00221A6008E000229A
:10A5E0000749064805F0A0F9024B01221A6000BF96
:10A5F00000BF80BD240C002024A60208EC530020DC
:10A600003CA6020880B500AF0220FEF747F9022001
:10A61000FEF744F900BF80BD80B584B000AF0D4B9C
:10A62000BB600D4B7B600023FB730AE07A68131D4F
:10A630007B60BB68191DB96012681A60FB7B01332F
:10A64000FB73FB7B3F2BF1D9FFF7DCFF00BF10371B
:10A65000BD4680BD980A002050D1020880B582B066
:10A6600000AFFFF7CFFF632005F0EAFD0C4805F0CF
:10A67000CFFB0023FB7109E004210A4808F0C5FA6A
:10A68000C82005F0DDFDFB790133FB71FB79042B5C
:10A69000F2D906F0B4FF00BF0837BD4680BD00BF49
:10A6A00054A602080014024080B588B004AFFFF73A
:10A6B000A9FF544805F0ACFB00230293002301934B
:10A6C000002300930023002200217C20FEF76AFC77
:10A6D00001210120FEF72EFA01210220FEF72AFABD
:10A6E0000023FB600BE04FF0FF313820FEF722FA29
:10A6F00040F22B1005F0A4FDFB680133FB60FB6802
:10A70000052BF0DD01213820FEF714FA632005F057
:10A7100097FD05F0B9FD3C4805F019FE3B4805F0F2
:10A7200016FE3B4805F013FE3748FDF741FD37485C
:10A73000FDF73EFD3648FDF73BFD364806F097FF36
:10A740003448FDF7DDFF34480BF0BCFB33480BF019
:10A75000B9FB33480BF0B6FB32480BF0B3FB324881
:10A760000BF088FE31480BF085FE2B4804F028FCE6
:10A770002A4804F025FC2A4804F0B2FC294804F0D9
:10A78000AFFC294804F074FC284804F071FC284808
:10A790000CF02AFF264805F091F800237B60254B3A
:10A7A0001B6C244A43F080531364224B1B6C03F050
:10A7B00080537B607B68012100200AF051F805F08E
:10A7C00073FD1D4B1B68DB6803F02003002B13D0C7
:10A7D0001A4805F01DFB0023BB600AE04FF0FF3173
:10A7E0003820FEF7A7F9632005F02AFDBB68013386
:10A7F000BB60BB68052BF1DD06F001FF00BF103721
:10A80000BD4680BDA0A602081C09002064090020E6
:10A81000AC090020840A0020680D0020880E00206A
:10A82000400E0020D00E0020B00D0020F80D0020BA
:10A83000A853002000380240EC530020B4A60208C0
:10A84000F0B5B7B004AF894B1B680133874A13607A
:10A85000874805F053FA0346A7F8B630B7F8B63084
:10A86000002B03D1834B00221A802CE0814B1B88E4
:10A87000B7F8B6209A4209D07E4AB7F8B6301380AE
:10A8800005F0D2FC03467C4A13601CE005F0CCFCCA
:10A89000C7F8B000784B1B68D7F8B020D31A642BE8
:10A8A00011D9B7F8B6301946714805F00FFB714B56
:10A8B00000221A80714B00221A70B7F8B630194680
:10A8C0006F4805F0A5FA6D4B1B78002B53D16848F3
:10A8D00005F014FA0346022B43F20A810021644872
:10A8E00005F0A0FA0346FF2B38D10121604805F09E
:10A8F00099FA0346FF2B31D102215D4805F092FA07
:10A900000346FF2B2AD00221594805F08BFA034653
:10A91000012B23DD0221564805F084FA0346DAB202
:10A92000564B1A70554B1B78023BDAB2554B1A70D6
:10A9300003214F4805F0CAFA4D4805F0DFF90346F8
:10A940001A464C4B1A804D4B1B7819464D4B1B78C1
:10A950001A464D4805F05CFA03F0CAB80121444894
:10A9600005F0B4FA424805F0C9F903461A46414BCE
:10A970001A8003F0BDB83E4805F0C0F903461A46F8
:10A980003E4B1B789A42C3F0B3800023C7F8C43013
:10A990001FE0D7F8C4309BB21946354805F042FA9B
:10A9A0000346DAB2374B1B781344DAB2354B1A70D0
:10A9B000D7F8C4309BB219462D4805F033FA034648
:10A9C0001946324805F024FAD7F8C4300133C7F8E5
:10A9D000C4302A4B1B781A46D7F8C4309342D8DBD0
:10A9E000284B1B78002B26D0264B1B78194628486D
:10A9F00005F00EFA274B1B680133264A136000222C
:10AA000025491B4804F090FF0021194805F00AFA77
:10AA10000346FF2B03D00121154805F057FA1448CF
:10AA200005F06CF903461A46124B1A80134B0022AC
:10AA30001A7003F05DB800210D4805F0F3F90346E4
:10AA4000DAB2164B1A70154B1B781946144805F0EC
:10AA5000DFF90021064805F0E5F90346072B00F36E
:10AA6000B781042B80F2A48103F032B8280C0020B7
:10AA7000EC530020360C0020380C00203C0C002049
:10AA8000D4A602083D0C0020F4A6020818A702086C
:10AA900020A70208300C00203CA70208340C00203C
:10AAA00050A70208413BBE2B03F2128001A252F8CC
:10AAB00023F000BFA1AF0108AFAF0108BDAF01088F
:10AAC000D1DA0108D1DA0108D1DA0108D1DA0108B6
:10AAD000D1DA0108D1DA0108D1DA0108D1DA0108A6
:10AAE000D1DA0108D1DA0108D1DA0108D1DA010896
:10AAF000D1DA0108D1DA0108D1DA0108D1DA010886
:10AB0000D1DA0108D1DA0108D1DA0108D1DA010875
:10AB1000D1DA0108D1DA0108D1DA0108D1DA010865
:10AB2000D1DA0108D1DA0108D1DA0108D1DA010855
:10AB3000D1DA0108C5AF010819B20108BDB5010895
:10AB40001DB6010861B90108E5B90108B9BD0108E0
:10AB50008FC00108A1C20108D1DA0108D1DA0108C9
:10AB6000D1DA0108D1DA0108D1DA0108D1DA010815
:10AB7000D1DA0108D1DA0108C7B4010871B50108BA
:10AB8000D1DA0108D1DA0108D1DA0108D1DA0108F5
:10AB9000D1DA0108D1DA0108D1DA0108D1DA0108E5
:10ABA000D1DA0108D1DA0108D1DA0108D1DA0108D5
:10ABB000D1DA0108E5C30108D1DA0108D1DA0108C8
:10ABC00009C40108D1DA0108D1DA0108D1DA010893
:10ABD000D1DA0108D1DA0108D1DA0108D1DA0108A5
:10ABE000D1DA0108D1DA0108D1DA0108D1DA010895
:10ABF000D1DA010847C40108D1DA0108D1DA010825
:10AC0000D1DA0108D1DA0108D1DA0108D1DA010874
:10AC1000D1DA0108D1DA0108D1DA0108D1DA010864
:10AC2000D1DA0108D1DA0108D1DA0108D1DA010854
:10AC3000D1DA0108D1DA0108D1DA0108D1DA010844
:10AC4000D1DA0108D1DA0108D1DA0108D1DA010834
:10AC5000D1DA0108D1DA0108D1DA0108D1DA010824
:10AC6000D1DA0108D1DA0108D1DA0108D1DA010814
:10AC7000D1DA0108D1DA0108D1DA0108D1DA010804
:10AC8000D1DA0108D1DA0108D1DA0108D1DA0108F4
:10AC9000D1DA0108D1DA0108D1DA0108D1DA0108E4
:10ACA000D1DA0108D1DA0108D1DA0108D1DA0108D4
:10ACB000D1DA0108D1DA0108D1DA0108D1DA0108C4
:10ACC000D1DA0108D1DA0108D1DA0108D1DA0108B4
:10ACD000D1DA0108D1DA0108D1DA0108D1DA0108A4
:10ACE000D1DA0108D1DA0108D1DA0108D1DA010894
:10ACF000D1DA0108D1DA0108D1DA0108D1DA010884
:10AD0000D1DA0108D1DA0108D1DA0108D1DA010873
:10AD1000D1DA0108D1DA0108D1DA0108D1DA010863
:10AD2000D1DA0108D1DA0108D1DA0108D1DA010853
:10AD3000D1DA0108D1DA0108D1DA0108D1DA010843
:10AD4000D1DA0108D1DA0108D1DA0108D1DA010833
:10AD5000D1DA0108D1DA0108D1DA0108D1DA010823
:10AD6000D1DA0108D1DA0108D1DA0108D1DA010813
:10AD7000D1C4010887C50108B1C60108D1C60108C0
:10AD8000D1DA010841C70108D1DA0108D1DA010896
:10AD9000D1DA0108D1DA01080FC70108D1DA0108B8
:10ADA00025C70108D1DA010833C7010871CD0108B0
:10ADB000043B032B02F28C8601A252F823F000BF61
:10ADC000E1AD010859AE010897AE010841AF010895
:10ADD000FF2B02F37D86412BBFF664AE02F078BEF6
:10ADE000A44805F015F8A44BB3F9143007EE903AD7
:10ADF000F8EEE77AC7ED237A9F4BB3F9163007EEEA
:10AE0000903AF8EEE77AC7ED227A00229B499C48F7
:10AE100004F08AFD002097ED230A05F0C5F80346EB
:10AE200000221946964804F07FFD00229549944877
:10AE300004F07AFD002097ED220A05F0B5F80346EC
:10AE4000002219468E4804F06FFD00228E498C487E
:10AE500004F06AFD02F03CBE8C4804F0D9FF0022E9
:10AE60008B49874804F060FD8A4BD3ED007A0220BD
:10AE7000B0EE670A05F098F80346002219468048AC
:10AE800004F052FD002284497D4804F04DFDFFF797
:10AE90003FFB02F01DBE784BD3ED037A77EEA77A25
:10AEA000FCEEE77A17EE903A99B2734B1B7818468E
:10AEB000714BD3ED047A77EEA77AFCEEE77A17EEC2
:10AEC000903A9BB26C4A5278009202466720FFF794
:10AED00059F8704BD3ED007A9FED707A67EE877A60
:10AEE000FCEEE77A17EE903A9AB26D4B1A806C4BF3
:10AEF0001B8819460520FEF783FF6A4B93F82A301A
:10AF000019466520FEF742FF674B1B781846664BD3
:10AF10005B781C46644B9B781D46634B9B881A46A6
:10AF2000614B9B791946604BDB790293019100924A
:10AF30002B46224601465D4804F014FF02F0C8BDCE
:10AF4000594B1B781946584B5B781A46564B9B78E1
:10AF50001846554BDB78009303460720FFF712F89D
:10AF6000514B1B781C46504B5B781D464E4B9B78D3
:10AF70001E464D4BDB781A464B4B9B8819464A4B75
:10AF80009B791846484BDB7903930290019100921C
:10AF900033462A462146464804F0E4FE02F098BDB6
:10AFA000444804F035FFFFF7E7FA02F091BD42484C
:10AFB00004F02EFFFFF7FAFA02F08ABDFFF7FEFA5F
:10AFC00002F086BD02212E4804F02CFF0346032B1D
:10AFD00006DC04212A4804F025FF0346032B06DD86
:10AFE00000223649264804F09FFC02F071BD012181
:10AFF000234804F017FF03461846F5F7C3F94FF04E
:10B0000000022F4BF5F728FA02460B461046194668
:10B010004FF000022B4BF5F7A5FC0346002B19D18E
:10B020000121174804F0FEFE03461846F5F7AAF979
:10B030004FF00002224BF5F70FFA02460B4610467E
:10B0400019464FF000024FF00003F5F777FC034676
:10B05000002B3DD01C4802F05FFD32230A220A215A
:10B060009620FEF73BF900221849054804F05CFCE5
:10B0700002F02EBD64A702084801002078A702084C
:10B08000EC53002088A702088CA7020894A70208A6
:10B090000CA602080004002018A602080000C842FE
:10B0A000200C0020D8010020B0000020A8A7020832
:10B0B000CCA70208F4A7020808A802081CA80208E6
:10B0C0000000E03F00004E400417030038A80208CB
:10B0D0000121AD4804F0A6FE03461846F5F752F9E3
:10B0E0004FF00002A94BF5F7B7F902460B461046A0
:10B0F0001946F5F74BFC0346A54A53600321A248C5
:10B1000004F090FE03461846F5F73CF94FF00002B4
:10B110009E4BF5F7A1F902460B46104619464FF033
:10B1200000029C4BF5F71EFC0346002B19D10321AE
:10B13000954804F077FE03461846F5F723F94FF0DB
:10B140000002924BF5F788F902460B461046194665
:10B150004FF000024FF00003F5F7F0FB0346002B21
:10B160000FD08D4802F0D8FC32230A220A21962003
:10B17000FEF7B4F800228949834804F0D5FB02F0B9
:10B18000A7BC0321804804F04DFE03461846F5F79E
:10B19000F9F84FF000027D4BF5F75EF902460B46D9
:10B1A00010461946F5F7F2FB0346794A936002F020
:10B1B0006BFE7B4802F000FE0221734804F032FE71
:10B1C0000346DAB2724B1A7004216F4804F02AFE6B
:10B1D0000346DAB26E4B5A706D4BD3ED037A77EEBD
:10B1E000A77AFCEEE77A17EE903A99B2684B1B7893
:10B1F0001846674BD3ED047A77EEA77AFCEEE77A30
:10B2000017EE903A9BB2624A527800920246612051
:10B21000FEF7B8FE02F05CBC624804F0F9FD0022C3
:10B220006149594804F080FB604BD3ED0B7AF5EE91
:10B23000C07AF1EE10FA07DC5C4BD3ED0C7AF5EE38
:10B24000C07AF1EE10FA09DD002259494E4804F0A7
:10B250006BFB00216220FEF799FD32E101214A4893
:10B2600004F0E0FD0346022B00F0AC80022B02F359
:10B270001E84002B03D0012B43D002F018BC022106
:10B28000414804F0CFFD0346DBB219460020F8F731
:10B29000B3F8002247493C4804F046FB3C4BB3F965
:10B2A000303007EE903AF8EEE77A0020B0EE670A09
:10B2B00004F07AFE034600221946334804F034FBBA
:10B2C00000223D49304804F02FFB314BB3F93430B4
:10B2D00007EE903AF8EEE77A0020B0EE670A04F045
:10B2E00063FE034600221946274804F01DFB002296
:10B2F0003249254804F018FB01216220FEF746FD83
:10B30000DFE00221204804F08DFD0346DBB2194640
:10B310000120F8F771F8002229491B4804F004FBCA
:10B320001B4BB3F9323007EE903AF8EEE77A002083
:10B33000B0EE670A04F038FE0346002219461248B0
:10B3400004F0F2FA00221C490F4804F0EDFA104B09
:10B35000B3F9363007EE903AF8EEE77A0020B0EE17
:10B36000670A04F021FE034600221946064804F04D
:10B37000DBFA00221149044804F0D6FA01216220C8
:10B38000FEF704FD9DE000BFEC5300200000E03F0D
:10B390004801002000004E40041703004CA802089A
:10B3A000B9DE010860A8020870A80208D8010020D0
:10B3B00074A802088CA80208A4A80208A8A8020879
:10B3C000B0A802080221884804F02CFD0346DBB235
:10B3D00019460020F8F710F80221834804F022FDF6
:10B3E0000346DBB219460120F8F706F800227F4930
:10B3F0007D4804F099FA7E4BB3F9303007EE903A6D
:10B40000F8EEE77A0020B0EE670A04F0CDFD0346BF
:10B4100000221946744804F087FA002275497248E0
:10B4200004F082FA724BB3F9343007EE903AF8EE3A
:10B43000E77A0020B0EE670A04F0B6FD034600226A
:10B440001946694804F070FA00226B49664804F016
:10B450006BFA00226949644804F066FA644BB3F958
:10B46000323007EE903AF8EEE77A0020B0EE670A45
:10B4700004F09AFD0346002219465B4804F054FA92
:10B4800000225C49584804F04FFA594BB3F9363062
:10B4900007EE903AF8EEE77A0020B0EE670A04F083
:10B4A00083FD0346002219464F4804F03DFA00226E
:10B4B00051494D4804F038FA01216220FEF766FC3C
:10B4C00000BF02F0F4BA4E4804F0A2FC00224D493D
:10B4D000454804F029FA4C4BD3ED0B7AF5EEC07ACF
:10B4E000F1EE10FA07DC484BD3ED0C7AF5EEC07A9A
:10B4F000F1EE10FA09DD002244493B4804F014FA49
:10B500003B4B012283F84A202CE00321364804F00B
:10B5100089FC03469BB21C020421334804F082FCE0
:10B520000346234307EE903AF8EEE77A9FED387A28
:10B5300067EE877AFCEEE77A17EE903AA7F8983034
:10B540000121294804F06EFC0346DCB202212648A2
:10B5500004F068FC0346DBB2B7F898201946204691
:10B56000F8F708F801217220FEF710FC02F0B0BADB
:10B57000254B93F82A30002B1AD1234B93F82B300C
:10B58000002B15D10121184804F04CFC0346022B76
:10B5900006D1F5F7C5FC00217320FEF7F7FB04E0A8
:10B5A00001217320FEF7F2FB00BF00BF02F090BA4A
:10B5B00001217320FEF7EAFB02F08ABA154804F075
:10B5C00027FC0121084804F02DFC0346DBB2013BB7
:10B5D000DBB21846F7F7C4FE00220F49024804F018
:10B5E000A3F902F075BA00BFEC5300208CA8020842
:10B5F00048010020A4A80208A8A80208B0A80208D0
:10B60000C8A8020870A80208D8010020E0A8020813
:10B61000CDCC4C3D00A9020818A90208BA4804F094
:10B62000F7FBBA4B5B68C7F89430B94B5B68C7F857
:10B6300090300022B749B84804F076F9B74802F0D4
:10B640006BFA0022B649B44804F06EF9D7F89400BA
:10B65000F4F7AAFEA0A3D3E90023F4F7FDFE024607
:10B660000B4610461946F5F791F90346A74A536071
:10B67000D7F89000F4F798FE97A3D3E90023F4F7E6
:10B68000EBFE02460B4610461946F5F77FF90346D6
:10B690009F4A5360A14802F03FFA0022A1499E4808
:10B6A00004F042F9D7F89400F4F77EFE8CA3D3E9B6
:10B6B0000023F4F7D1FE02460B4610461946F5F773
:10B6C00065F90346914A5360D7F89000F4F76CFE91
:10B6D00083A3D3E90023F4F7BFFE02460B461046CE
:10B6E0001946F5F753F90346894A53608E4802F02C
:10B6F00013FA00228D49884804F016F9D7F894000F
:10B70000F4F752FE78A3D3E90023F4F7A5FE02462E
:10B710000B4610461946F5F739F903467B4A536044
:10B72000D7F89000F4F740FE6FA3D3E90023F4F7B5
:10B7300093FE02460B4610461946F5F727F90346D5
:10B74000734A53607A4802F0E7F900227949724857
:10B7500004F0EAF8D7F89400F4F726FE64A3D3E9DE
:10B760000023F4F779FE02460B4610461946F5F71A
:10B770000DF90346654A5360D7F89000F4F714FEBC
:10B780005BA3D3E90023F4F767FE02460B4610469D
:10B790001946F5F7FBF803465D4A5360644802F02A
:10B7A000BBF9002264495C4804F0BEF8D7ED257A65
:10B7B000B6EE007A67EE877A544BC3ED017AD7ED87
:10B7C000247AB6EE007A67EE877A514BC3ED017AA0
:10B7D0005A4802F0A1F9002259494F4804F0A4F850
:10B7E000D7F89400F4F7E0FD43A3D3E90023F4F77E
:10B7F00033FE02460B4610461946F5F7C7F80346D6
:10B80000424A5360D7F89000F4F7CEFD3AA3D3E94B
:10B810000023F4F721FE02460B4610461946F5F7C1
:10B82000B5F803463A4A5360464802F075F90022DB
:10B830004549394804F078F8D7F89400F4F7B4FD96
:10B840002FA3D3E90023F4F707FE02460B46104668
:10B850001946F5F79BF803462C4A5360D7F8900039
:10B86000F4F7A2FD26A3D3E90023F4F7F5FD024681
:10B870000B4610461946F5F789F80346244A5360EB
:10B88000304802F049F900223049234804F04CF8CE
:10B8900000222F49204804F047F81C4B4FF00002CB
:10B8A0005A601B4B4FF000025A602A4B4FF00002C7
:10B8B000DA60284B4FF000021A61274B00221A7001
:10B8C000264B1B680133254A13606420FEF72AFAD1
:10B8D00002F0FEB8AFF30080CDCCCCCCCCCCEC3FAA
:10B8E0009A9999999999E93F666666666666E63F10
:10B8F000333333333333E33F333333333333D33FB0
:10B900009A9999999999B93F30A90208740500202C
:10B910000407002040A90208EC530020E03229006F
:10B9200058A9020870A9020828E61E0088A9020882
:10B9300070991400A0A90208B8A90208B84C0A001E
:10B94000D0A902085C260500E8A9020800AA02089E
:10B9500010AA020848010020040C00202C0C002032
:10B960000121AD4804F05EFA0346002B1DD0012BE7
:10B9700042F09F80A94B93F82A30012B0CD1A74BA2
:10B9800093F82A3019466520FEF700FA0022A449F0
:10B99000A14803F0C9FF23E0A04B012283F82A202D
:10B9A0009E4B012283F82B201AE09C4B93F82A30FF
:10B9B000002B0CD1994B93F82A3019466520FEF7DD
:10B9C000E5F900229749944803F0AEFF07E0934B56
:10B9D000002283F82A20914B002283F82B2000BFFD
:10B9E00002F067B8052328220A211E20FDF776FC05
:10B9F0000121894804F016FA0346022B00F0018168
:10BA0000022B02F35880002B03D0012B7DD002F0D3
:10BA100052B80221804804F005FA0346012B02D0F7
:10BA2000022B34D0C6E1804BD3ED017AB6EE007A1A
:10BA300077EE877A7C4BC3ED017A7B4B93ED017AED
:10BA40007A4BD3ED056A794BD3ED0D7A66EEA77A82
:10BA5000B4EEE77AF1EE10FA13DB754802F05CF809
:10BA600032230A220A219620FDF738FC6F4B93ED12
:10BA7000057A6E4BD3ED0D7A67EE277A6A4BC3EDEC
:10BA8000017A02F001FA6B4802F096F93CE06A484C
:10BA900002F042F80A2332220A212820FDF71EFC78
:10BAA000614BD3ED017AB1EE047A77EE877A5E4B83
:10BAB000C3ED017A5C4B93ED017A5C4BD3ED056AE3
:10BAC0005A4BD3ED0D7A66EEA77AB4EEE77AF1EE33
:10BAD00010FA13DB584802F01FF832230A220A2119
:10BAE0009620FDF7FBFB514B93ED057A4F4BD3EDC1
:10BAF0000D7A67EE277A4C4BC3ED017A02F0C4F958
:10BB00004C4802F059F900BF54E10221424804F0C8
:10BB100089F90346012B02D0022B34D04AE1424B73
:10BB2000D3ED027AB6EE007A77EE877A3E4BC3ED1C
:10BB3000027A3D4B93ED027A3C4BD3ED056A3B4BC9
:10BB4000D3ED0D7A66EEA77AB4EEE77AF1EE10FA4D
:10BB500013DB374801F0E0FF32230A220A21962046
:10BB6000FDF7BCFB314B93ED057A304BD3ED0D7AED
:10BB700067EE277A2C4BC3ED027A02F085F92D4847
:10BB800002F01AF93CE02C4801F0C6FF0A233222E9
:10BB90000A212820FDF7A2FB234BD3ED027AB1EE58
:10BBA000047A77EE877A204BC3ED027A1E4B93ED31
:10BBB000027A1E4BD3ED056A1C4BD3ED0D7A66EE6F
:10BBC000A77AB4EEE77AF1EE10FA13DB1A4801F027
:10BBD000A3FF32230A220A219620FDF77FFB134B95
:10BBE00093ED057A114BD3ED0D7A67EE277A0E4B64
:10BBF000C3ED027A02F048F90E4802F0DDF800BF0A
:10BC0000D8E00221044804F00DF90346012B15D0B9
:10BC1000022B6CD0CDE000BFEC530020D8010020F7
:10BC200030AA020848AA020848010020100100209A
:10BC3000AC070100B9DE010804170300B04BD3EDD7
:10BC4000017AB6EE007A77EE877AAD4BC3ED017AD2
:10BC5000AB4BD3ED027AB6EE007A77EE877AA84B3B
:10BC6000C3ED027AA64B93ED017AA64BD3ED056A9C
:10BC7000A44BD3ED0D7A66EEA77AB4EEE77AF1EE37
:10BC800010FA0FDA9E4B93ED027A9E4BD3ED056AC4
:10BC90009C4BD3ED0D7A66EEA77AB4EEE77AF1EE1F
:10BCA00010FA1EDB984801F037FF32230A220A21DE
:10BCB0009620FDF713FB934B93ED057A914BD3ED53
:10BCC0000D7A67EE277A8E4BC3ED017A8D4B93ED9B
:10BCD000057A8C4BD3ED0D7A67EE277A884BC3ED4E
:10BCE000027A02F0D1F8894802F066F861E08648ED
:10BCF00001F012FF0A2332220A212820FDF7EEFA72
:10BD00007F4BD3ED017AB1EE047A77EE877A7C4BE4
:10BD1000C3ED017A7A4BD3ED027AB1EE047A77EE75
:10BD2000877A774BC3ED027A754B93ED017A754BA9
:10BD3000D3ED056A734BD3ED0D7A66EEA77AB4EEB8
:10BD4000E77AF1EE10FA0FDA6D4B93ED027A6D4B54
:10BD5000D3ED056A6B4BD3ED0D7A66EEA77AB4EEA0
:10BD6000E77AF1EE10FA1EDB674801F0D5FE3223C8
:10BD70000A220A219620FDF7B1FA624B93ED057A6B
:10BD8000604BD3ED0D7A67EE277A5D4BC3ED017AF8
:10BD90005C4B93ED057A5B4BD3ED0D7A67EE277A1A
:10BDA000574BC3ED027A02F06FF8584802F004F8DE
:10BDB00000BF00BF01F07FBE0A231E2232210A20ED
:10BDC000FDF78CFA0121524804F02CF80346022BAF
:10BDD00000F0D180022B01F37086002B03D0012BE1
:10BDE0005FD001F06ABE0221494804F01BF8034607
:10BDF000012B02D0022B25D047E1414BD3ED017A34
:10BE0000B6EE007A77EEC77A3D4BC3ED017A3C4B34
:10BE1000D3ED017AF5EEC07AF1EE10FA0CD83D4878
:10BE200001F07AFE32230A220A219620FDF756FA03
:10BE3000334B4FF000025A6002F026F8334801F00D
:10BE4000BBFF2DE0304801F067FE0A233C22502161
:10BE50000A20FDF743FA2A4BD3ED017AB1EE047ABA
:10BE600077EEC77A264BC3ED017A254BD3ED017AE5
:10BE7000F5EEC07AF1EE10FA0CD8234801F04CFE32
:10BE800032230A220A219620FDF728FA1C4B4FF094
:10BE900000025A6001F0F8FF1C4801F08DFF00BF5E
:10BEA000F3E002211A4803F0BDFF0346012B02D044
:10BEB000022B31D0E9E0124BD3ED017AB6EE007AD5
:10BEC00077EEC77A0E4BC3ED017A0D4BD3ED017AB5
:10BED000F5EEC07AF1EE10FA0CD80B4801F01CFE1A
:10BEE00032230A220A219620FDF7F8F9044B4FF07D
:10BEF00000029A6001F0C8FF044801F05DFF39E0DC
:10BF0000480100201001002004170300B9DE0108D9
:10BF1000EC530020AC070100A94801F0FDFD0A2305
:10BF20003C2250210A20FDF7D9F9A64BD3ED017A26
:10BF3000B1EE047A77EEC77AA24BC3ED017AA14B3A
:10BF4000D3ED017AF5EEC07AF1EE10FA0CD89C48E8
:10BF500001F0E2FD32230A220A219620FDF7BEF904
:10BF6000984B4FF000029A6001F08EFF964801F066
:10BF700023FF00BF89E00221944803F053FF0346EA
:10BF8000012B02D0022B3BD07EE08E4BD3ED017A09
:10BF9000B6EE007A77EEC77A8A4BC3ED017A894B09
:10BFA000D3ED027AB6EE007A77EEC77A854BC3ED11
:10BFB000027A844BD3ED017AF5EEC07AF1EE10FAF5
:10BFC00007D9804BD3ED027AF5EEC07AF1EE10FA84
:10BFD00010D87B4801F0A0FD32230A220A219620C6
:10BFE000FDF77CF9774B4FF000025A60754B4FF02C
:10BFF00000029A6001F048FF734801F0DDFE43E063
:10C000006F4801F089FD0A233C2250210A20FDF7E8
:10C0100065F96C4BD3ED017AB1EE047A77EEC77A0D
:10C02000684BC3ED017A674BD3ED027AB1EE047A27
:10C0300077EEC77A634BC3ED027A624BD3ED017A98
:10C04000F5EEC07AF1EE10FA07D95E4BD3ED027A25
:10C05000F5EEC07AF1EE10FA10D8594801F05CFD07
:10C0600032230A220A219620FDF738F9554B4FF06A
:10C0700000025A60534B4FF000029A6001F004FF37
:10C08000514801F099FE00BF00BF01F016BD01212B
:10C090004E4803F0C7FE0346052B09DD00224C493C
:10C0A0004A4803F041FC474B02229A7001F010BD50
:10C0B000484B1B78002B18D1424BB3F91420414B4D
:10C0C000B3F92C309A4207DC3E4BB3F916203D4BB6
:10C0D000B3F92E309A4208DD00223F493B4803F075
:10C0E00023FC384B01229A70C8E00121374803F045
:10C0F00099FE0346DAB2334B1A700121334803F03C
:10C1000091FE0346DAB22F4B5A702E4B00229A70E2
:10C110002C4B1B78022B69D0022B00F38280002B62
:10C1200002D0012B1BD07CE000222C49274803F0D1
:10C13000FBFB2B4B08221A70294B04225A70284B08
:10C1400050229A70264B1B781846254B5B7819466F
:10C15000234B9B781A461423FDF7C0F861E0204B6F
:10C1600014221A701E4B04225A701D4B50229A70D2
:10C170001B4B1B7818461A4B5B781946184B9B785B
:10C180001A461423FDF7AAF8002216490F4803F0B7
:10C19000CBFB0C4BD3ED1B7A77EEA77A0120B0EEE8
:10C1A000670A03F001FF034600221946074803F01F
:10C1B000BBFB00220C49054803F0B6FB31E000BF91
:10C1C0000417030048010020B9DE0108EC530020E9
:10C1D00060AA02087203002084AA0208A4AA020826
:10C1E00028030020B8AA0208D0AA0208A44B0A22F9
:10C1F0001A70A34B28225A70A14B28229A70A04B88
:10C200001B7818469E4B5B7819469D4B9B781A46C7
:10C210001423FDF763F800229A499B4803F084FB3E
:10C2200000BF00229949984803F07EFB984BD3ED5C
:10C23000037A0220B0EE670A03F0B6FE034600223E
:10C240001946914803F070FB002292498E4803F092
:10C250006BFB914B93F82A30012B05D100228F49BB
:10C26000894803F061FB04E000228D49864803F011
:10C270005BFB00228B49844803F056FB844B1B7800
:10C280001946834B5B781A46814B9B781846804B46
:10C290009B78009303466820FDF774FE01F018BCFC
:10C2A0000121794803F0BEFD034607EE903AF8EE0F
:10C2B000E77AB6EE007A67EE877A754BC3ED1C7AA3
:10C2C0000221714803F0AEFD034607EE903AF8EE06
:10C2D000E77AB6EE007A67EE877A6D4BC3ED1D7A8A
:10C2E0006B4B93ED1C7A6A4BD3ED037AB4EEE77A8D
:10C2F000F1EE10FA0ADC664B93ED1D7A644BD3ED38
:10C30000047AB4EEE77AF1EE10FA09DD002266490C
:10C310005D4803F009FB5E4B012283F87C2027E097
:10C320005B4B93ED1C7A5A4BD3ED1E7AB4EEE77A51
:10C33000F1EE10FA0ADC564B93ED1D7A544BD3ED17
:10C340001E7AB4EEE77AF1EE10FA09DD00225749C1
:10C350004D4803F0E9FA4E4B022283F87C2007E0B7
:10C360004B4B1B6F4A4AD366494B002283F87C2013
:10C3700000224F49444803F0D7FA454BD3ED1B7ACE
:10C3800077EEA77A0120B0EE670A03F00DFE0346B0
:10C39000002219463C4803F0C7FA002245493A48B2
:10C3A00003F0C2FA3A4BD3ED1C7A77EEA77AFCEE93
:10C3B000E77A17EE903A99B2354BD3ED1D7A77EEC6
:10C3C000A77AFCEEE77A17EE903A9AB2304B93F8E0
:10C3D0007C3018460023009303466920FDF7D2FD08
:10C3E00001F076BB0121284803F01CFD0346DAB2B8
:10C3F000294B83F82820284B93F8283019468120B0
:10C40000FDF7C4FC01F064BB00222B491E4803F079
:10C410008BFA2A4B01221A60294B1B68002B09D189
:10C420000C2214210220FCF7C1FF254B1B680133AD
:10C43000234A1360214B1B68DBB219468120FDF7AC
:10C44000A5FC01F045BB1F4B1B78002B03D0012B33
:10C450000AD001F03DBB1B4B01221A7000221A4981
:10C46000094803F061FA08E0164B00221A70002216
:10C470001649054803F058FA00BF01F029BB00BF78
:10C4800028030020D8AA0208EC530020E8AA0208DA
:10C4900048010020F4AA0208D8010020FCAA0208E2
:10C4A00000AB0208D0AA020808AB020828AB0208B9
:10C4B00044AB020854AB02085CAB020898030020AE
:10C4C0008C030020100C002084AB02089CAB0208F7
:10C4D0000022C549C54803F027FAC54B1B78052B38
:10C4E00041F2ED820121C14803F09CFC03469BB25E
:10C4F0001B029CB20221BD4803F094FC0346DBB250
:10C500002344A7F89C300321B84803F08BFC034672
:10C5100087F89B30B7F89C3097F89B201946B548B0
:10C5200003F020FCB7F89C2097F89B301344FC2BB9
:10C5300001F2C782002387F8C33018E097F8C330B0
:10C540009BB204339BB21946A84803F06BFC034628
:10C550001946B7F89C2097F8C3301344A64A1344F1
:10C56000CAB21A7097F8C330013387F8C33097F80E
:10C57000C32097F89B309A42E0D3F9F7E9FDF4F72E
:10C5800027FC01F09CBA9D4803F042FC984B1B78B5
:10C59000042B41F298820121944803F043FC0346A6
:10C5A0009BB21B029CB20221904803F03BFC034665
:10C5B000DBB22344A7F8A03003218C4803F032FCFF
:10C5C000034687F89F30B7F8A03097F89F201946A8
:10C5D000884803F01DFCB7F8A02097F89F3013445B
:10C5E000FC2B01F27282FF233B70854BFF221A70F5
:10C5F000FF237B70824B1B78013BDAB2804B1A70B1
:10C6000097F89F300233DBB2BB707D4B1A7897F8F6
:10C610009F301344DBB20233DAB2794B1A70F12344
:10C62000FB70774B1B780F3BDAB2754B1A70002307
:10C6300087F8C23020E0B7F8A02097F8C230134442
:10C640006D4A1A4497F8C23004331278C8333B4419
:10C6500003F8C82C97F8C2300433C8333B4413F8AE
:10C66000C82C674B1B781344DAB2654B1A7097F8E5
:10C67000C230013387F8C23097F8C22097F89F3054
:10C680009A42D8D35E4B1A7897F89F3004335242BF
:10C69000D2B2C8333B4403F8C82C97F89F30053317
:10C6A000DAB23B461946514803F03EF901F00BBAA5
:10C6B000544803F0ADFBFDF7A5FF002387F8A33036
:10C6C00097F8A3301946494803F0AAFA01F000BAD6
:10C6D000474B1B78022B41F2FA810121434803F0BA
:10C6E000A1FB0346002B14BF01230023DBB21A4633
:10C6F000454B1A70444B1B78002B01F0E881434BEB
:10C700001B681946F320FDF7BBFB01F0E0B9404878
:10C7100003F07EFBFDF780FFF9F71AFDF4F758FBF5
:10C7200001F0D6B93B4803F073FBFDF797FF01F02A
:10C73000CFB9394803F06CFBFDF7B6FF01F0C8B97B
:10C740002B4B1B78022B40F2FE820121274803F07D
:10C7500069FB0346013B202B00F2E48201A252F860
:10C7600023F000BF1DC8010885C8010895C801084D
:10C7700081C9010891C9010825CD010825CD01080D
:10C7800025CD010825CD010825CD010825CD0108BD
:10C7900025CD010825CD010825CD010825CD0108AD
:10C7A000D9CC0108E9CC010825CD010825CD010827
:10C7B00025CD010825CD010825CD010825CD01088D
:10C7C00025CD010825CD010825CD010825CD01087D
:10C7D00025CD010825CD010825CD010825CD01086D
:10C7E000F9CC01080FCD0108B8AB0208EC530020CA
:10C7F0003C0C0020C8AB0208980A0020E8AB0208F5
:10C800003D0C0020F8AB0208180C0020140C00208E
:10C8100010AC020824AC020838AC0208D44B012248
:10C820001A70D44B03221A70D34B03221A700121C1
:10C830000120FCF77FF901210220FCF77BF9CF4BA7
:10C840004FF07E52DA62CD4B4FF07E521A63CB4BE3
:10C85000012283F82A20C94B012283F82B20C84BE0
:10C86000C84ADA60C64BC74A1A61C54BC54A5A6006
:10C87000C34BC44A9A60FDF77FFE0121F520FDF706
:10C8800085FA73E2BA4B00221A700221F520FDF7F7
:10C890007DFA6BE2BC4B1B78062B40F26682BB4BE9
:10C8A00001221A700221BA4803F0BCFA03461B02A7
:10C8B0001CB20321B64803F0B5FA03462343A7F898
:10C8C000AA300421B24803F0ADFA03461B021CB2A1
:10C8D0000521AF4803F0A6FA03462343A7F8A83082
:10C8E000B7F9AA30A64A9361B7F9A830A44AD36130
:10C8F000B7F9AA30DA0F13445B101BB21A46A04BEB
:10C900001A62B7F9A830DA0F13445B101BB21A464B
:10C910009B4B5A629C4B1B780A2B40F226820621C5
:10C920009B4803F07FFA03461B021CB2072198487C
:10C9300003F078FA03462343A7F8A6300821944869
:10C9400003F070FA03461B021CB20921904803F061
:10C9500069FA03462343A7F8A430B7F9A63007EED7
:10C96000903AF8EEE77A864BC3ED157AB7F9A43022
:10C9700007EE903AF8EEE77A814BC3ED167AF4E1D0
:10C98000824B00221A700421F520FDF7FFF9EDE13A
:10C9900002217F4803F046FA034687F8AF300321AF
:10C9A0007B4803F03FFA03461B021CB2042178487F
:10C9B00003F038FA034623431BB2A7F8AC3097F8CC
:10C9C000AF30013B4F2B00F2828101A252F823F0DD
:10C9D00011CB010825CB010839CB010855CB010843
:10C9E000CFCC0108CFCC0108CFCC0108CFCC0108B7
:10C9F000CFCC0108CFCC0108CFCC0108CFCC0108A7
:10CA0000CFCC0108CFCC0108CFCC010899CB0108CD
:10CA1000ADCB0108C9CB0108E5CB010801CC010869
:10CA20001DCC0108CFCC0108CFCC0108CFCC010828
:10CA3000CFCC0108CFCC0108CFCC0108CFCC010866
:10CA4000CFCC0108CFCC0108CFCC010839CC0108EC
:10CA5000CFCC0108CFCC0108CFCC0108CFCC010846
:10CA6000CFCC0108CFCC0108CFCC0108CFCC010836
:10CA7000CFCC0108CFCC0108CFCC0108CFCC010826
:10CA8000CFCC0108CFCC0108CFCC01084DCC010898
:10CA900069CC010885CC0108CFCC0108CFCC0108B6
:10CAA000CFCC0108CFCC0108CFCC0108CFCC0108F6
:10CAB000CFCC0108CFCC0108CFCC0108CFCC0108E6
:10CAC000CFCC0108CFCC0108CFCC0108A1CC010804
:10CAD000CFCC0108CFCC0108CFCC0108CFCC0108C6
:10CAE000CFCC0108CFCC0108CFCC0108CFCC0108B6
:10CAF000CFCC0108CFCC0108CFCC0108CFCC0108A6
:10CB0000CFCC0108CFCC0108CFCC0108BDCC0108A7
:10CB1000B7F8AC3007EE903AF8EE677A174BC3EDF2
:10CB20001B7AD4E0B7F8AC3007EE903AF8EE677AAB
:10CB3000124BC3ED1B7ACAE0B7F8AC3007EE903A5F
:10CB4000B8EE677ADFED136AC7EE267A0B4BC3EDBA
:10CB50001C7ABCE0B7F8AC3007EE903AB8EE677AD2
:10CB6000DFED0C6AC7EE267A044BC3ED1D7AAEE00A
:10CB7000050C002018000020040C0020D801002023
:10CB800048010020000020413C0C002072030020DE
:10CB9000EC5300200000C842B7F8AC3007EE903AE2
:10CBA000F8EE677AAA4BC3ED1E7A90E0B7F8AC3086
:10CBB00007EE903AB8EE677ADFEDA66AC7EE267AFE
:10CBC000A34BC3ED1F7A82E0B7F8AC3007EE903A82
:10CBD000B8EE677ADFED9F6AC7EE267A9C4BC3ED0D
:10CBE000207A74E0B7F8AC3007EE903AB8EE677A86
:10CBF000F2EE046AC7EE267A954BC3ED217A66E021
:10CC0000B7F8AC3007EE903AB8EE677AF2EE046A05
:10CC1000C7EE267A8E4BC3ED227A58E0B7F8AC30D7
:10CC200007EE903AB8EE677AF2EE046AC7EE267A1B
:10CC3000874BC3ED237A4AE0B7F8AC3007EE903A61
:10CC4000F8EE677A824BC3ED287A40E0B7F8AC3053
:10CC500007EE903AB8EE677ADFED7E6AC7EE267A85
:10CC60007B4BC3ED247A32E0B7F8AC3007EE903A54
:10CC7000B8EE677ADFED776AC7EE267A744BC3EDBC
:10CC8000257A24E0B7F8AC3007EE903AB8EE677A30
:10CC9000DFED706AC7EE267A6D4BC3ED267A16E09B
:10CCA000B7F8AC3007EE903AB8EE677ADFED696A14
:10CCB000C7EE267A664BC3ED277A08E0B7F8AC30AA
:10CCC0004FF47A7202FB03F3634A136000BF05213D
:10CCD000F520FDF75BF849E0604B01221A70102146
:10CCE000F520FDF753F841E05C4B00221A7011214A
:10CCF000F520FDF74BF839E0594B01221A705948DD
:10CD000001F06AF82021F520FDF740F82EE0544BA1
:10CD100000221A70544801F05FF82121F520FDF738
:10CD200035F823E04D4B1B78002B0CBF012300236B
:10CD3000DBB21A46494B1A70484B1B781946F5204E
:10CD4000FDF724F812E0454B1B78002B0CBF0123A4
:10CD50000023DBB21A46414B1A70404B1B78194630
:10CD6000F520FDF713F800F0B3BE00BF00F0B0BE31
:10CD70003E4803F04DF801213D4803F053F80346C7
:10CD8000032B00F38D800121394803F04BF8034653
:10CD9000032B2FD801A252F823F000BFD1CD0108F8
:10CDA000E3CD0108ADCD0108BFCD01080022314916
:10CDB0002F4802F0B9FD304BC7F8BC301AE0002212
:10CDC0002E492B4802F0B0FD2D4BC7F8BC3011E0C6
:10CDD00000222C49264802F0A7FD2B4BC7F8BC3097
:10CDE00008E000222949224802F09EFD284BC7F89E
:10CDF000BC3000BF0023C7F8B8301DE0D7F8B8300A
:10CE000003F00F03002B04D1D7F8B810214802F02B
:10CE1000A9FFD7F8BC305A1CC7F8BC201B781946AC
:10CE20001D4802F09FFF41F65E2000F075FED7F826
:10CE3000B8300133C7F8B830D7F8B830FF2BDDD998
:10CE4000002216490A4802F06FFD00F041BE00BF03
:10CE5000D80100200000C842140000204003002038
:10CE6000190C002019A0010855A301084CAC0208B8
:10CE7000EC53002068AC0208008000087CAC02087B
:10CE800000C0000890AC020850D10208A8AC02080B
:10CE9000980A0020B8AC0208C4AC020870A80208C6
:10CEA000CF4B1B781946CE4B5B781A46CD4802F023
:10CEB00059FFCD4B1B781946CB4B5B781A46CA4BB2
:10CEC0009B78CA4802F04EFFC74B9B881946C64B59
:10CED0009B791A46C44BDB79C54802F043FFC54A2B
:10CEE000C549C64802F03EFFC54B93F87C31194650
:10CEF000C44802F037FFC24BD3ED617A0220B0EE96
:10CF0000670A03F051F803461946BF4802F02AFFAA
:10CF1000BB4BD3ED627A0220B0EE670A03F044F80F
:10CF200003461946B94802F01DFFB54BD3ED607AB0
:10CF30000220B0EE670A03F037F803461946B448FA
:10CF400002F010FFAE4BD3ED637A0320B0EE670A18
:10CF500003F02AF803461946AE4802F003FFA84B37
:10CF6000D3ED2F7A0220B0EE670A03F01DF80346D6
:10CF70001946A94802F0F6FEA14BD3ED307A022003
:10CF8000B0EE670A03F010F803461946A34802F012
:10CF9000E9FE9B4BD3ED317A0220B0EE670A03F035
:10CFA00003F8034619469E4802F0DCFE944BD3ED8D
:10CFB000337A0220B0EE670A02F0F6FF0346194604
:10CFC000984802F0CFFE8E4BD3ED347A0220B0EEBB
:10CFD000670A02F0E9FF03461946904802F0C2FED4
:10CFE000874BD3ED357A0220B0EE670A02F0DCFF02
:10CFF000034619468A4802F0B5FE814BD3ED377AD5
:10D000000220B0EE670A02F0CFFF034619468648B9
:10D0100002F0A8FE7A4BD3ED387A0220B0EE670A10
:10D0200002F0C2FF034619467C4802F09BFE744B97
:10D03000D3ED397A0220B0EE670A02F0B5FF03465D
:10D040001946774802F08EFE6D4BD3ED3B7A0220F5
:10D05000B0EE670A02F0A8FF03461946734802F0D3
:10D0600081FE674BD3ED3C7A0220B0EE670A02F0F6
:10D070009BFF03461946694802F074FE6C4B1B7B0C
:10D0800019466C4802F06EFE694B9B8819466A4847
:10D0900002F068FE664BD3ED027A0220B0EE670A1A
:10D0A00002F082FF03461946644802F05BFE604BC3
:10D0B000D3ED047A0220B0EE670A02F075FF034652
:10D0C00019465F4802F04EFE594BD3ED007A01201D
:10D0D000B0EE670A02F068FF03461946594802F0AD
:10D0E00041FE534BD3ED127A0120B0EE670A02F0F5
:10D0F0005BFF03461946544802F034FE4C4BD3ED17
:10D10000137A0120B0EE670A02F04EFF034619467B
:10D110004E4802F027FE464BB3F8643019464C489F
:10D1200002F020FE424BB3F866301946494802F03F
:10D1300019FE3F4BB3F860301946474802F012FE23
:10D140003B4BB3F862301946444802F00BFE384BB3
:10D15000B3F868301946424802F004FE344BB3F885
:10D160006A3019463F4802F0FDFD314BD3ED1B7A82
:10D170000120B0EE670A02F017FF034619463A484D
:10D1800002F0F0FD2A4BD3ED1C7A0120B0EE670AC5
:10D1900002F00AFF03461946344802F0E3FD40F26C
:10D1A0008F1003F04DF8324B93F87C31194631481B
:10D1B00002F0D8FD2E4BD3ED617A0220B0EE670A63
:10D1C00002F0F2FE034619460F4802F0CBFD284B51
:10D1D000D3ED627A0220B0EE670A02F0E5FE4BE082
:10D1E000980A0020CCAC0208B0000020E4AC020891
:10D1F000F8AC020810AD02081CAD020828AD020808
:10D200007405002044AD02085CAD020864AD02085C
:10D210006CAD020874AD020880AD020898AD02083A
:10D22000A0AD0208A8AD0208B8AD0208CCAD020856
:10D230007C040020DCAD0208F4AD0208FCAD02085D
:10D2400008AE020814AE020820AE02082CAE020896
:10D2500038AE020848AE020854AE020860AE0208BA
:10D260006CAE020878AE020884AE020890AE0208E6
:10D27000040700209CAE020803461946D64802F077
:10D2800071FDD64BD3ED607A0220B0EE670A02F052
:10D290008BFE03461946D24802F064FDCF4BD3ED16
:10D2A000637A0320B0EE670A02F07EFE0346194659
:10D2B000CC4802F057FDC94BD3ED2F7A0220B0EED7
:10D2C000670A02F071FE03461946C74802F04AFD9C
:10D2D000C24BD3ED307A0220B0EE670A02F064FE52
:10D2E00003461946C14802F03DFDBC4BD3ED317AEF
:10D2F0000220B0EE670A02F057FE03461946BC480A
:10D3000002F030FDB54BD3ED337A0220B0EE670A60
:10D3100002F04AFE03461946B64802F023FDAF4B21
:10D32000D3ED347A0220B0EE670A02F03DFE0346E8
:10D330001946AE4802F016FDA84BD3ED357A02200F
:10D34000B0EE670A02F030FE03461946A84802F024
:10D3500009FDA24BD3ED377A0220B0EE670A02F046
:10D3600023FE03461946A44802F0FCFC9B4BD3ED78
:10D37000387A0220B0EE670A02F016FE034619461C
:10D380009A4802F0EFFC954BD3ED397A0220B0EECB
:10D39000670A02F009FE03461946954802F0E2FCCE
:10D3A0008E4BD3ED3B7A0220B0EE670A02F0FCFD13
:10D3B00003461946914802F0D5FC884BD3ED3C7AE0
:10D3C0000220B0EE670A02F0EFFD034619468748D7
:10D3D00002F0C8FC8A4B1B7B19468A4802F0C2FC4B
:10D3E000874B9B881946884802F0BCFC844BD3EDE0
:10D3F000027A0220B0EE670A02F0D6FD0346194613
:10D40000824802F0AFFC7E4BD3ED047A0220B0EEEE
:10D41000670A02F0C9FD034619467D4802F0A2FCE6
:10D42000774BD3ED007A0120B0EE670A02F0BCFD25
:10D4300003461946774802F095FC714BD3ED127AFA
:10D440000120B0EE670A02F0AFFD034619467248AC
:10D4500002F088FC6A4BD3ED137A0120B0EE670A24
:10D4600002F0A2FD034619466C4802F07BFC644BB7
:10D47000B3F8643019466A4802F074FC604BB3F8A4
:10D4800066301946674802F06DFC5D4BB3F86030BA
:10D490001946654802F066FC594BB3F862301946EC
:10D4A000624802F05FFC564BB3F86830194660489A
:10D4B00002F058FC524BB3F86A3019465D4802F04E
:10D4C00051FC4F4BD3ED1B7A0120B0EE670A02F0FE
:10D4D0006BFD03461946584802F044FC484BD3ED17
:10D4E0001C7A0120B0EE670A02F05EFD0346194681
:10D4F000524802F037FC40F28F1002F0A1FE504B70
:10D50000D3ED167A0420B0EE670A02F04DFD034613
:10D5100019464C4802F026FC494BD3ED177A0420FB
:10D52000B0EE670A02F040FD03461946464802F095
:10D5300019FC434BD3ED187A0420B0EE670A02F0D1
:10D5400033FD03461946414802F00CFC3C4BD3ED39
:10D55000197A0420B0EE670A02F026FD0346194648
:10D560003B4802F0FFFB364BD3ED1A7A0420B0EEB5
:10D57000670A02F019FD03461946364802F0F2FB2D
:10D580002F4BD3ED1C7A0420B0EE670A02F00CFD9D
:10D5900003461946304802F0E5FB294BD3ED1B7AD0
:10D5A0000420B0EE670A02F0FFFC034619462B4840
:10D5B00002F0D8FB224BD3ED1E7A0220B0EE670AB0
:10D5C00002F0F2FC03461946254802F0CBFB1C4B47
:10D5D000D3ED1D7A022045E064AD02080407002067
:10D5E0006CAD020874AD020880AD020898AD020867
:10D5F000A0AD0208A8AD0208B8AD0208CCAD020883
:10D60000F8040020DCAD0208F4AD0208FCAD02080D
:10D6100008AE020814AE020820AE02082CAE0208C2
:10D6200038AE020848AE020854AE020860AE0208E6
:10D630006CAE020878AE020884AE020890AE020812
:10D6400000040020B4AE0208CCAE0208D8AE020836
:10D65000E4AE0208F0AE0208F8AE020804AF020819
:10D6600010AF0208B0EE670A02F09EFC03461946AE
:10D67000D84802F077FBD84BD3ED077A0120B0EE03
:10D68000670A02F091FC03461946D44802F06AFB8F
:10D69000D14BD3ED097A0120B0EE670A02F084FC89
:10D6A00003461946CE4802F05DFBCE4BD3ED007A1F
:10D6B0000120B0EE670A02F077FC03461946CA481B
:10D6C00002F050FBC74BD3ED017A0120B0EE670AA0
:10D6D00002F06AFC03461946C44802F043FBC44BFF
:10D6E000D3ED007A0120B0EE670A02F05DFC03463C
:10D6F0001946C04802F036FBBD4BD3ED017A01203C
:10D70000B0EE670A02F050FC03461946B74802F033
:10D7100029FBB94BD3ED007A0120B0EE670A02F085
:10D7200043FC03461946B54802F01CFBB24BD3ED4F
:10D73000017A0120B0EE670A02F036FC0346194672
:10D74000AA4802F00FFBAE4BD3ED057A0120B0EEF4
:10D75000670A02F029FC03461946AA4802F002FBB8
:10D76000A74BD3ED047A0120B0EE670A02F01CFC4F
:10D7700003461946A44802F0F5FAA14BD3ED067A08
:10D780000120B0EE670A02F00FFC034619469F48DD
:10D7900002F0E8FA9A4BD3ED077A0120B0EE670A5F
:10D7A00002F002FC03461946994802F0DBFA944B5A
:10D7B000D3ED027A0120B0EE670A02F0F5FB0346D2
:10D7C0001946944802F0CEFA8D4BD3ED037A01202E
:10D7D000B0EE670A02F0E8FB034619468E4802F0F5
:10D7E000C1FA874BD3ED007A0120B0EE670A02F050
:10D7F000DBFB03461946894802F0B4FA804BD3EDAF
:10D80000017A0120B0EE670A02F0CEFB034619460A
:10D81000834802F0A7FA834BD3ED007A0120B0EEE3
:10D82000670A02F0C1FB034619467F4802F09AFAE4
:10D830007C4BD3ED017A0120B0EE670A02F0B4FB15
:10D8400003461946794802F08DFA764BD3ED027AF9
:10D850000120B0EE670A02F0A7FB034619467448A0
:10D8600002F080FA6F4BD3ED047A0120B0EE670A24
:10D8700002F09AFB034619466E4802F073FA694BB0
:10D880009B8907EE903AF8EE677A0120B0EE670ABE
:10D8900002F08AFB03461946674802F063FA614BBF
:10D8A000D3ED0C7A0120B0EE670A02F07DFB03464F
:10D8B0001946624802F056FA5A4BD3ED067A012017
:10D8C000B0EE670A02F070FB034619465C4802F0AE
:10D8D00049FA544BD3ED077A0120B0EE670A02F003
:10D8E00063FB03461946574802F03CFA4D4BD3ED13
:10D8F000087A0120B0EE670A02F056FB034619468B
:10D90000514802F02FFA474BD3ED0A7A0120B0EECE
:10D91000670A02F049FB034619464C4802F022FA16
:10D92000404BD3ED0B7A0120B0EE670A02F03CFBCE
:10D9300003461946464802F015FA464802F012FA24
:10D94000454802F00FFA454B1C68444B1B6807EE34
:10D95000903AF8EE677ADFED426A87EEA67A012008
:10D96000B0EE470A02F020FB03461A4621463D4826
:10D9700002F0F8F9394B5C68384B5B6807EE903A77
:10D98000F8EE677ADFED366A87EEA67A0120B0EE10
:10D99000470A02F009FB03461A462146324802F0C4
:10D9A000E1F92E4B9C682D4B9B6807EE903AF8EE00
:10D9B000677ADFED2B6A87EEA67A0120B0EE470A80
:10D9C00002F0F2FA03461A462146284802F0CAF944
:10D9D0004EE000BF1CAF02080004002028AF020880
:10D9E00034AF0208EC08002040AF020858AF02082C
:10D9F000E008002060AF0208F80800206CAF0208C1
:10DA0000E003002078AF020890AF02089CAF020844
:10DA1000A8AF0208B4AF0208C4AF0208D0AF020832
:10DA2000DCAF020810010020E8AF0208FCAF0208DA
:10DA300008B0020814B0020824B0020834B002088A
:10DA400040B0020850B002085CB0020868B002089A
:10DA500078B0020888B0020890B0020830030020B5
:10DA600000003443B8B00208D8B00208F8B0020889
:10DA7000214BDB681946214802F074F91E4B5B68A4
:10DA800007EE903AB8EE677ADFED1D6AC7EE267AA8
:10DA90009FED1C7A67EE877A0120B0EE670A02F0EC
:10DAA00083FA03461946184802F05CF910E000BFFB
:10DAB0000EE000BF0CE000BF0AE000BF08E000BFBE
:10DAC00006E000BF04E000BF02E000BF00E000BFCE
:10DAD0000E4B1B7819460E4802F0F8F90C4802F07C
:10DAE0000DF903461A460B4B1A80084B00221A7098
:10DAF000CC37BD46F0BD00BF3003002018B102088E
:10DB000000A00C470000C84228B102083C0C0020CD
:10DB1000EC530020360C002080B485B000AF786054
:10DB20000023FB6002E0FB680133FB60FB687A685E
:10DB30009A42F8D800BF00BF1437BD465DF8047B99
:10DB40007047000080B500AF804B1B68002B02D0EF
:10DB50007E4B1B6898477E4B1B68002B0FD002F052
:10DB600063FB01467B4BA3FB01239A0813469B00F2
:10DB70001344CA1A002A02D1754B1B689847764B8A
:10DB80001B68002B10D002F04FFB0146714BA3FB2A
:10DB90000123DA0813469B0013445B00CA1A012ACA
:10DBA00002D16D4B1B6898476C4B1B68002B10D043
:10DBB00002F03AFB0146674BA3FB0123DA08134648
:10DBC0009B0013445B00CA1A022A02D1634B1B68F4
:10DBD0009847634B1B68002B0FD002F025FB0246D1
:10DBE000604BA3FB02131B09322101FB03F3D31A81
:10DBF000032B02D15A4B1B6898475B4B1B68002BC9
:10DC00000FD002F011FB0246564BA3FB02131B0977
:10DC1000322101FB03F3D31A0D2B02D1524B1B68A7
:10DC20009847524B1B68002B0FD002F0FDFA0246BA
:10DC30004C4BA3FB02135B09642101FB03F3D31AD2
:10DC4000042B02D1494B1B689847494B1B68002B9A
:10DC50000FD002F0E9FA0246464BA3FB02131B0960
:10DC6000FA2101FB03F3D31A052B02D1404B1B68A9
:10DC70009847414B1B68002B10D002F0D5FA0246A2
:10DC80003C4BA3FB02135B094FF4FA7101FB03F356
:10DC9000D31A062B02D1384B1B689847374B1B68A9
:10DCA000002B10D002F0C0FA0246324BA3FB021345
:10DCB0009B094FF47A7101FB03F3D31A072B02D1AE
:10DCC0002E4B1B6898472E4B1B68002B10D002F080
:10DCD000ABFA02462B4BA3FB02135B0B42F2107113
:10DCE00001FB03F3D31A082B02D1254B1B6898477D
:10DCF000254B1B68002B10D002F096FA0246234BEE
:10DD0000A3FB02139B0B4EF6602101FB03F3D31A16
:10DD1000092B02D11C4B1B6898471D4B1B68002B1D
:10DD200011D002F081FA03461A4A1288B3FBF2F1CD
:10DD300001FB02F29B1A174A1288013A934202D160
:10DD4000134B1B68984700BF80BD00BF580C0020D4
:10DD50005C0C0020CDCCCCCC600C0020640C0020EE
:10DD6000680C00201F85EB516C0C0020700C00200B
:10DD7000740C0020D34D6210780C00207C0C002025
:10DD8000800C00205917B7D1840C002073B2E745EE
:10DD9000880C00208C0C002080B483B000AF786029
:10DDA000044A7B68136000BF0C37BD465DF8047BF6
:10DDB000704700BF5C0C002080B483B000AF786077
:10DDC000044A7B68136000BF0C37BD465DF8047BD6
:10DDD000704700BF640C002080B483B000AF78604F
:10DDE000044A7B68136000BF0C37BD465DF8047BB6
:10DDF000704700BF680C002080B483B000AF78602B
:10DE0000044A7B68136000BF0C37BD465DF8047B95
:10DE1000704700BF6C0C002080B483B000AF786006
:10DE2000044A7B68136000BF0C37BD465DF8047B75
:10DE3000704700BF700C002080B483B000AF7860E2
:10DE4000044A7B68136000BF0C37BD465DF8047B55
:10DE5000704700BF840C002080B400AF034B002249
:10DE60001A6000BFBD465DF8047B7047600C00205F
:10DE700080B400AF034B00221A6000BFBD465DF8BE
:10DE8000047B7047680C002080B400AF034B002275
:10DE90001A6000BFBD465DF8047B7047640C00202B
:10DEA00080B400AF034B00221A6000BFBD465DF88E
:10DEB000047B70476C0C002080B500AF104BD3ED95
:10DEC0000B7AF5EE407AF1EE10FA0CD10C4BD3ED53
:10DED0000C7AF5EE407AF1EE10FA04D19FED090AC2
:10DEE000F4F726FF03E09FED080AF4F721FF074B44
:10DEF0001B8901339AB2054B1A8100BF80BD00BF58
:10DF0000D8010020CDCCCC3DCDCCCC3C400C002069
:10DF100080B400AF054B5B8901339AB2034B5A8141
:10DF200000BFBD465DF8047B704700BF400C002079
:10DF300080B500AF002001F02DFA012001F02AFA8F
:10DF4000084B1B68002B04D0012B03D1FCF7E0FA2F
:10DF500000E000BF044B9B8901339AB2024B9A81C7
:10DF600000BF80BD240C0020400C002080B500AF15
:10DF7000174B184A1A60164B4FF482725A60144BB2
:10DF800000229A60124B0022DA60114B00221A61C3
:10DF90000F4B00225A610E4B4FF400729A610C4BEA
:10DFA0001822DA610A4B00221A62094B00225A62D7
:10DFB000074B00229A62064B0A22DA62044807F0F5
:10DFC00047FD0346002B01D0FBF793FE00BF80BD49
:10DFD000900C00200030014080B500AF174B184A6C
:10DFE0001A60164B4FF482725A60144B00229A60EA
:10DFF000124B0022DA60114B00221A610F4B0022F3
:10E000005A610E4B4FF480229A610C4B0022DA6168
:10E010000A4B00221A62094B00225A62074B002267
:10E020009A62064B0A22DA62044807F011FD0346A1
:10E03000002B01D0FBF75DFE00BF80BDE80C002087
:10E040000034014080B58CB000AF786007F11C034C
:10E0500000221A605A609A60DA601A617B681B6855
:10E06000424A934244D10023BB61414B5B6C404A1E
:10E0700043F4805353643E4B5B6C03F48053BB61A9
:10E08000BB6900237B613A4B1B6B394A43F00203A7
:10E090001363374B1B6B03F002037B617B6918230F
:10E0A000FB6102233B6200237B620323BB620523E7
:10E0B000FB6207F11C0319462E4804F0EDFA2023F9
:10E0C000FB6102233B6202237B620323BB620523C5
:10E0D000FB6207F11C031946264804F0DDFA002212
:10E0E0000A21232003F053FA232003F06CFA39E0CD
:10E0F0007B681B68204A934234D100233B611C4B50
:10E100005B6C1B4A43F400535364194B5B6C03F480
:10E1100000533B613B690023FB60154B1B6B144AAA
:10E1200043F040031363124B1B6B03F04003FB608F
:10E13000FB684FF4F043FB6102233B6200237B62E8
:10E140000323BB620623FB6207F11C0319460B483D
:10E1500004F0A2FA00220A21542003F018FA5420F5
:10E1600003F031FA00BF3037BD4680BD00300140BA
:10E170000038024000040240003401400018024010
:10E1800080B483B000AF00237B60104B5B6C0F4A00
:10E1900043F4804353640D4B5B6C03F480437B601A
:10E1A0007B6800233B60094B1B6C084A43F080539B
:10E1B0001364064B1B6C03F080533B603B6800BF4D
:10E1C0000C37BD465DF8047B704700BF0038024045
:10E1D00080B400AF00BFFDE780B400AF00BFFDE733
:10E1E00080B400AF00BFFDE780B400AF00BFFDE723
:10E1F00080B400AF00BFFDE780B400AF00BFBD46F4
:10E200005DF8047B704780B400AF00BFBD465DF889
:10E21000047B704780B400AF00BFBD465DF8047B4F
:10E22000704780B500AF01F0EBFF03F0F8F900BFD5
:10E2300080BD000080B500AF054B5B8801339AB20A
:10E24000034B5A80012004F0FBFC00BF80BD00BFDF
:10E25000400D002080B500AF084BDB8801339AB237
:10E26000064BDA80064802F0A4F8064802F0A1F84E
:10E27000054802F09EF800BF80BD00BF400D0020A1
:10E280001C09002064090020AC09002080B500AF03
:10E29000064B1B8901339AB2044B1A81044808F0DB
:10E2A000BBF9044808F0B8F900BF80BD400D00205C
:10E2B000680D0020D00E002080B500AF054B5B89B3
:10E2C00001339AB2034B5A81034808F0A5F900BF05
:10E2D00080BD00BF400D0020680D002080B500AF5C
:10E2E000054B9B8901339AB2034B9A81034808F08E
:10E2F00093F900BF80BD00BF400D0020680D0020D5
:10E3000080B500AF054BDB8901339AB2034BDA814C
:10E31000034808F081F900BF80BD00BF400D002018
:10E32000B00D002080B500AF054B1B8A01339AB2B7
:10E33000034B1A82034808F06FF900BF80BD00BF8D
:10E34000400D0020F80D002080B500AF054B5B8A22
:10E3500001339AB2034B5A82034804F0CDFD00BF4B
:10E3600080BD00BF400D0020980B002080B500AF9D
:10E37000054B9B8A01339AB2034B9A82034804F0FF
:10E380000EFF00BF80BD00BF400D0020980B002095
:10E3900080B500AF054BDB8A01339AB2034BDA82BA
:10E3A000034807F0DFFB00BF80BD00BF400D002029
:10E3B000900C002080B500AF054B1B8B01339AB247
:10E3C000034B1A83034809F0B3F900BF80BD00BFB7
:10E3D000400D0020A853002080B500AF054B5B8B9B
:10E3E00001339AB2034B5A83034809F0A1F900BFE5
:10E3F00080BD00BF400D0020EC53002080B500AF71
:10E40000074B9B8B01339AB2054B9A834FF4005014
:10E4100004F016FC4FF4004004F012FC00BF80BD75
:10E42000400D002080B500AF024808F0F5F800BFAD
:10E4300080BD00BF880E002080B500AF054BDB8B90
:10E4400001339AB2034BDA83034808F0E5F800BFC2
:10E4500080BD00BF400D0020880E002080B500AFB9
:10E46000054B1B8C01339AB2034B1A84034808F006
:10E47000D3F800BF80BD00BF400D0020880E0020F3
:10E4800080B500AF054B5B8C01339AB2034B5A84C5
:10E49000034803F0A1FB00BF80BD00BF400D00207A
:10E4A000F409002080B500AF024807F05BFB00BF15
:10E4B00080BD00BFE80C002080B586B000AF78605A
:10E4C000144A154BD31A7B617B693B61134B1B6864
:10E4D000002B02D1114B124A1A60104B1A687B684C
:10E4E00013443A699A4207D209F0ACFF03460C2262
:10E4F0001A604FF0FF3309E0084B1B68FB60074BC5
:10E500001A687B681344054A1360FB68184618377D
:10E51000BD4680BD0000022000040000640D002004
:10E52000B855002080B400AF074BD3F88830064AB6
:10E5300043F47003C2F88830034B044A9A6000BF6A
:10E54000BD465DF8047B704700ED00E00040000828
:10E5500080B596B000AF07F1480300221A605A60F8
:10E560009A60DA6007F1400300221A605A6007F1EE
:10E57000240300221A605A609A60DA601A615A61B4
:10E580009A613B1D20220021184609F053FF534B8E
:10E59000534A1A60514B00225A60504B60229A60D5
:10E5A0004E4B42F22732DA604C4B00221A614B4B41
:10E5B00001225A61494B00229A61484807F0E4FB66
:10E5C0000346002B01D0FBF794FB4FF48053BB6450
:10E5D00007F148031946414808F0E8F90346002BC3
:10E5E00001D0FBF786FB3D4807F01DFC0346002BDE
:10E5F00001D0FBF77EFB20233B6480237B6407F183
:10E6000040031946354808F0A5FE0346002B01D00B
:10E61000FBF76FFB60237B620023BB620023FB627E
:10E6200000233B6300237B630023BB630023FB6366
:10E6300007F1240300221946284808F0F5F803469C
:10E64000002B01D0FBF755FB07F1240304221946E8
:10E65000224808F0E9F80346002B01D0FBF749FBFC
:10E6600007F12403082219461C4808F0DDF8034688
:10E67000002B01D0FBF73DFB42F22633BB6207F1D2
:10E6800024030C221946154808F0CEF80346002B47
:10E6900001D0FBF72EFB4FF400637B604FF48063E7
:10E6A000BB600023FB606B233B614FF480537B61B5
:10E6B0000023BB6100233B623B1D1946074808F05D
:10E6C000C5FE0346002B01D0FBF713FB034800F007
:10E6D0008DFB00BF5837BD4680BD00BF680D0020D0
:10E6E0000000014080B58CB000AF07F10C0324227C
:10E6F0000021184609F09EFE3B1D00221A605A6058
:10E70000214B4FF080421A601F4B00225A601E4B73
:10E7100000229A601C4B4FF6FF72DA601A4B0022FF
:10E720001A61194B00229A610323FB6000233B61AD
:10E7300001237B610023BB610023FB6100233B625B
:10E7400001237B620023BB620023FB6207F10C0301
:10E7500019460D4807F0E8FD0346002B01D0FBF7F2
:10E76000C8FA00237B600023BB603B1D19460648A6
:10E7700008F0F0FD0346002B01D0FBF7BAFA00BF0A
:10E780003037BD4680BD00BFB00D002080B58CB0D5
:10E7900000AF07F10C0324220021184609F04AFEBD
:10E7A0003B1D00221A605A60204B214A1A601F4B01
:10E7B00000225A601D4B00229A601C4B4FF6FF72DC
:10E7C000DA601A4B00221A61184B00229A61032367
:10E7D000FB6000233B6101237B610023BB610023BD
:10E7E000FB6100233B6201237B620023BB620023A9
:10E7F000FB6207F10C0319460C4807F095FD034630
:10E80000002B01D0FBF775FA00237B600023BB606F
:10E810003B1D1946054808F09DFD0346002B01D01D
:10E82000FBF767FA00BF3037BD4680BDF80D00200A
:10E830000008004080B58AB000AF07F12003002235
:10E840001A605A603B1D00221A605A609A60DA60B2
:10E850001A615A619A61204B204A1A601E4B0022AD
:10E860005A601D4B20229A601B4B1D4ADA601A4BDE
:10E8700000221A61184B00229A61174807F0D3FA58
:10E880000346002B01D0FBF734FA00233B62002340
:10E890007B6207F1200319460F4808F05BFD034631
:10E8A000002B01D0FBF725FA60237B600123BB60BE
:10E8B0000023FB6000237B613B1D002219460648B4
:10E8C00007F0B2FF0346002B01D0FBF712FA00BF9E
:10E8D0002837BD4680BD00BF400E0020000C004020
:10E8E0008F5F010080B596B000AF07F148030022AA
:10E8F0001A605A609A60DA6007F1400300221A60D9
:10E900005A6007F1240300221A605A609A60DA60A4
:10E910001A615A619A613B1D20220021184609F0B4
:10E9200089FD4B4B4B4A1A60494B00225A60484BB9
:10E9300060229A60464B42F22732DA60444B002252
:10E940001A61434B01225A61414B00229A614048AF
:10E9500007F01AFA0346002B01D0FBF7CAF94FF46F
:10E960008053BB6407F148031946394808F01EF884
:10E970000346002B01D0FBF7BCF9354807F053FAEA
:10E980000346002B01D0FBF7B4F920233B6480231E
:10E990007B6407F1400319462D4808F0DBFC034671
:10E9A000002B01D0FBF7A5F960237B620023BB623B
:10E9B0000023FB6200233B6300237B630023BB63D4
:10E9C0000023FB6307F1240300221946204807F0C7
:10E9D0002BFF0346002B01D0FBF78BF907F1240333
:10E9E000042219461A4807F01FFF0346002B01D0E6
:10E9F000FBF77FF907F1240308221946144807F0B2
:10EA000013FF0346002B01D0FBF773F94FF40063AB
:10EA10007B604FF48063BB600023FB606B233B6132
:10EA20004FF480537B610023BB6100233B623B1D9D
:10EA30001946074808F00AFD0346002B01D0FBF7F2
:10EA400058F9034800F0D2F900BF5837BD4680BDE1
:10EA5000880E00200004014080B588B000AF3B1D47
:10EA600000221A605A609A60DA601A615A619A61EB
:10EA70001F4B204A1A601E4B00225A601C4B00227A
:10EA80009A601B4B44F24E62DA60194B00221A6105
:10EA9000174B00229A61164807F0C5F90346002B70
:10EAA00001D0FBF726F960237B600023BB600023C5
:10EAB000FB6000237B613B1D002219460C4807F0D8
:10EAC000B3FE0346002B01D0FBF713F93B1D0422D4
:10EAD0001946074807F0A8FE0346002B01D0FBF7B4
:10EAE00008F9034800F082F900BF2037BD4680BD19
:10EAF000D00E00200040014080B58CB000AF78609F
:10EB000007F11C0300221A605A609A60DA601A61E9
:10EB10007B681B684A4A934245D10023BB61494B3D
:10EB20005B6C484A43F001035364464B5B6C03F053
:10EB30000103BB61BB6900237B61424B1B6B414AF4
:10EB400043F0100313633F4B1B6B03F010037B6117
:10EB50007B694FF40043FB6102233B6201237B622C
:10EB60000023BB620123FB6207F11C0319463648F0
:10EB700003F092FD00220021182002F008FD182069
:10EB800002F021FD00220021192002F000FD1920D1
:10EB900002F019FD002200211A2002F0F8FC1A20D0
:10EBA00002F011FD48E07B681B68284A934243D17C
:10EBB00000233B61234B5B6C224A43F00203536406
:10EBC000204B5B6C03F002033B613B690023FB605D
:10EBD0001C4B1B6B1B4A43F001031363194B1B6B4C
:10EBE00003F00103FB60FB684023FB6102233B62EF
:10EBF00001237B620023BB620323FB6207F11C033A
:10EC00001946134803F048FD002200212B2002F092
:10EC1000BEFC2B2002F0D7FC002200212C2002F0A9
:10EC2000B6FC2C2002F0CFFC002200212D2002F0A7
:10EC3000AEFC2D2002F0C7FC00BF3037BD4680BDC2
:10EC40000000014000380240001002400004014072
:10EC50000000024080B58CB000AF786007F11C0363
:10EC600000221A605A609A60DA601A617B681B6839
:10EC7000B3F1804F35D10023BB61394B1B6C384A4F
:10EC800043F001031364364B1B6C03F00103BB61BB
:10EC9000BB6900237B61324B1B6B314A43F002039B
:10ECA00013632F4B1B6B03F002037B617B694FF4F3
:10ECB0004073FB6102233B6200237B620023BB6243
:10ECC0000123FB6207F11C031946264803F0E4FC0C
:10ECD000002200211C2002F05AFC1C2002F073FCD0
:10ECE00039E07B681B68204A934234D100233B61A2
:10ECF0001B4B1B6C1A4A43F004031364184B1B6C28
:10ED000003F004033B613B690023FB60144B1B6B66
:10ED1000134A43F008031363114B1B6B03F0080302
:10ED2000FB60FB684FF44053FB6102233B6200230E
:10ED30007B620023BB620223FB6207F11C031946BE
:10ED40000A4803F0A9FC002200211E2002F01FFC4B
:10ED50001E2002F038FC00BF3037BD4680BD00BF2A
:10ED6000003802400004024000080040000C02404D
:10ED700080B584B000AF78607B681B68184A934206
:10ED80000ED10023FB60174B1B6C164A43F008039F
:10ED90001364144B1B6C03F00803FB60FB681AE060
:10EDA0007B681B68104A934215D10023BB600D4B52
:10EDB0005B6C0C4A43F4803353640A4B5B6C03F482
:10EDC0008033BB60BB6800220021182002F0DFFB0B
:10EDD000182002F0F8FB00BF1037BD4680BD00BF11
:10EDE000000C0040003802400040014080B58EB069
:10EDF00000AF786007F1240300221A605A609A601D
:10EE0000DA601A617B681B68654A93423ED1002331
:10EE10003B62644B1B6B634A43F010031363614B0B
:10EE20001B6B03F010033B623B6A0023FB615D4BED
:10EE30001B6B5C4A43F0020313635A4B1B6B03F0DA
:10EE40000203FB61FB694FF478537B620223BB62D0
:10EE50000023FB6200233B6301237B6307F1240350
:10EE60001946514803F018FC4FF400537B6202230B
:10EE7000BB620023FB6200233B6301237B6307F13A
:10EE800024031946494803F007FC84E07B681B68AB
:10EE9000474A93425CD10023BB61424B1B6B414A02
:10EEA00043F0010313633F4B1B6B03F00103BB6192
:10EEB000BB6900237B613B4B1B6B3A4A43F0020367
:10EEC0001363384B1B6B03F002037B617B690023E8
:10EED0003B61344B1B6B334A43F004031363314BE8
:10EEE0001B6B03F004033B613B6980237B620223BD
:10EEF000BB620023FB6200233B6303237B6307F1B8
:10EF0000240319462B4803F0C7FB4FF440437B62B0
:10EF10000223BB620023FB6200233B6303237B636A
:10EF200007F124031946214803F0B6FB4FF4E073C0
:10EF30007B620223BB620023FB6200233B6303234B
:10EF40007B6307F1240319461B4803F0A5FB22E06D
:10EF50007B681B68194A93421DD10023FB60114B4B
:10EF60001B6B104A43F0100313630E4B1B6B03F033
:10EF70001003FB60FB6860237B620223BB620023FB
:10EF8000FB6200233B6303237B6307F124031946E1
:10EF9000054803F081FB00BF3837BD4680BD00BF88
:10EFA000000001400038024000100240000402400E
:10EFB00000040140000002400008024000400140FF
:10EFC00080B582B000AF78607B681B68214A9342AD
:10EFD00019D1214B5B6C204A23F0010353644FF499
:10EFE0003E411E4803F0ECFC4FF400511C4803F076
:10EFF000E7FC182002F0F5FA192002F0F2FA1A20C4
:10F0000002F0EFFA21E07B681B68164A93421CD19C
:10F01000114B5B6C104A23F002035364C021124869
:10F0200003F0CEFC4FF440410D4803F0C9FC4FF40F
:10F03000E0710E4803F0C4FC2B2002F0D2FA2C2021
:10F0400002F0CFFA2D2002F0CCFA00BF0837BD46FF
:10F0500080BD00BF000001400038024000100240A7
:10F060000004024000040140000002400008024089
:10F0700080B582B000AF78607B681B68B3F1804FC9
:10F080000ED1134B1B6C124A23F0010313644FF48F
:10F090004071104803F094FC1C2002F0A2FA12E028
:10F0A0007B681B680C4A93420DD1094B1B6C084AC4
:10F0B00023F0040313644FF44051084803F080FC2C
:10F0C0001E2002F08EFA00BF0837BD4680BD00BF8B
:10F0D000003802400004024000080040000C0240DA
:10F0E00080B582B000AF78607B681B680D4A9342A0
:10F0F00006D10D4B1B6C0C4A23F0080313640DE082
:10F100007B681B68094A934208D1074B5B6C064A2F
:10F1100023F480335364182002F063FA00BF0837E9
:10F12000BD4680BD000C0040003802400040014058
:10F1300080B500AF094B1B6800225A63074B1B6860
:10F1400044F24F62DA62054B44F24F62DA6000210A
:10F15000024806F0D3FF00BF80BD00BFD00E0020E4
:10F1600080B500AF874B1B68874A5362F9F7FCF9FB
:10F17000F0EE407A844BC3ED0A7A834B1B78002B68
:10F1800008D0814BDB69804AD3627F4B1B6A7E4A81
:10F19000136307E07C4B5B6A7B4AD3627A4B9B6AC2
:10F1A000794A1363784BD3ED117AB7EE007A37EED4
:10F1B000677A754BD3ED0D7A27EE277A724BD3ED34
:10F1C000116A714BD3ED0B7A66EEA77A77EE277A48
:10F1D0006D4BC3ED0D7A6C4BD3ED127AB7EE007A1E
:10F1E00037EE677A684BD3ED0E7A27EE277A664BB7
:10F1F000D3ED126A644BD3ED0C7A66EEA77A77EE04
:10F20000277A614BC3ED0E7A5F4B93ED017A5E4B2B
:10F21000D3ED027A37EE677AF7EE006AC6EE877AA8
:10F22000594BC3ED037A584B93ED047A564BD3ED0B
:10F23000057A37EE677AF7EE006AC6EE877A524BA8
:10F24000C3ED067A504B93ED0D7A4F4BD3ED027A16
:10F25000B4EEE77AF1EE10FA24DD4B4B93ED0D7A24
:10F26000494BD3ED027A77EE677A474BC3ED0F7ABD
:10F27000454B93ED0F7A444BD3ED037A27EE277A73
:10F28000414BD3ED137A67EE277A9FED407A67EE14
:10F29000877AFDEEE77A17EE903A9AB23A4BA3F8E6
:10F2A000542003E0384B0022A3F85420364B93ED52
:10F2B0000E7A354BD3ED057AB4EEE77AF1EE10FA1B
:10F2C00024D5314B93ED0E7A2F4BD3ED057A77EEA3
:10F2D000677A2D4BC3ED107A2B4B93ED107A2A4BA6
:10F2E000D3ED067A27EE277A274BD3ED147A67EE13
:10F2F000277A9FED267A67EE877AFDEEE77A17EE9A
:10F30000903A9AB2204BA3F8562003E01E4B0022FD
:10F31000A3F856201C4BB3F856201B4BB3F85430BF
:10F32000934238BF13469AB2174BA3F85820164B96
:10F33000B3F8583044F2CB22934204D9124B44F232
:10F34000CB22A3F85820104BB3F85A200E4BB3F839
:10F3500058309A4208D20C4BB3F85A3001339AB263
:10F36000094BA3F85A2005E0074BB3F85820064B89
:10F37000A3F85A20044BB3F85A20054B1B685A6374
:10F3800000BF80BD0004002080020020009E8C464B
:10F39000D00E002080B485B000AF0346FB71FB792E
:10F3A000012B00F24B81FB79002B02D0012B0DD0F9
:10F3B00019E0A54BD3ED017AB2EE047A67EE877AB5
:10F3C000FDEEE77A17EE903AFB600CE09F4BD3ED31
:10F3D000017AB2EE047A67EE877AFDEEE77A17EEED
:10F3E000903AFB6000BFFB79994A04335B001344F9
:10F3F000B3F902301946FB79954A04335B00134494
:10F40000B3F902301A46FB7901FB02F29049083346
:10F410009B000B445A608E4B1B78002B02D0012BB3
:10F420000AD022E0F979FB6803FB03F288488B1DC0
:10F430009B0003445A6018E0FB79854A08335B005F
:10F440001344B3F902301946FB79814A08335B0053
:10F450001344B3F902301A46FB7901FB02F27C49EE
:10F4600006339B000B445A6000BFFB79784A063391
:10F470009B0013445A68FB79754908339B000B4481
:10F480005B68D31ABB60BB68002B0DDABB6807EE64
:10F49000903AF8EEE77AB6EE007A67EE877AFDEEFC
:10F4A000E77A17EE903ABB60FB79694A0A339B0012
:10F4B00013445968FB79BA680A4465490A339B00CA
:10F4C0000B445A60FB79624A0A339B0013445B6821
:10F4D000002B06DAFB795E4A0A339B0013440022B4
:10F4E0005A60FB795A4A0A339B0013445A68584BB6
:10F4F0009B6B9A4207DDFB79554A926B54490A335C
:10F500009B000B445A60524B9B6B07EE903AF8EE0F
:10F51000E77ADFED506A86EEA77A4D4B9A6BFB795E
:10F520004B490A339B000B445B68D31A07EE903AB1
:10F53000F8EEE77A67EE277AFDEEE77AC7ED007A14
:10F54000FB793978424A13440A4683F83C20FB7918
:10F550003F4A134493F83C30642B05D9FB793C4A6D
:10F560001344642283F83C20394B93F8483007EE6B
:10F57000903AB8EEE77AFB79354A134493F83C3079
:10F5800007EE903AF8EEE77ADFED336A67EEA66AA7
:10F59000324BD3ED057AB2EE046A27EE866A2C4B25
:10F5A00093F8483007EE903AF8EEE77A76EE677A0D
:10F5B00066EEA77A77EE277AFB799FED297A67EED8
:10F5C000877A234A10339B001344C3ED007A204B03
:10F5D0005B6801331E4A53601D4B1B78002B2AD0F9
:10F5E000012B00D02AE0FB79194A08335B00134451
:10F5F000B3F90220FB79164904335B000B44B3F9DD
:10F6000002309A4219DDFB79114A10339B001344F2
:10F61000D3ED007AB2EE047A67EE877AFDEEE77AF0
:10F62000FB7917EE902A11B2094A08335B001344A4
:10F630000A465A8001E000BF00E000BF00BF143757
:10F64000BD465DF8047B7047740500200407002068
:10F65000DC0200200000C8420AD7233C1001002031
:10F66000CDCCCC3D80B483B000AF786000BF0C3708
:10F67000BD465DF8047B704780B483B000AF78600E
:10F6800000BF0C37BD465DF8047B704780B483B083
:10F6900000AF786000BF0C37BD465DF8047B704753
:10F6A00080B483B000AF786000BF0C37BD465DF812
:10F6B000047B704780B483B000AF78607B681B68C0
:10F6C000034A934200BF0C37BD465DF8047B704788
:10F6D0000040014080B582B000AF164B164A1A6058
:10F6E000144B4FF4E1325A60124B00229A60114BD6
:10F6F0000022DA600F4B00221A610E4B0C225A6175
:10F700000C4B00229A610B4B0022DA61094807F08A
:10F710001EFF0346002B01D0FAF7EBFA0023FB7122
:10F72000FB791946034800F07BFA00BF0837BD4655
:10F7300080BD00BFA85300200044004080B582B0C7
:10F7400000AF164B164A1A60144B4FF4E1325A6060
:10F75000124B00229A60114B0022DA600F4B0022FC
:10F760001A610E4B0C225A610C4B00229A610B4B12
:10F770000022DA61094807F0EAFE0346002B01D0B7
:10F78000FAF7B7FA0023FB71FB791946034800F03A
:10F7900047FA00BF0837BD4680BD00BFEC530020CC
:10F7A0000048004080B58CB000AF786007F11C03C2
:10F7B00000221A605A609A60DA601A617B681B68DE
:10F7C0003A4A934234D10023BB61394B1B6C384A0F
:10F7D00043F400331364364B1B6C03F40033BB61FA
:10F7E000BB6900237B61324B1B6B314A43F008033A
:10F7F00013632F4B1B6B03F008037B617B69602352
:10F80000FB6102233B6200237B620323BB6207236D
:10F81000FB6207F11C031946264802F03DFF002257
:10F820000A21262001F0B3FE262001F0CCFE39E0AB
:10F830007B681B68204A934234D100233B611C4BF8
:10F840001B6C1B4A43F480231364194B1B6C03F499
:10F8500080233B613B690023FB60154B1B6B144A03
:10F8600043F008031363124B1B6B03F00803FB60A8
:10F87000FB684FF44073FB6102233B6200237B6211
:10F880000323BB620723FB6207F11C0319460948E7
:10F8900002F002FF01220021272001F078FE27203C
:10F8A00001F091FE00BF3037BD4680BD00440040EE
:10F8B00000380240000C02400048004080B582B091
:10F8C00000AF78607B681B68134A93420DD1134BDD
:10F8D0001B6C124A23F4003313646021104803F0B8
:10F8E0006FF8262001F07DFE12E07B681B680D4A50
:10F8F00093420DD1094B1B6C084A23F480231364F7
:10F900004FF4E061064803F05BF8272001F069FE40
:10F9100000BF0837BD4680BD0044004000380240AB
:10F92000000C02400048004090B589B000AFF8607C
:10F93000B9601346FB71FB79002B10D1BB68FB61EA
:10F9400005E0FB790133FB71FB79802B06D0FB6965
:10F950005A1CFA611B78002BF3D100E000BFFB6852
:10F960001B68704A934269D16F4B1B781A466E4BE5
:10F970005B78013303F03F039A4235D00023FB76D6
:10F9800011E0FB7EBA681A44674B5B781C46FB7E2D
:10F9900010786549E2010A441344023302461A70A2
:10F9A000FB7E0133FB76FA7EFB799A42E9D35E4B0C
:10F9B0005B781A465C4B134403F500530233FA7923
:10F9C0001A70262001F00DFE574B5B780133DAB236
:10F9D000554B5A70544B5B7803F03F03DAB2524BED
:10F9E0005A70262001F0EFFD262001F0FAFD4F4B62
:10F9F00093F83D30DBB2202B1DD14B4B1B78DB0144
:10FA0000494A134402337B61474B1B780133DAB216
:10FA1000454B1A70444B1B7803F03F03DAB2424B5C
:10FA20001A70262001F0CFFDFB799BB21A46796946
:10FA3000F86807F008FE262001F0C5FDFB681B688A
:10FA40003B4A934269D13B4B1B781A46394B5B7852
:10FA5000013303F03F039A4235D00023BB7611E017
:10FA6000BB7EBA681A44334B5B781C46BB7E107869
:10FA70003049E2010A441344023302461A70BB7E45
:10FA80000133BB76BA7EFB799A42E9D3294B5B7886
:10FA90001A46284B134403F500530233FA791A70BF
:10FAA000272001F09EFD234B5B780133DAB2214B16
:10FAB0005A70204B5B7803F03F03DAB21D4B5A704B
:10FAC000272001F080FD272001F08BFD1A4B93F8D1
:10FAD0003D30DBB2202B1DD1164B1B78DB01154AC4
:10FAE000134402337B61134B1B780133DAB2114BA1
:10FAF0001A70104B1B7803F03F03DAB20D4B1A70EB
:10FB0000272001F060FDFB799BB21A467969F868FD
:10FB100007F099FD272001F056FD00BF2437BD46B0
:10FB200090BD00BF00440040180F0020A8530020E3
:10FB30000048004060310020EC53002080B584B0C4
:10FB400000AF78607B681B68304A93422AD1304B03
:10FB50001A782F4B5B789A4224D02D4B1B78DB010F
:10FB60002B4A13440233FB60294B1B781A46284B5F
:10FB7000134403F5005302331B78FB72244B1B78AC
:10FB80000133DAB2224B1A70214B1B7803F03F038A
:10FB9000DAB21F4B1A70FB7A9BB21A46F9681D48FD
:10FBA00007F051FD7B681B681B4A93422AD11B4B0F
:10FBB0001A781A4B5B789A4224D0184B1B78DB01D9
:10FBC000164A13440233FB60144B1B781A46134B3E
:10FBD000134403F5005302331B78FB720F4B1B7861
:10FBE0000133DAB20D4B1A700C4B1B7803F03F0354
:10FBF000DAB20A4B1A70FB7A9BB21A46F968786837
:10FC000007F021FD00BF1037BD4680BD0044004015
:10FC1000180F0020A8530020004800406031002049
:10FC200080B582B000AF78600B46FB70FB1C0122F0
:10FC30001946786807F04CFD00BF0837BD4680BD07
:10FC400080B483B000AF78607B681B68274A93421A
:10FC500020D1274B1B881A46254B5B880133DBB22A
:10FC60009A4217D07B681B685B68DAB2204B5B88CE
:10FC700011461F4A5B0013440A469A801C4B5B885E
:10FC800001339AB21A4B5A80194B5B88DBB29AB295
:10FC9000174B5A807B681B68164A934220D1164B3B
:10FCA0001B881A46144B5B880133DBB29A4217D08B
:10FCB0007B681B685B68DAB20F4B5B8811460E4AA3
:10FCC0005B0013440A469A800B4B5B8801339AB25F
:10FCD000094B5A80084B5B88DBB29AB2064B5A80BC
:10FCE00000BF0C37BD465DF8047B70470044004000
:10FCF0005C2F002000480040A451002080B485B053
:10FD000000AF78607B681B68124A93420AD1124B9D
:10FD10005B88DAB2104B1B88DBB2D31ABB73BB7B98
:10FD20009BB210E07B681B680C4A93420AD10C4BD3
:10FD30005B88DAB20A4B1B88DBB2D31AFB73FB7BFE
:10FD40009BB200E0002318461437BD465DF8047BE3
:10FD5000704700BF004400405C2F00200048004076
:10FD6000A45100200FB480B5C2B000AF07F58A726D
:10FD700007F58473A3F582731A6007F58473A3F5FE
:10FD8000827307F108001A68D7F8101108F048FBD1
:10FD900007F10803002219460548FFF7C5FD00BF1B
:10FDA00007F58477BD46BDE8804004B0704700BFCA
:10FDB000EC5300200FB480B5C2B000AF124B1B78DB
:10FDC000002B19D007F58A7207F58473A3F58273A7
:10FDD0001A6007F58473A3F5827307F108001A68A7
:10FDE000D7F8101108F01CFB07F108030022194690
:10FDF0000648FFF799FD00E000BF07F58477BD4690
:10FE0000BDE8804004B07047100C0020EC53002087
:10FE10000FB480B400AF00BFBD465DF8047B04B0F2
:10FE20007047000080B584B000AF78600B467B80DF
:10FE30007B681B681F4A934218D11F48FFF75EFF7B
:10FE400003461A467B88934202D34FF0FF332DE0DE
:10FE50001A4B1A887B8813449BB2DBB2174A5B00AB
:10FE600013449B88FB73FB7B1BB21FE07B681B6802
:10FE7000134A934218D11348FFF740FF03461A462E
:10FE80007B88934202D34FF0FF330FE00E4B1A886A
:10FE90007B8813449BB2DBB20B4A5B0013449B8804
:10FEA000FB73FB7B1BB201E04FF0FF3318461037AA
:10FEB000BD4680BD00440040A85300205C2F0020B8
:10FEC00000480040EC530020A451002080B584B0CD
:10FED00000AF78600B467B807B681B682C4A93429E
:10FEE00026D1262001F07DFB2A48FFF707FF0346B5
:10FEF000FB737B88002B04D1274B5A88264B1A8032
:10FF000013E0FB7B9BB27A889A4201D9FB7B7B8012
:10FF1000214B1A887B8813449AB21F4B1A801E4BC0
:10FF20001B88DBB29AB21C4B1A80262001F04BFBD7
:10FF30007B681B68194A934226D1272001F051FBA8
:10FF40001748FFF7DBFE0346FB737B88002B04D1C9
:10FF5000144B5A88134B1A8013E0FB7B9BB27A88B0
:10FF60009A4201D9FB7B7B800E4B1A887B88134415
:10FF70009AB20C4B1A800B4B1B88DBB29AB2094B1E
:10FF80001A80272001F01FFB00BF1037BD4680BD3F
:10FF900000440040A85300205C2F0020004800408F
:10FFA000EC530020A451002090B587B000AF87ED3E
:10FFB000010A38600A237B61D7ED017AF5EEC07A39
:10FFC000F1EE10FA08D50123FB74D7ED017AF1EEBA
:10FFD000677AC7ED017A01E00023FB743B68092BC7
:10FFE00002DD09233B6004E03B68002B01DC0123B8
:10FFF0003B603B68DBB2FA7CF97C05313033DCB224
:020000040802F0
:100000001F481346DB00134403440B4422461A7076
:1000100008E07A6913469B0013445B007B613B68F0
:10002000013B3B603B68012BF3DC7B6907EE903AB8
:10003000B8EEE77AD7ED017A67EE277AFDEEE77A38
:1000400017EE903AFB60FA7C1346DB0013440C4A2F
:100050009818FA687B6992FBF3F4FB687A6993FB62
:10006000F2F2796901FB02F29B1A22460146054829
:1000700008F0A0F9034B18461C37BD4690BD00BFE1
:10008000280000203854002080B582B000AF2C4BEF
:100090001B687B600720F8F729FD0346002B0CBF87
:1000A00001230023DBB21A46254B1A60244B1B6840
:1000B0007A68D31A012B0DD1224B01221A60224BF0
:1000C00003221A71214B002283F82A201F4B0022A1
:1000D00083F82B207B68002B06D1194B1B68012B62
:1000E00002D1194BFD221A71164B1B68012B22D12C
:1000F000F0F786FF154BD3ED0B7A9FED157AF4EEF2
:10010000C77AF1EE10FA00D415E0104BD3ED0C7A5B
:100110009FED0F7AF4EEC77AF1EE10FA00D40AE000
:100120000C4B4FF00002DA600A4B4FF000021A61EC
:10013000044B00221A6000BF0837BD4680BD00BFD7
:10014000305400203454002028030020D80100201F
:10015000CDCCCC3D4801002080B400AF00BFBD46EF
:100160005DF8047B70470000DFF834D00D480E497D
:100170000E4A002302E0D458C4500433C4188C4201
:10018000F9D30B4A0B4C002301E013600432A24266
:10019000FBD3FEF7C7F908F05BF9F9F703FB7047EB
:1001A00000000220000000209400002024DB020850
:1001B00094000020B8550020FEE7000080B500AF95
:1001C0000E4B1B680D4A43F4007313600B4B1B6806
:1001D0000A4A43F480631360084B1B68074A43F4E0
:1001E00080731360032001F0C7F90F20F9F7AAFA12
:1001F000FDF7C6FF0023184680BD00BF003C02404B
:1002000080B400AF064B1B781A46064B1B6813449C
:10021000044A136000BFBD465DF8047B704700BF11
:10022000400000204C54002080B400AF034B1B68FA
:100230001846BD465DF8047B704700BF4C54002053
:1002400080B584B000AF7860FFF7EEFFB8607B68E0
:10025000FB60FB68B3F1FF3F05D00A4B1B781A46E1
:10026000FB681344FB6000BFFFF7DEFF0246BB687C
:10027000D31AFA689A42F7D800BF00BF1037BD46BC
:1002800080BD00BF4000002080B400AF054B1B685C
:10029000044A23F00203136000BFBD465DF8047BEF
:1002A000704700BF10E000E080B400AF054B1B6852
:1002B000044A43F00203136000BFBD465DF8047BAF
:1002C000704700BF10E000E080B584B000AF7860F8
:1002D0000023FB737B68002B01D1012333E07B6893
:1002E0001B6C002B09D17868F7F7C8FD7B680022EA
:1002F0005A647B68002283F83C207B681B6C03F007
:100300001003002B18D17B681B6C23F4885323F057
:10031000020343F002027B681A64786800F0BAFBBB
:100320007B6800225A647B681B6C23F0030343F054
:1003300001027B681A6401E00123FB737B680022E1
:1003400083F83C20FB7B18461037BD4680BD80B546
:1003500084B000AF78600023FB737B68002B01D171
:10036000012322E07B681B6C43F002027B681A6465
:100370007B681B689A687B681B6822F001029A60A0
:100380007B681B689B6803F00103002B08D1786829
:10039000F7F70EFF7B6800225A647B6800221A641C
:1003A0007B68002283F83C20FB7B18461037BD4653
:1003B00080BD80B586B000AF786000237B610023EC
:1003C0003B617B681B681B68FB607B681B685B6824
:1003D000BB60FB6803F002037B61BB6803F0200392
:1003E0003B617B69002B49D03B69002B46D07B6881
:1003F0001B6C03F01003002B05D17B681B6C43F4CE
:1004000000727B681A647B681B689B6803F040532A
:10041000002B2BD17B681B7E002B27D17B681B68B0
:10042000DB6A03F47003002B06D07B681B689B68B3
:1004300003F48063002B19D17B681B685A687B68C2
:100440001B6822F020025A607B681B6C23F48072C8
:100450007B681A647B681B6C03F48053002B05D106
:100460007B681B6C43F001027B681A647868F8F7BC
:1004700071F87B681B686FF012021A60FB6803F06A
:1004800004037B61BB6803F080033B617B69002B45
:1004900057D03B69002B54D07B681B6C03F01003D2
:1004A000002B05D17B681B6C43F400527B681A64F7
:1004B0007B681B689B6803F44013002B39D17B6871
:1004C0001B689B6B03F44013002B06D07B681B68F2
:1004D0009B6803F48063002B2BD17B681B685B68EF
:1004E00003F48063002B24D17B681B689B6803F0B6
:1004F0004053002B1DD17B681B7E002B19D17B68DC
:100500001B685A687B681B6822F080025A607B680F
:100510001B6C23F480527B681A647B681B6C03F4A9
:100520008073002B05D17B681B6C43F001027B6854
:100530001A647868F7F7AAFE7B681B686FF00C02F4
:100540001A60FB6803F001037B61BB6803F04003A2
:100550003B617B69002B17D03B69002B14D07B6873
:100560001B681B6803F00103012B0DD17B681B6C1A
:1005700043F480327B681A64786800F045F97B6840
:100580001B686FF001021A60FB6803F020037B61B7
:10059000BB6803F080633B617B69002B15D03B692E
:1005A000002B12D07B685B6C43F002027B685A64BC
:1005B0007B681B686FF020021A60786800F02EF9E3
:1005C0007B681B686FF020021A6000BF1837BD46B9
:1005D00080BD000080B586B000AFF860B9607A6079
:1005E00000233B61FB6893F83C30012B01D10223CF
:1005F000E9E0FB68012283F83C20FB681B689B68EC
:1006000003F00103012B18D0FB681B689A68FB6894
:100610001B6842F001029A606D4B1B686D4AA2FB99
:1006200003239A0C13465B0013443B6102E03B69D1
:10063000013B3B613B69002BF9D1FB681B689B6860
:1006400003F48073B3F5807F07D1FB681B689A6859
:10065000FB681B6822F480729A60FB681B689B68C9
:1006600003F00103012B40F0A180FB681B6C23F415
:10067000E06323F0010343F48072FB681A64FB68B3
:100680001B685B6803F48063002B07D0FB681B6C5E
:1006900023F4405343F48052FB681A64FB681B6CDC
:1006A00003F48053B3F5805F06D1FB685B6C23F0E5
:1006B0000602FB685A6402E0FB6800225A64FB6889
:1006C000002283F83C20444B7B61FB689B6B434AD0
:1006D000DA63FB689B6B424A1A64FB689B6B414A76
:1006E000DA64FB681B686FF022021A60FB681B6803
:1006F0005A68FB681B6842F080625A60FB681B689E
:100700009A68FB681B6842F480729A60FB68986B79
:10071000FB681B684C331946BA687B6801F072F9B4
:100720007B695B6803F01F03002B2AD1FB681B6801
:100730002D4A934215D0FB681B682C4A934205D181
:10074000254B5B6803F01F03002B0AD0FB681B6876
:10075000274A934236D1204B5B6803F01003002BED
:1007600030D1FB681B689B6803F04053002B29D1F4
:10077000FB681B689A68FB681B6842F080429A60BD
:1007800020E0FB681B68184A93421BD1FB681B687A
:100790009B6803F04053002B14D1FB681B689A68D8
:1007A000FB681B6842F080429A600BE0FB681B6CA0
:1007B00043F01002FB681A64FB685B6C43F00102B3
:1007C000FB685A64002318461837BD4680BD00BF39
:1007D0002400002083DE1B43002301408D0C02080F
:1007E000470D0208630D020800200140002101406E
:1007F0000022014080B483B000AF786000BF0C37A6
:10080000BD465DF8047B704780B483B000AF78606C
:1008100000BF0C37BD465DF8047B704780B483B0E1
:1008200000AF786000BF0C37BD465DF8047B7047B1
:1008300080B485B000AF786039600023BB607B680E
:1008400093F83C30012B01D1022313E17B68012294
:1008500083F83C203B681B68092B25D97B681B6803
:10086000D9683B681B689BB21A4613465B00134469
:100870001E3B072202FA03F3DA437B681B680A4037
:10088000DA607B681B68D9683B689A683B681B68BC
:100890009BB2184603465B0003441E3B9A407B68AC
:1008A0001B680A43DA6022E07B681B6819693B68B1
:1008B0001B689BB21A4613465B001344072202FAD8
:1008C00003F3DA437B681B680A401A617B681B6884
:1008D00019693B689A683B681B689BB218460346D7
:1008E0005B0003449A407B681B680A431A613B68BB
:1008F0005B68062B24D87B681B68596B3B685A6879
:1009000013469B001344053B1F2202FA03F3DA430C
:100910007B681B680A405A637B681B68596B3B689D
:100920001B689BB218463B685A6813469B001344E9
:10093000053B00FA03F27B681B680A435A634CE0EC
:100940003B685B680C2B24D87B681B68196B3B6881
:100950005A6813469B001344233B1F2202FA03F3F9
:10096000DA437B681B680A401A637B681B68196B53
:100970003B681B689BB218463B685A6813469B004D
:100980001344233B00FA03F27B681B680A431A6393
:1009900023E07B681B68D96A3B685A6813469B0052
:1009A0001344413B1F2202FA03F3DA437B681B68BE
:1009B0000A40DA627B681B68D96A3B681B689BB295
:1009C00018463B685A6813469B001344413B00FAA3
:1009D00003F27B681B680A43DA62294BFB607B6881
:1009E0001B68284A93420FD13B681B68122B0BD11E
:1009F000FB685B6823F40002FB685A60FB685B6875
:100A000043F48002FB685A607B681B681D4A93426E
:100A10002BD13B681B681C4A934203D03B681B6880
:100A2000112B22D1FB685B6823F48002FB685A60BB
:100A3000FB685B6843F40002FB685A603B681B6814
:100A4000114A934211D1114B1B68114AA2FB032397
:100A50009A0C13469B0013445B00BB6002E0BB682A
:100A6000013BBB60BB68002BF9D17B68002283F897
:100A70003C20002318461437BD465DF8047B7047C0
:100A8000002301400020014012000010240000203B
:100A900083DE1B4380B485B000AF7860794BFB6088
:100AA000FB685B6823F44032FB685A60FB685A6855
:100AB0007B685B681A43FB685A607B681B685A68EE
:100AC0007B681B6822F480725A607B681B685968D7
:100AD0007B681B691A027B681B680A435A607B6843
:100AE0001B685A687B681B6822F040725A607B68FA
:100AF0001B6859687B689A687B681B680A435A6060
:100B00007B681B689A687B681B6822F400629A60A5
:100B10007B681B6899687B68DA687B681B680A4396
:100B20009A607B689B6A584A934222D07B681B6814
:100B30009A687B681B6822F070629A607B681B6809
:100B400099687B689A6A7B681B680A439A607B682D
:100B50001B689A687B681B6822F040529A607B6829
:100B60001B6899687B68DA6A7B681B680A439A602D
:100B70000FE07B681B689A687B681B6822F07062D4
:100B80009A607B681B689A687B681B6822F04052F9
:100B90009A607B681B689A687B681B6822F0020277
:100BA0009A607B681B6899687B681B7E5A007B682B
:100BB0001B680A439A607B6893F82030002B1BD097
:100BC0007B681B685A687B681B6842F400625A6045
:100BD0007B681B685A687B681B6822F460425A6015
:100BE0007B681B6859687B685B6A013B5A037B68BA
:100BF0001B680A435A6007E07B681B685A687B6879
:100C00001B6822F400625A607B681B68DA6A7B68A2
:100C10001B6822F47002DA627B681B68D96A7B6801
:100C2000DB69013B1A057B681B680A43DA627B6853
:100C30001B689A687B681B6822F400729A607B6864
:100C40001B6899687B6893F830305A027B681B6890
:100C50000A439A607B681B689A687B681B6822F469
:100C600080629A607B681B6899687B685B699A02FE
:100C70007B681B680A439A6000BF1437BD465DF865
:100C8000047B7047002301400100000F80B584B051
:100C900000AF78607B689B6BFB60FB681B6C03F0AC
:100CA0005003002B3CD1FB681B6C43F40072FB68C3
:100CB0001A64FB681B689B6803F04053002B2BD120
:100CC000FB681B7E002B27D1FB681B68DB6A03F4E3
:100CD0007003002B06D0FB681B689B6803F48063DD
:100CE000002B19D1FB681B685A68FB681B6822F04F
:100CF00020025A60FB681B6C23F48072FB681A6444
:100D0000FB681B6C03F48053002B05D1FB681B6C44
:100D100043F00102FB681A64F868F7F71BFC0EE069
:100D2000FB681B6C03F01003002B03D0F868FFF77F
:100D300075FD04E0FB689B6BDB6C7868984700BF2F
:100D40001037BD4680BD80B584B000AF78607B6849
:100D50009B6BFB60F868FFF74DFD00BF1037BD4689
:100D600080BD80B584B000AF78607B689B6BFB6012
:100D7000FB6840221A64FB685B6C43F00402FB686A
:100D80005A64F868FFF74AFD00BF1037BD4680BDC2
:100D900080B487B000AF78600023BB6000237B6124
:100DA00000233B617B6893F83C30012B01D1022387
:100DB000B2E07B68012283F83C207B681B689B685B
:100DC00003F00103012B18D07B681B689A687B68CD
:100DD0001B6842F001029A60524B1B68524AA2FB08
:100DE00003239A0C13465B001344BB6002E0BB680C
:100DF000013BBB60BB68002BF9D17B681B689B681B
:100E000003F00103012B7AD17B681B6C23F4405360
:100E100023F0010343F480527B681A647B681B6CE7
:100E200003F48073002B02D17B6800225A647B6834
:100E3000002283F83C207B681B686FF004021A6074
:100E40007B681B685A687B681B6842F080025A60A6
:100E5000364BFB60FB685B6803F01F03002B24D15B
:100E60007B681B689B6803F44013002B0CBF0123B5
:100E70000023DBB27B617B681B685B6803F48063E3
:100E8000002B0CBF01230023DBB23B617B69002BED
:100E900041D03B69002B3ED07B681B689A687B6819
:100EA0001B6842F480029A6035E07B681B689B688F
:100EB00003F44013002B0CBF01230023DBB27B6142
:100EC0007B681B685B6803F48063002B0CBF012305
:100ED0000023DBB23B617B681B68154A93421AD141
:100EE0007B69002B17D03B69002B14D07B681B68F3
:100EF0009A687B681B6842F480029A600BE07B680A
:100F00001B6C43F010027B681A647B685B6C43F0D7
:100F100001027B685A64002318461C37BD465DF801
:100F2000047B70472400002083DE1B430023014024
:100F30000020014080B485B000AF786039600023A4
:100F4000FB607B681B686FF004021A603B68013B22
:100F5000032B1FD801A252F823F000BF8B0F020809
:100F6000810F0208770F02086D0F02087B681B686B
:100F70009B6CFB600FE07B681B685B6CFB600AE0AE
:100F80007B681B681B6CFB6005E07B681B68DB6B88
:100F9000FB6000E000BFFB6818461437BD465DF8F3
:100FA000047B704780B485B000AF786039607B689F
:100FB00093F83C30012B01D102237EE17B680122B2
:100FC00083F83C203B681B68092B25D97B681B688C
:100FD000D9683B681B689BB21A4613465B001344F2
:100FE0001E3B072202FA03F3DA437B681B680A40C0
:100FF000DA607B681B68D9683B689A683B681B6845
:101000009BB2184603465B0003441E3B9A407B6834
:101010001B680A43DA6022E07B681B6819693B6839
:101020001B689BB21A4613465B001344072202FA60
:1010300003F3DA437B681B680A401A617B681B680C
:1010400019693B689A683B681B689BB2184603465F
:101050005B0003449A407B681B680A431A617B6803
:101060001B689A6B7B681B6822F440129A637B684A
:101070001B68996B3B681B69013B1A057B681B6801
:101080000A439A637B681B68996B3B685B68DAB2BA
:101090003B681B69DBB2D31ADBB20333DBB21A46FF
:1010A00013469B0013441F2202FA03F3DA437B68C2
:1010B0001B680A409A637B681B68996B3B681B68D6
:1010C0009BB218463B685B68DAB23B681B69DBB2CF
:1010D000D31ADBB20333DBB21A4613469B00134428
:1010E00000FA03F27B681B680A439A633B689B69BA
:1010F000754A934222D07B681B689A687B681B689C
:1011000022F470229A607B681B6899683B689A6930
:101110007B681B680A439A607B681B689A687B68D7
:101120001B6822F440129A607B681B6899683B68D0
:10113000DA697B681B680A439A600FE07B681B686A
:101140009A687B681B6822F470229A607B681B682F
:101150009A687B681B6822F440129A603B685B7D4A
:10116000002B08D07B681B685A687B681B6842F4B8
:1011700080625A6007E07B681B685A687B681B685E
:1011800022F480625A603B681B7D002B08D07B688C
:101190001B685A687B681B6842F480525A6007E0FB
:1011A0007B681B685A687B681B6822F480525A600F
:1011B0003B685B68032B2ED0032B40D8012B02D059
:1011C000022B14D03BE07B681B685B697A6812686D
:1011D00023F47F6323F00F0353617B681B68596915
:1011E0003B68DA687B681B680A435A613BE07B68AE
:1011F0001B689B697A68126823F47F6323F00F03EE
:1012000093617B681B6899693B68DA687B681B6837
:101210000A439A6127E07B681B68DB697A68126879
:1012200023F47F6323F00F03D3617B681B68D969C4
:101230003B68DA687B681B680A43DA6113E07B6805
:101240001B681B6A7A68126823F47F6323F00F031C
:1012500013627B681B68196A3B68DA687B681B68E5
:101260000A431A6200BF194BFB607B681B68184A6F
:10127000934209D13B681B68122B05D1FB685B6860
:1012800043F48002FB685A607B681B68104A9342F3
:101290000ED13B681B680F4A934203D03B681B6822
:1012A000112B05D1FB685B6843F40002FB685A60B0
:1012B0007B68002283F83C20002318461437BD4683
:1012C0005DF8047B704700BF01000F000023014060
:1012D000002001401200001080B485B000AF78609B
:1012E00039607B6893F83C30012B01D1022331E057
:1012F0007B68012283F83C20194BFB60FB685B682C
:1013000023F01F02FB685A60FB685A683B681B6841
:101310001A43FB685A60FB685B6823F44042FB6831
:101320005A60FB685A683B685B681A43FB685A60FE
:10133000FB685B6823F47062FB685A60FB685A685C
:101340003B689B681A43FB685A607B68002283F8FD
:101350003C20002318461437BD465DF8047B7047D7
:101360000023014080B485B000AF78607B6803F053
:101370000703FB600C4BDB68BB60BA684FF6FF03EA
:101380001340BB60FB681A02BB68134343F0BF63A2
:1013900043F40033BB60044ABB68D36000BF14371A
:1013A000BD465DF8047B704700ED00E080B400AFFF
:1013B000044BDB681B0A03F007031846BD465DF8C3
:1013C000047B704700ED00E080B483B000AF0346BB
:1013D000FB7197F90730002B0BDBFB7903F01F0241
:1013E000074997F907305B09012000FA02F241F83A
:1013F000232000BF0C37BD465DF8047B704700BF5B
:1014000000E100E080B483B000AF0346FB7197F9C0
:101410000730002B12DBFB7903F01F020A4997F912
:1014200007305B09012000FA02F2203341F8232043
:10143000BFF34F8F00BFBFF36F8F00BF00BF0C37EC
:10144000BD465DF8047B704700E100E080B483B0E6
:1014500000AF03463960FB7197F90730002B0ADBB8
:101460003B68DAB20C4997F907301201D2B20B444B
:1014700083F800230AE03B68DAB20849FB7903F0FD
:101480000F03043B1201D2B20B441A7600BF0C3793
:10149000BD465DF8047B704700E100E000ED00E030
:1014A00080B489B000AFF860B9607A60FB6803F07F
:1014B0000703FB61FB69C3F10703042B28BF042367
:1014C000BB61FB690433062B02D9FB69033B00E0D7
:1014D00000237B614FF0FF32BB6902FA03F3DA436A
:1014E000BB681A407B699A404FF0FF317B6901FA73
:1014F00003F3D9437B680B40134318462437BD469A
:101500005DF8047B7047000080B400AFBFF34F8FDD
:1015100000BF064BDB6803F4E0620449044B13434D
:10152000CB60BFF34F8F00BF00BFFDE700ED00E0D1
:101530000400FA0580B582B000AF78607B68013B9B
:10154000B3F1807F01D301230FE00A4A7B68013B9E
:1015500053600F214FF0FF30FFF778FF054B00225B
:101560009A60044B07221A60002318460837BD46CC
:1015700080BD00BF10E000E080B582B000AF7860B1
:101580007868FFF7EFFE00BF0837BD4680BD80B525
:1015900086B000AF0346B9607A60FB7300237B61BD
:1015A000FFF704FF78617A68B9687869FFF778FF18
:1015B000024697F90F3011461846FFF747FF00BF64
:1015C0001837BD4680BD80B582B000AF0346FB71C1
:1015D00097F907301846FFF7F7FE00BF0837BD46FA
:1015E00080BD80B582B000AF0346FB7197F907302C
:1015F0001846FFF707FF00BF0837BD4680BD80B51E
:1016000000AFFFF781FF80B582B000AF78607868E7
:10161000FFF790FF034618460837BD4680BD80B5EA
:1016200000AFFCF78FFA00BF80BD80B582B000AF7D
:1016300078607B68002B01D1012314E07B681B7963
:10164000DBB2002B05D17B6800225A717868F7F76E
:1016500013F87B6802221A717B6800221A617B688A
:1016600001221A71002318460837BD4680BD80B597
:1016700082B000AF78607B68002B01D101230FE0BE
:101680007B6802221A717868F7F73AF87B680022C3
:101690001A617B6800221A717B6800225A7100234C
:1016A00018460837BD4680BD80B483B000AF78606F
:1016B00039607B685B79012B01D1022340E07B68B4
:1016C00001225A717B6802221A717B681B681968B3
:1016D0003B6803F0100301229A407B681B680A43B1
:1016E0001A603B68002B0FD17B681B681B6803F0F6
:1016F0003C033C2B1DD17B681B685A687B681B68C8
:1017000042F001025A6014E07B681B681B6803F416
:1017100070123B6803F010033C2101FA03F39A4274
:1017200007D17B681B685A687B681B6842F002021D
:101730005A607B6801221A717B6800225A7100236B
:1017400018460C37BD465DF8047B704780B487B0FF
:1017500000AFF860B9607A60FB685B79012B01D15A
:1017600002233CE0FB6801225A71FB6802221A71D5
:10177000FB681B681B687B617B6803F0100340F605
:10178000FE7202FA03F3DB437A6913407B61BB68A4
:101790001A68BB685B6813433B617B6803F0100306
:1017A0003A6902FA03F37A6913437B61FB681B68A9
